:020000040800F2
:1000000000500020CD0F00087D1000087D4300083F
:100010007D1000087D1000087D1000080000000021
:100020000000000000000000000000007D1000083B
:100030007D100008000000007D100008A551000898
:100040007D1000087D1000087D1000087D1000085C
:100050007D1000087D1000087D1000087D1000084C
:100060007D1000087D1000087D1000087D1000083C
:100070007D1000087D100008692A00087D10000826
:100080007D1000087D1000087D1000087D1000081C
:100090007D1000087D1000087D1000087D1000080C
:1000A0007D1000087D1000087D100008692D0008F3
:1000B000752D00087D2D0008892D0008691700089E
:1000C000E91A00086D170008E51A00087D100008FD
:1000D0007D1000089D2A0008D92A00087D1000081C
:1000E0007D1000087D1000087D1000080000000051
:1000F0000000000000000000000000000000000000
:0C01000000000000000000005FF808F1A3
:1001100010B5054C237833B9044810B10448AFF347
:1001200000800121217010BDD405002000000000D6
:10013000C827010808B5064B1BB106480649AFF3AE
:1001400000800648016811B1054A02B1904708BD18
:1001500000000000C8270108D8050020D4050020B1
:100160000000000081F0004102E000BF83F0004386
:1001700030B54FEA41044FEA430594EA050F08BF42
:1001800090EA020F1FBF54EA000C55EA020C7FEA06
:10019000645C7FEA655C00F0E2804FEA5454D4EB83
:1001A0005555B8BF6D420CDD2C4480EA020281EA4D
:1001B000030382EA000083EA010180EA020281EA85
:1001C0000303362D88BF30BD11F0004F4FEA0131D7
:1001D0004FF4801C4CEA113102D0404261EB4101E6
:1001E00013F0004F4FEA03334CEA133302D052426C
:1001F00063EB430394EA050F00F0A780A4F1010428
:10020000D5F1200E0DDB02FA0EFC22FA05F2801861
:1002100041F1000103FA0EF2801843FA05F3594147
:100220000EE0A5F120050EF1200E012A03FA0EFCC6
:1002300028BF4CF0020C43FA05F3C01851EBE371F0
:1002400001F0004507D54FF0000EDCF1000C7EEB0D
:1002500000006EEB0101B1F5801F1BD3B1F5001F4B
:100260000CD349085FEA30004FEA3C0C04F101046A
:100270004FEA445212F5800F80F09A80BCF1004F93
:1002800008BF5FEA500C50F1000041EB045141EA15
:10029000050130BD5FEA4C0C404141EB010111F416
:1002A000801FA4F10104E9D191F0000F04BF0146C1
:1002B0000020B1FA81F308BF2033A3F10B03B3F19F
:1002C00020020CDA0C3208DD02F1140CC2F10C022F
:1002D00001FA0CF021FA02F10CE002F11402D8BF8D
:1002E000C2F1200C01FA02F120FA0CFCDCBF41EA59
:1002F0000C019040E41AA2BF01EB0451294330BD28
:100300006FEA04041F3C1CDA0C340EDC04F1140404
:10031000C4F1200220FA04F001FA02F340EA0300DB
:1003200021FA04F345EA030130BDC4F10C04C4F121
:10033000200220FA02F001FA04F340EA0300294601
:1003400030BD21FA04F0294630BD94F0000F83F44B
:10035000801306BF81F480110134013D4EE77FEA2E
:10036000645C18BF7FEA655C29D094EA050F08BF7A
:1003700090EA020F05D054EA000C04BF194610465B
:1003800030BD91EA030F1EBF0021002030BD5FEA9F
:10039000545C05D14000494128BF41F0004130BDC7
:1003A00014F580043CBF01F5801130BD01F000451B
:1003B00045F0FE4141F470014FF0000030BD7FEA8E
:1003C000645C1ABF194610467FEA655C1CBF0B4689
:1003D000024650EA013406BF52EA033591EA030FA0
:1003E00041F4002130BD00BF90F0000F04BF002198
:1003F000704730B54FF4806404F132044FF00005CB
:100400004FF0000150E700BF90F0000F04BF002143
:10041000704730B54FF4806404F1320410F00045A9
:1004200048BF40424FF000013EE700BF42004FEAA4
:10043000E2014FEA31014FEA02701FBF12F07F4321
:1004400093F07F4F81F06051704792F0000F14BF1E
:1004500093F07F4F704730B54FF4607401F0004562
:1004600021F0004120E700BF50EA010208BF7047B9
:1004700030B54FF000050AE050EA010208BF7047AE
:1004800030B511F0004502D5404261EB41014FF417
:10049000806404F132045FEA915C3FF4DCAE4FF01B
:1004A00003025FEADC0C18BF03325FEADC0C18BF02
:1004B000033202EBDC02C2F1200300FA03FC20FA53
:1004C00002F001FA03FE40EA0E0021FA02F11444A0
:1004D000C1E600BF70B54FF0FF0C4CF4E06C1CEAB5
:1004E00011541DBF1CEA135594EA0C0F95EA0C0F2A
:1004F00000F0DEF82C4481EA030621EA4C5123EA9D
:100500004C5350EA013518BF52EA033541F48011CB
:1005100043F4801338D0A0FB02CE4FF00005E1FB7E
:1005200002E506F00042E0FB03E54FF00006E1FBC8
:1005300003569CF0000F18BF4EF0010EA4F1FF040B
:10054000B6F5007F64F5407404D25FEA4E0E6D414B
:1005500046EB060642EAC62141EA55514FEAC5205C
:1005600040EA5E504FEACE2EB4F1FD0C88BFBCF5D8
:10057000E06F1ED8BEF1004F08BF5FEA500E50F189
:10058000000041EB045170BD06F0004646EA01014F
:1005900040EA020081EA0301B4EB5C04C2BFD4EB81
:1005A0000C0541EA045170BD41F480114FF0000E7A
:1005B000013C00F3AB8014F1360FDEBF002001F0E8
:1005C000004170BDC4F10004203C35DA0C341BDC62
:1005D00004F11404C4F1200500FA05F320FA04F034
:1005E00001FA05F240EA020001F0004221F0004168
:1005F00010EBD37021FA04F642EB06015EEA430EDB
:1006000008BF20EAD37070BDC4F10C04C4F120050A
:1006100000FA04F320FA05F001FA04F240EA0200BD
:1006200001F0004110EBD37041F100015EEA430E8E
:1006300008BF20EAD37070BDC4F1200500FA05F2AE
:100640004EEA020E20FA04F301FA05F243EA02032D
:1006500021FA04F001F0004121FA04F220EA02003C
:1006600000EBD3705EEA430E08BF20EAD37070BD82
:1006700094F0000F0FD101F00046400041EB010162
:1006800011F4801F08BF013CF7D041EA060195F044
:10069000000F18BF704703F00046520043EB0303FE
:1006A00013F4801F08BF013DF7D043EA06037047EB
:1006B00094EA0C0F0CEA135518BF95EA0C0F0CD0F6
:1006C00050EA410618BF52EA4306D1D181EA03013C
:1006D00001F000414FF0000070BD50EA410606BF36
:1006E0001046194652EA430619D094EA0C0F02D17B
:1006F00050EA013613D195EA0C0F05D152EA0336C0
:100700001CBF104619460AD181EA030101F00041DD
:1007100041F0FE4141F470014FF0000070BD41F026
:10072000FE4141F4780170BD70B54FF0FF0C4CF400
:10073000E06C1CEA11541DBF1CEA135594EA0C0F1F
:1007400095EA0C0F00F0A7F8A4EB050481EA030E6C
:1007500052EA03354FEA013100F088804FEA033353
:100760004FF0805545EA131343EA12634FEA022221
:1007700045EA111545EA10654FEA00260EF00041E2
:100780009D4208BF964244F1FD0404F5407402D234
:100790005B084FEA3202B61A65EB03055B084FEAC5
:1007A00032024FF480104FF4002CB6EB020E75EBC2
:1007B000030E22BFB61A754640EA0C005B084FEAEA
:1007C0003202B6EB020E75EB030E22BFB61A754667
:1007D00040EA5C005B084FEA3202B6EB020E75EBB2
:1007E000030E22BFB61A754640EA9C005B084FEA2A
:1007F0003202B6EB020E75EB030E22BFB61A754637
:1008000040EADC0055EA060E18D04FEA051545EA25
:1008100016754FEA06164FEAC30343EA52734FEACE
:10082000C2025FEA1C1CC0D111F4801F0BD141EA47
:1008300000014FF000004FF0004CB6E711F4801FAC
:1008400004BF01430020B4F1FD0C88BFBCF5E06F8C
:100850003FF6AFAEB5EB030C04BFB6EB020C5FEA9C
:10086000500C50F1000041EB045170BD0EF0004EF1
:100870004EEA113114EB5C04C2BFD4EB0C0541EA23
:10088000045170BD41F480114FF0000E013C90E620
:1008900045EA060E8DE60CEA135594EA0C0F08BFE4
:1008A00095EA0C0F3FF43BAF94EA0C0F0AD150EAE3
:1008B00001347FF434AF95EA0C0F7FF425AF104676
:1008C00019462CE795EA0C0F06D152EA03353FF49E
:1008D000FDAE1046194622E750EA410618BF52EA1B
:1008E00043067FF4C5AE50EA41047FF40DAF52EAEF
:1008F00043057FF4EBAE12E74FEA4102B2F1E04369
:1009000024BFB3F5001CDCF1FE5C0DD901F0004CF6
:100910004FEAC0024CEA5070B2F1004F40EB830046
:1009200008BF20F00100704711F0804F21D113F172
:100930003872BCBF01F00040704741F480114FEAAB
:100940005252C2F11802C2F1200C10FA0CF320FA34
:1009500002F018BF40F001004FEAC1234FEAD32351
:1009600003FA0CFC40EA0C0023FA02F34FEA4303BB
:10097000CCE77FEA625307D150EA01331EBF4FF044
:10098000FE4040F44000704701F0004040F0FE405F
:1009900040F40000704700BF80F0004002E000BF5C
:1009A00081F0004142001FBF5FEA410392EA030F5A
:1009B0007FEA226C7FEA236C6AD04FEA1262D2EBA4
:1009C0001363C1BFD218414048404140B8BF5B42A9
:1009D000192B88BF704710F0004F40F4000020F042
:1009E0007F4018BF404211F0004F41F4000121F058
:1009F0007F4118BF494292EA030F3FD0A2F10102A2
:100A000041FA03FC10EB0C00C3F1200301FA03F1DF
:100A100000F0004302D5494260EB4000B0F5000F02
:100A200013D3B0F1807F06D340084FEA310102F1C1
:100A30000102FE2A51D2B1F1004F40EBC25008BF73
:100A400020F0010040EA03007047490040EB00003D
:100A500010F4000FA2F10102EDD1B0FA80FCACF16C
:100A6000080CB2EB0C0200FA0CF0AABF00EBC2506B
:100A700052421843BCBFD0401843704792F0000F59
:100A800081F4000106BF80F400000132013BB5E7AC
:100A90004FEA41037FEA226C18BF7FEA236C21D022
:100AA00092EA030F04D092F0000F08BF0846704787
:100AB00090EA010F1CBF0020704712F07F4F04D155
:100AC000400028BF40F00040704712F100723CBF68
:100AD00000F50000704700F0004343F0FE4040F492
:100AE000000070477FEA226216BF08467FEA236350
:100AF0000146420206BF5FEA412390EA010F40F43B
:100B0000800070474FF0000304E000BF10F0004386
:100B100048BF40425FEA000C08BF704743F096436D
:100B200001464FF000001CE050EA010208BF704788
:100B30004FF000030AE000BF50EA010208BF70470F
:100B400011F0004302D5404261EB41015FEA010C24
:100B500002BF84460146002043F0B64308BFA3F11C
:100B60008053A3F50003BCFA8CF2083AA3EBC253FE
:100B700010DB01FA02FC634400FA02FCC2F120021D
:100B8000BCF1004F20FA02F243EB020008BF20F054
:100B90000100704702F1200201FA02FCC2F12002BA
:100BA00050EA4C0021FA02F243EB020008BF20EAAF
:100BB000DC7070474FF0FF0C1CEAD0521EBF1CEADD
:100BC000D15392EA0C0F93EA0C0F6FD01A4480EACB
:100BD000010C400218BF5FEA41211ED04FF00063B4
:100BE00043EA501043EA5111A0FB01310CF00040E0
:100BF000B1F5000F3EBF490041EAD3715B0040EA06
:100C0000010062F17F02FD2A1DD8B3F1004F40EBD5
:100C1000C25008BF20F00100704790F0000F0CF0A8
:100C2000004C08BF49024CEA502040EA51207F3A6C
:100C3000C2BFD2F1FF0340EAC250704740F4000047
:100C40004FF00003013A5DDC12F1190FDCBF00F038
:100C500000407047C2F10002410021FA02F1C2F1E6
:100C6000200200FA02FC5FEA310040F1000053EA82
:100C70004C0308BF20EADC70704792F0000F00F0D0
:100C8000004C02BF400010F4000F013AF9D040EAD6
:100C90000C0093F0000F01F0004C02BF490011F46A
:100CA000000F013BF9D041EA0C018FE70CEAD15368
:100CB00092EA0C0F18BF93EA0C0F0AD030F0004CE8
:100CC00018BF31F0004CD8D180EA010000F000409C
:100CD000704790F0000F17BF90F0004F084691F05A
:100CE000000F91F0004F14D092EA0C0F01D1420294
:100CF0000FD193EA0C0F03D14B0218BF084608D15D
:100D000080EA010000F0004040F0FE4040F40000A6
:100D1000704740F0FE4040F4400070474FF0FF0C39
:100D20001CEAD0521EBF1CEAD15392EA0C0F93EA80
:100D30000C0F69D0A2EB030280EA010C49024FEAD2
:100D4000402037D04FF0805343EA111143EA10138B
:100D50000CF000408B4238BF5B0042F17D024FF443
:100D6000000C8B4224BF5B1A40EA0C00B3EB510F1E
:100D700024BFA3EB510340EA5C00B3EB910F24BF07
:100D8000A3EB910340EA9C00B3EBD10F24BFA3EB8C
:100D9000D10340EADC001B0118BF5FEA1C1CE0D154
:100DA000FD2A3FF650AF8B4240EBC25008BF20F007
:100DB000010070470CF0004C4CEA50207F32C2BF5B
:100DC000D2F1FF0340EAC250704740F400004FF0F8
:100DD0000003013A37E792F0000F00F0004C02BF29
:100DE000400010F4000F013AF9D040EA0C0093F0F3
:100DF000000F01F0004C02BF490011F4000F013B4D
:100E0000F9D041EA0C0195E70CEAD15392EA0C0FB4
:100E100008D142027FF47DAF93EA0C0F7FF470AFEC
:100E2000084676E793EA0C0F04D14B023FF44CAF2F
:100E300008466EE730F0004C18BF31F0004CCAD1C4
:100E400030F000427FF45CAF31F000437FF43CAF00
:100E50005FE700BF4FF0FF3C06E000BF4FF0010C22
:100E600002E000BF4FF0010C4DF804CD4FEA400204
:100E70004FEA41037FEA226C18BF7FEA236C11D04E
:100E800001B052EA530C18BF90EA010F58BFB2EB01
:100E9000030088BFC81738BF6FEAE17018BF40F081
:100EA000010070477FEA226C02D15FEA402C05D135
:100EB0007FEA236CE4D15FEA412CE1D05DF8040BBA
:100EC000704700BF844608466146FFE70FB5FFF74D
:100ED000C9FF002848BF10F1000F0FBD4DF808ED05
:100EE000FFF7F4FF0CBF012000205DF808FB00BFF6
:100EF0004DF808EDFFF7EAFF34BF012000205DF850
:100F000008FB00BF4DF808EDFFF7E0FF94BF01209C
:100F100000205DF808FB00BF4DF808EDFFF7D2FF99
:100F200094BF012000205DF808FB00BF4DF808EDDC
:100F3000FFF7C8FF34BF012000205DF808FB00BFA9
:100F40004FEA4002B2F1FE4F0FD34FF09E03B3EBD6
:100F500012620DD94FEA002343F0004310F0004F16
:100F600023FA02F018BF404270474FF0000070476C
:100F700012F1610F01D1420205D110F0004008BF0B
:100F80006FF0004070474FF00000704742000ED2F3
:100F9000B2F1FE4F0BD34FF09E03B3EB126209D4B4
:100FA0004FEA002343F0004323FA02F070474FF06A
:100FB0000000704712F1610F01D1420202D14FF0DF
:100FC000FF3070474FF00000704700BF1D481E49BA
:100FD000026800608A4200F01F80002100F004B81F
:100FE0001A4B5B584350043119481A4B42189A4225
:100FF000FFF4F6AF184A00F003B8002342F8043BB0
:10100000164B9A42FFF4F9AF0AF06CF80DF0C2F8F3
:1010100003F0AEF9FFF7FEBF114E124830601248E0
:10102000016821F070610160410201600F4C1820DD
:1010300020600F490F4808600F48D0F800D0406882
:1010400000470000F04F0020EFBEADDEEC270108A6
:1010500000000020D4050020D4050020881F0020B7
:10106000181002400900000004000140140C014067
:10107000000C01404434434400F0FF1FFFF7FEBF63
:10108000064B187820B1012806D14FF4805201E0B8
:101090004FF4006202490A80704700BFF00500204B
:1010A0000400002007B5232004F0AFF86820752164
:1010B00001220DF1070300F0F3FB30B19DF80700AA
:1010C000B0F16803594251EB03000EBD13B506227F
:1010D000044643216B46682000F0E2FB9DF80020A7
:1010E0009DF8013043EA022001B2042391FBF3F2A0
:1010F0009DF802009DF80310228041EA002210B200
:1011000090FBF3F19DF805209DF80400618042EA10
:10111000002108B290FBF3F3A3801CBD13B5062297
:1011200004463B216B46682000F0BAFB9DF8002086
:101130009DF801309DF8021043EA02209DF803203B
:10114000208042EA01239DF804009DF80510638089
:1011500041EA0022A2801CBD07B5204A02204FF4BC
:101160000053ADF804308DF8070013681C480421C3
:1011700083428DF8061001D11A4803E01A498B42C8
:1011800003D11A4801A900F05DFD6B21802268207F
:1011900000F04AFC052004F038F8192100226820EC
:1011A00000F042FC6B210322682000F03DFC372157
:1011B0000222682000F038FC0D4A1A2168201278BB
:1011C00000F032FC1B211822682000F02DFC682062
:1011D0001C21102200F028FC0EBD00BF840100205D
:1011E00000127A00000C0140001BB7000010014003
:1011F0000000002030B585B00446FFF753FF0028FB
:1012000041D006210A46682002AB00F049FB9DF858
:101210000B309DF80D5003F0010105F001004A006C
:1012200042EA80059DF8090000F001031D4307D044
:10123000012D164801D1002318E0022D0CD114E035
:101240000C21682001220DF1070300F029FB9DF815
:10125000071011F00F0203D1052004F049F806E051
:10126000042A0A4801D1057001E0012303700748F0
:1012700007490378074A2160002B14BF6E216F21B4
:1012800062602172012005B030BD00BFF005002072
:10129000811000081D11000838B505460C46FFF7FF
:1012A00001FF28B3134B14481449142C2B606860B9
:1012B000E960134B15D004D8052C16D00A2C0ED19A
:1012C00011E0BC2C08D0B4F5807F03D0622C06D18D
:1012D00002220BE0002209E00120187038BD032231
:1012E00004E0042202E0052200E006221A70012038
:1012F00038BD00BF59110008CD10000819449231C3
:1013000000000020044B054903EB4000427831F80F
:10131000123098B2704700BFC4140020BE140020E1
:1013200070B5424B04221A70414A424D11782E6822
:10133000414D4C1CE4B2AE4290B05970147004D1CF
:1013400005259D70DC708B1C1370007830B1384C13
:10135000364922780871551C4A712570344D37483A
:101360000AF0A8FE297836480024364B01298CBFA4
:1013700080222246069008914FF480602021059338
:101380000A924FF480734FF400520C900D912B4849
:1013900005A90B930E92079409940F940AF002FF8B
:1013A000264801210AF02BFF2B784FF46022012BF5
:1013B00094BF0020012001218DF804008DF8051054
:1013C000214869460094029203948DF810300AF087
:1013D0000FF8174B1878A0420AD914491A4811F887
:1013E00014100134E4B2224603230AF052F8F0E765
:1013F000154801210AF029F8134801210AF01CF8C8
:1014000011480AF02BF810480AF02DF80028FAD1FC
:101410000D480AF02CF80C480AF02EF80028FAD1F2
:10142000094801210AF02CF810B070BDC414002046
:10143000F105002084010020001BB70008000240D5
:10144000BE1400204C240140002401402DE9F84F37
:101450009C4C2068838A9BB213F0010239D001882A
:1014600021F400631A04110C018001210AF000FE2E
:10147000954A964B117800201870D9B1944803789A
:101480001BB9944A1178FF2914D1012303709248A3
:101490000278022A06D18B490B68188882B242F47E
:1014A000006119808D4B87481978006801220AF085
:1014B000F9FD2FE18948834B0178002218680AF072
:1014C000F1FD844A1178FF2900F02481FF207F4B31
:1014D000DEE003F00201C9B200293DD0BFF35F8F07
:1014E0007D4D2E78012E354616D177490B789BB16C
:1014F00077490B7883B111460AF0BAFDBFF35F8FCD
:1015000020683146038B0AF0A7FD754A20681670E3
:101510004FF480613246FBE0038BBFF35F8F6E496F
:101520000A78022A09D1684B1A7832B1684B1A78C6
:101530001AB100210AF09CFDE5E00978032907D1E2
:10154000614B1A7822B162490B78002B40F0DD80A4
:101550004FF480610122DBE003F00406F6B2002EB6
:1015600071D0594BDFF878811A78012688F800602D
:10157000574B002A4DD01A78002A4AD0564D2F7862
:10158000524D022F574F29D90AF072FD206895F865
:101590000090D7F800A00AF082FD4FFA89FB0AF804
:1015A0000B0009EB06003146287020680AF054FD54
:1015B000206888F800603F6895F800800AF06FFDA9
:1015C0004FFA88F907F80900B04420684FF48061A9
:1015D000324685F800800AF057FD2BE031460AF0CC
:1015E0003BFD20682E78D7F800800AF058FD4FFAAE
:1015F00086F9731C08F80900D9B220684FFA81F8FF
:101600003F6829700AF04BFD033607F808002E707A
:1016100010E01B78012113B9334A13782BB10AF07B
:101620001BFD2A480278511C03E00AF009FD2848F6
:1016300001210170234A11680B8803F4807082B283
:10164000002AF9D166E003F040010F461F4D09B3AF
:10165000244B2F78D3F800800AF021FD4FFA87F948
:1016600008F80900781CC1B229701B4D4FB22A78C6
:101670000337BA4205D120684FF4806132460AF040
:1016800003FD124B28781A7851B2884242D1501C7F
:1016900018703FE01B063DD52B785EB2721C27D038
:1016A000124901330A682B70915D0AF0F6FC0A4872
:1016B00095F90020017891422CD120684FF4806187
:1016C0003A4625E008060020050600200406002012
:1016D000FC050020F6050020F70500200D0600207F
:1016E000F5050020F8050020F40500200006002084
:1016F000154A297011780AF0D0FC1448017811B904
:10170000134B1A7832B9134800684FF480610022F5
:101710000AF0BAFC0E4A104B117893F900004A1CEB
:1017200090420ED10D4B0E49187800220A7028B154
:10173000084908684FF440710AF0A6FC094B0022E2
:101740001A70BDE8F88F00BFF605002005060020DE
:10175000F70500200806002004060020F5050020FB
:10176000FC0500200C060020FFF770BEFFF76EBEE0
:10177000F0B5484C89B04FF440651C23074602265B
:10178000204602A9ADF808508DF80A308DF80B609C
:1017900000F058FA4048142107608DF80E102046DA
:1017A00003A9ADF80C508DF80F6000F04BFA2561DD
:1017B0000825384CA268520503D40A2003F01AFD0C
:1017C000F7E74FF480660A20666103F013FD6F1E91
:1017D0000A20266103F00EFD17F0FF05E9D14FF452
:1017E000006767610A2003F005FD66610A2003F0C7
:1017F00001FD26610A2003F0FDFC022027611C2167
:101800008DF80F002046244C4FF440638DF80E10E5
:1018100003A9ADF80C3000F015FA20680AF072FB4D
:1018200004A80AF0F3FB20682A464FF440710AF03E
:101830002BFC1A484FF480434BF6FF7204900121B1
:101840002068ADF81C30ADF81620ADF814500AF041
:10185000EBFB04A920680AF06FFB4FF4A06009F0CD
:1018600065FE2221012201A88DF804108DF8055093
:101870008DF806508DF8072009F062FE212301A89B
:101880002E468DF804308DF8055009F059FE09B048
:10189000F0BD00BF000C014008060020801A0600C1
:1018A00010B54000244CC0B220702448244C017074
:1018B00000212170234C01202070234C2360234CF5
:1018C0002360234B1A70234A107023480170234968
:1018D0000868838803F4007291B2A1B9038803F405
:1018E000807291B241B9038803F4007291B2002969
:1018F000F9D101210AF0A4FB18484FF440710068A7
:1019000001220AF0C1FB47F23053124A117811B19B
:10191000013BFAD100E053B911490A88501C83B247
:101920000B800E490868FFF723FF002010BD0A4B0B
:10193000187880F0010010BD0D060020F60500208B
:10194000F405002005060020F80500200006002010
:10195000F70500200C060020FD05002008060020E9
:10196000F205002010B54000244CC0B2207024487D
:10197000244C017024490120087000212170234C5F
:101980002360234C2360234B1A70234A1070234892
:10199000017023490868838803F4007291B2A1B9E9
:1019A000038803F4807291B241B9038803F4007292
:1019B00091B20029F9D101210AF042FB18484FF4F5
:1019C0004071006801220AF05FFB47F23053124A6F
:1019D000117811B1013BFAD100E053B911490A88DD
:1019E000501C83B20B800E490868FFF7C1FE00202F
:1019F00010BD0A4B187880F0010010BD0D060020C4
:101A0000F605002005060020F40500200006002051
:101A1000F8050020F70500200C060020FD05002039
:101A200008060020F205002007B502AB03F8012DDF
:101A30000122FFF797FF0EBD274B37B51868818A43
:101A40008AB20192019B13F4706F02D0234A0121E4
:101A50001170019B13F4E06F31D04FF480610022CC
:101A6000038B0AF011FB0198810528D41A4D2868D0
:101A7000018801F4007293B20BBB048804F48071F6
:101A80008CB29CB1028802F4807399B20029F9D11A
:101A900001210AF0E1FA10480068028802F400739C
:101AA00099B20029F9D1FFF763FE08E001210AF09D
:101AB000D3FA28684FF4407122460AF0E5FA064846
:101AC0000268938A23F470610804030C044993822A
:101AD00000220A703EBD00BF08060020FD05002060
:101AE0000C060020FFF7A8BFFFF7A6BF014B188820
:101AF00080B27047F2050020F8B5134B05469B896C
:101B00000E461446ECB116B116F8017B00E0FF2733
:101B10000D48022109F066FC0028F9D00A48394630
:101B200009F05BFC0848012109F05CFC0028F9D0B1
:101B3000054809F054FCC0B20DB105F8010B013C99
:101B4000E0E70120F8BD00BF003800402DE9F04774
:101B5000012188B04FF480400AF0A8F9374C0121E8
:101B60004FF480400AF0BAF903214FF420401823C3
:101B7000ADF800008DF80310204669468DF802305C
:101B80004FF0040800F05EF82D4E4FF480422046DE
:101B90006946ADF800204FF480554FF0100A8DF8DB
:101BA000028000F04FF869462046ADF800508DF8ED
:101BB00002A000F047F8304609F0B2FB07214FF4CD
:101BC000007000230222ADF81600ADF81C104FF093
:101BD0000109304603A94FF48277ADF80C30ADF817
:101BE0001030ADF81A30ADF81220ADF80E70ADF827
:101BF00014901F46ADF818A009F0C4FB30464946C2
:101C000009F0DFFB9F238DF804308DF805708DF807
:101C100006708DF807700DEB08014246656102A859
:101C2000FFF76AFF25619DF80900B0F1EF014A4214
:101C300052EB010008B0BDE8F08700BF000C014086
:101C4000003800402DE9F0410F88002347FA03F2E5
:101C5000D2072DD58A7803F00705DC08AD0012F015
:101C6000100F18BF91F803C002F00F0618BF46EA24
:101C70000C064FF00F0C0CFA05FC06FA05F550F8AF
:101C80002480282A28EA0C0C45EA0C0540F8245048
:101C900006D1012202FA03F2C46824EA020206E035
:101CA000482A05D1012202FA03F2C4682243C26025
:101CB0000133102BCAD1BDE8F08100002DE9F843B3
:101CC0000446C3796278002B14BF0220002002B1C1
:101CD00001303C49002551F82090A8462F462E4659
:101CE00039F805304FF6FF729342D8B267D0E178E9
:101CF00011B1821E012A5FD9217911B1021F032A75
:101D00005AD9217A09B1814256D0190A022905D13E
:101D10002278002A14BF022100210CE0012901D100
:101D2000617808E0032906D1A17821B12378002B3E
:101D30000CBF03210021637933B1E27922B9A0F10C
:101D40000803012B98BF0521A27922B1E37913B9C9
:101D5000021F032A27D9012902D100F055FA2BE0EE
:101D6000022904D1F1B200F019FA013624E0032966
:101D700002D100F063F91FE0042912D16289124BED
:101D80004FEA0010B2F5FA7F18445FFA88F1E38950
:101D900002D900F0E3F801E000F0F6F808F10108DC
:101DA0000AE0052908D10849A28901EB0010238A1D
:101DB000F9B200F0FFF8013702351C2D90D1BDE8D3
:101DC000F88300BFF0FE00086CFF0008074BA1F588
:101DD0007A7153F82000838802684B434FF47A707D
:101DE00093FBF0F18BB21380704700BF1006002008
:101DF000024B53F820000268118070471006002043
:101E00002DE9F04F044647488E46057889B0691C95
:101E10000170914611462068724601930C2600F02D
:101E2000F1FEA268182303A96E4360684FF0020A0E
:101E3000ADF80C208DF80E308DF80FA0FFF702FFE3
:101E400004A8394F256894F80CB009F06EFD702095
:101E5000019BADF81000012100224FF4807007EBC8
:101E60000608ADF81210ADF81420ADF81630ADF834
:101E700018A0ADF81C00BBF10C0F2BD8DFE80BF05D
:101E8000072A2A2A102A2A2A192A2A2A2200284618
:101E900004A909F043FC2846082109F07BFD19E05C
:101EA000284604A909F07EFC2846082109F07AFD9D
:101EB00010E0284604A909F0B9FC2846082109F0D9
:101EC0007BFD07E0284604A909F0F2FC284608211A
:101ED00009F07AFDA17B19B12068012109F043FDC9
:101EE0002068012109F033FD237B0C2B14D8DFE897
:101EF00003F0071313130A1313130D131313100016
:101F00002268343207E02268383204E022683C322A
:101F100001E022684032BA51A8F80490404609B066
:101F2000BDE8F08F0E0600206006002008B5044BC7
:101F300053F820301BB10B2801D89A68904708BD90
:101F400010060020044B53F820201AB107289CBF2C
:101F500012681180704700BF4006002010B50C4683
:101F60000649B1FBF2F292B20821FFF749FF044B98
:101F7000044943F82400816010BD00BF00127A00BC
:101F800010060020CD1D000810B50C460649B1FB17
:101F9000F2F292B20121FFF733FF044B044943F8F8
:101FA0002400816010BD00BF40420F0010060020D9
:101FB000F11D000810B50C46054991FBF2F292B2F2
:101FC0000121FFF71DFF034B43F8240010BD00BFA4
:101FD00040420F004006002010B50B4B1A785C6998
:101FE00032B901221A7059602068217B022207E071
:101FF000586899600022091A19821A702068217B9A
:10200000BDE8104000F08CB8F00600207FB5044613
:1020100001A80D46164609F092FC00200123ADF8F8
:102020000A00ADF80C0001A92046ADF80450ADF847
:102030000660ADF8083009F003FD7FBDF7B5144D1B
:10204000144F060174190021182238460CF09AF931
:10205000A368E27B022160688DF8071001A9ADF842
:1020600004308DF806207C61FFF7ECFD7059217B70
:102070000022FFF7CBFF204601224FF6FF7100F050
:10208000E3FD20460021044A00F09EFDFEBD00BF96
:102090006CFF0008F0060020D91F0008014B188AC9
:1020A000704700BFF00600200D4A0E48136811600B
:1020B0000360C91A40F68C220B4B91421A7807DD57
:1020C000032A03D9094A1178481C1070002005E042
:1020D0000B2A9CBF064820F81210501C187070473D
:1020E000D0070020C8070020C4070020CC0700202C
:1020F0000A070020034B044918780A78801A18BF91
:1021000001207047CC07002008070020024B03483D
:102110001A780270704700BFCC0700200807002023
:102120007FB5044601A80D46164609F008FC0020BC
:1021300003210123ADF80A00ADF80C10204601A9D7
:10214000ADF80450ADF80660ADF8083009F078FC41
:102150007FBD00000F4B142210B502FB00308278C7
:10216000036932B94160012181701868197B02222C
:102170000BE044688160084A091B4478C16022F87A
:102180001410002282701868197BBDE81040FFF718
:10219000C7BF00BF240700200A0700202DE9F34134
:1021A00014220D466A43154F4FEA0018144908EBF4
:1021B000070401268B188E54E17BA2685D701C61B8
:1021C000606802238DF8061001A98DF80730ADF87C
:1021D0000420FFF737FD58F80700217B0022FFF7A6
:1021E0009FFF204632464FF6FF7100F02DFD20463E
:1021F0002946044A00F0E8FCBDE8FC816CFF0008B9
:102200002407002055210008F7B5124E0701BC191C
:10221000A168114B0025E27B1D701C6160680223E0
:10222000ADF8041001A98DF807308DF80620FFF7EE
:1022300009FDB859217B2A46FFF772FF204601228B
:102240004FF6FF7100F000FD20462946034A00F0DA
:10225000BBFCFEBD6CFF000824070020A92000087D
:10226000014B33F8100070470A0700204171704796
:10227000426A806A131A594251EB030070477FB5D6
:10228000044601A80D46164609F059FB002001231B
:10229000ADF80A00ADF80C0001A92046ADF80450D5
:1022A000ADF80660ADF8083009F0CAFB7FBD437990
:1022B00013F0010107D00269C169006A531E0A1AAE
:1022C0001A40D0B2704708467047437910B513F0F2
:1022D000010104460DD0FFF7EAFF58B1226A606998
:1022E000E368805C0132B2FBF3F103FB112222624E
:1022F00010BD084610BD43799A070AD5436A826922
:10230000D154416A03694A1CB2FBF3F103FB112269
:10231000426270478379012B03D1D1F1010138BFAB
:102320000021D0F834014268836809B11361704715
:102330005361704707B5034699684822ADF8041009
:102340000223406801A98DF806208DF80730FFF7B9
:1023500079FC0EBD2DE9F74391464FF412724243CA
:102360001F463B4B0646D41808B93A4802E00128FC
:1023700004D1394820631030C4F83401374D0020AF
:10238000D55003224FF001086271D4F8342184F84B
:10239000388284F83C0284F8390284F84662E162AB
:1023A0004FF48071E1602161916804F1340304F518
:1023B0009C75636120621023E061A561A062606288
:1023C000A4F84202A4F84402ADF80410506801A930
:1023D000C4F80890A77102258DF806308DF80750D3
:1023E000FFF730FC206BFFF7A5FF41462046FFF7C3
:1023F00091FF322002F009FF1948D4F834810368B4
:102400001846B0FBF9F1B1F5803F03D30128F8D9A4
:102410004008F6E7134A4046B3FBF2F5EAB289B248
:1024200000F012FC404631460F4A00F0CDFB256B10
:10243000012F14BF022200222868297BFFF71FFF0B
:1024400028463146094A00F0BFFB2046BDE8FE831E
:10245000CC140020ACFF0008CCFF00083CFF0008B3
:102460008801002040420F00892600080D25000841
:1024700003460A4690F84602D96A9B79FFF76ABF7D
:1024800010B590F83C220446AAB9836A416A994281
:1024900025D080692169C05C01338B42A36228BFCB
:1024A000A26242000A2342F4007084F83D32A4F88C
:1024B0003E02012311E090F93D3273B1B0F83E12B3
:1024C0004A08A0F83E2201F00101FFF723FF94F82B
:1024D0003D02431E84F83D3210BD84F83C3210BDED
:1024E00090F83B3210B583B990F83A3290F839221F
:1024F00093420AD2012101FA03F1B0F840420133BC
:102500002143A0F84012DBB2F2E710BD2C4B10B50E
:102510004FF4127404FB00346079C1074ED594F86F
:10252000381219B3236B0021186809F057FA94F890
:102530003C1221B1B4F84202421CA4F84222236B9F
:10254000A2791868197B012A0CBF02220022FFF72A
:1025500096FE0020012184F83B1284F8390284F8A9
:102560003A02A4F8400284F8380210BD94F83B22E5
:102570002046012A04BF94F8392284F83A22FFF752
:10258000AFFF94F83B02236B50B90120A27984F885
:102590003B021868197B012A0CBF0222002209E0C5
:1025A000002184F83B12A2791868197B012A14BF14
:1025B00002220022BDE81040FFF761BE10BD00BF3F
:1025C000CC14002090F83B1200230122012980F84E
:1025D000393280F838220BD180F83B32036B827994
:1025E000197B1868012A14BF02220022FFF747BE98
:1025F0007047427908B5D10703461ED5B0F84002AE
:1026000000F400718AB20AB9C20705D4B3F84422B3
:10261000501CA3F8440208BDD96AC0F3470009B1B1
:10262000884708BDDA6959698854D869DA68411C55
:10263000B1FBF2F002FB1011D96108BD10B590F8A2
:1026400038320446002B1ED190F839124A1CD3B2FE
:10265000092B80F8393203D1BDE81040FFF740BFA5
:102660000A2B10D190F83B0228B9B4F8401241F07F
:102670000102A4F840222046FFF7BBFF2046BDE838
:102680001040FFF79FBF10BD064B10B54FF41274FA
:1026900004FB00342046FFF7F3FE2046BDE810405F
:1026A000FFF7CCBFCC140020436B13B190F844006B
:1026B0007047826A406A111A4B4253EB010070471F
:1026C0001FB58368002100934379ADF8041003F02F
:1026D000040101F0FF0231B14FF40051ADF80610D2
:1026E0004FF4806201E0ADF80620ADF8082000222A
:1026F00013F0010118BF0421ADF80C209A07ADF8C2
:102700000A1005D5BDF80A3043F00802ADF80A20DA
:10271000006D694609F04CFA05B000BD4171FFF744
:10272000CFBF8160FFF7CCBF026B03691AB151685C
:10273000013B006C02E0C169006A013B0A1A1A40C1
:10274000D0B27047026B034610B5406942B11A6CB3
:10275000D9688C1A013A18BF1146005D196410BD82
:10276000196ADA68405C0131B1FBF2F402FB141122
:10277000196210BD2DE9F0411E464B4B8CB09842BA
:102780008846174604D11046314600F0C7F807E0E6
:102790004649884240F083801046314600F014F9E3
:1027A000002587600562C56185624562C0F82C809E
:1027B000467185710446FFF783FF01A809F012FDF9
:1027C000E06C802701904FF48052F0070A920B953D
:1027D000059507950697089527D5206BD0B1E36836
:1027E00003956569202104930991029509F062FC23
:1027F000206B01A909F0D6FC206B012109F0FFFC38
:10280000206D4021012209F051FA206B09F00CFDE6
:1028100020640AE0206D40F2255109F050FA206D45
:1028200040F22551012209F027FA01A809F0DAFC4B
:10283000A06C002580274FF48052B10701900A92C6
:102840000B95059507950697089523D5606BD8B12C
:102850002369102104930391099509F02BFC606B07
:1028600001A909F09FFC0122606B022109F0D2FC52
:10287000606B294609F0D6FC606B39464560012241
:10288000206D09F013FA05E0206D40F22771012256
:1028900009F0F2F9206D012109F0E2F900E00024CD
:1028A00020460CB0BDE8F0810038014000440040F3
:1028B000836A8169426BC918D160416A994203D920
:1028C000CB1A5360816204E00169CB1A5360002285
:1028D0008262002180F84410406B012109F08FBC16
:1028E00010B5426A8469A154416A02690131B1FBA1
:1028F000F2F402FB1411426B416232B11368DB0740
:102900000BD4BDE81040FFF7D3BF006D40F2277134
:102910000122BDE8104009F0AFB910BD234B13B53B
:10292000234A986023481A6058614FF48072224805
:102930000C462249DA601A61214A9961011D186525
:102940009964D9641A630121143A4FF480405A63A0
:1029500009F0A0FA022318214FF40070A2078DF8A5
:102960000330ADF800008DF8021003D51548694614
:10297000FFF768F948234FF480628DF80230E307CF
:10298000ADF8002003D50F486946FFF75BF90E202C
:1029900001218DF8040001A88DF805108DF80610AE
:1029A0008DF8071008F0CCFD00481CBD940A0020EB
:1029B00054FF0008D407002000380140140900200B
:1029C0005800024000080140214B224A13B598608C
:1029D0000C46802040211A60D86019611E4A1F49A8
:1029E0001F485A6198610A1D19654FF40030012192
:1029F0009A64DA6409F05AFA042002231821ADF827
:102A00000000A0078DF803308DF8021003D515489B
:102A10006946FFF717F908224823E107ADF80020BF
:102A20008DF8023003D50F486946FFF70BF92620D1
:102A300001218DF80400022201A88DF805108DF8FF
:102A400006208DF8071008F07BFD01481CBD00BF73
:102A5000E80A002054FF0008140A00200044004047
:102A6000D40800200008014010B50B4C4FF4005072
:102A700009F0DEFB0021606B09F0C1FB626AA36A0A
:102A80009A4204D02046BDE81040FFF711BF012054
:102A900084F8440010BD00BF940A00200D4B186D4F
:102AA000028802F080018AB29AB19A6A596A8A420F
:102AB0000AD09969895C013281801969B2FBF1F011
:102AC00001FB10229A62704740F22771002209F040
:102AD000D3B87047940A00201C4B10B51A6D1488A7
:102AE000A4B204F0200188B290B1D96A19B19388D8
:102AF00098B288470CE09288D9695869D2B242549A
:102B0000D869DA68411CB1FBF2F002FB1011D961FF
:102B100004F08004A4B2C4B10C4B9A6A586A824291
:102B20000BD09869196D805C013288801969B2FBFD
:102B3000F1F001FB10229A6210BD186D40F227716E
:102B40000022BDE8104009F097B810BDE80A002047
:102B500030B500240E4D55F82450854202D0013482
:102B6000E4B2F7E700200B4D35F810508D4202D04B
:102B7000451CE8B2F7E704EB8000C0B20F2805D887
:102B8000054C04EB001083600171027330BD00BF7F
:102B90004C0001085C0001083C0B00200C2912D8F5
:102BA000DFE801F007111111091111110B111111B9
:102BB0000D00022104E0042102E0082100E01021C0
:102BC000012208F0DEBE704738B504460D461346B4
:102BD000217B00682A46FFF7BBFF2068217BBDE808
:102BE0003840FFF7DBBF07B58DF804000120002354
:102BF0008DF806008DF8070001A88DF8053008F063
:102C00009FFC0EBD7FB5044601A80D46164608F090
:102C100083FE0B4B0B485E4301680023B1FBF6F2C9
:102C2000013D561E204601A9ADF80850ADF80460DC
:102C3000ADF80A30ADF8063008F026FD7FBD00BFC4
:102C400040420F008801002010B504460068FFF7DD
:102C5000D9FF2068012108F07AFE607BBDE81040B2
:102C6000FFF7C1BF00230C4A52F82320824202D052
:102C70000133DBB2F7E70022084830F8120088423F
:102C800002D0501CC2B2F7E703EB82030449DAB268
:102C900001EB0210704700BF4C0001085C00010806
:102CA0003C0B002070B5044600262E4B9D5D95B967
:102CB0000221204608F06DFF01284FD12046022155
:102CC00008F072FF29462046FFF7CCFF0546204654
:102CD00008F052FF3DE0042D12D12046294608F0AD
:102CE00058FF01283AD12046294608F05DFF2946C1
:102CF0002046FFF7B7FF0546204608F040FF28E0D2
:102D0000082D12D12046294608F043FF012825D17D
:102D10002046294608F048FF29462046FFF7A2FF33
:102D20000546204608F02EFF13E00C2D16D1102189
:102D3000204608F02EFF012810D12046102108F06F
:102D400033FF29462046FFF78DFF0546204608F051
:102D50001CFFAA6801460AB1287B90470236082E5C
:102D6000A3D170BD5C0001080148FFF79BBF00BF05
:102D7000002C01404FF08040FFF794BF0148FFF75F
:102D800091BF00BF000400400148FFF78BBF00BFA8
:102D900000080040024800214FF480720BF0F2BAA4
:102DA0003C0B002010B5FDF7B1FE0A49FDF702FF0C
:102DB0000949FDF7B3FF094B044618680078FDF791
:102DC000A5FE01462046FDF7F5FEFEF7DFF880B2CE
:102DD00010BD00BF3333534000F07F45500C00203E
:102DE00038B50D4C00202578FEF78CFA0B4A05F01B
:102DF000070322F813000135002325701846D15A25
:102E000002334018102B80B2F9D1C008FFF7CAFF77
:102E1000034A107038BD00BF3C0C00203E0C00205F
:102E20005C190020074B084A19781088884207D39C
:102E3000064B1A68907888428CBF002001207047AA
:102E4000002070475C1900205E190020500C002003
:102E500038B5114B2024186000250020FEF752FAE7
:102E60002D180A2002F0D1F9013CF6D1C5F34F101C
:102E7000FFF798FF084901230A6851786418A042B7
:102E800002D30133062BF9D10448927803705343DF
:102E900003490B8038BD00BF500C0020010000200A
:102EA0005E1900202DE9F04F0446008885B048B92E
:102EB000B4F9023043B9B4F90420D2F1010138BFAA
:102EC000002102E0002100E0014611F0010377D16A
:102ED0003D4D00B22B7000F0BBFD0646B4F9020078
:102EE00000F0B6FD0546B4F9040000F0B1FD04465B
:102EF000304609F0A7F90746304609F017FA804630
:102F0000284609F09FF90646284609F00FFA0546BB
:102F1000204609F097F98246204609F007FA39461B
:102F200081465046FDF746FE394683464846FDF742
:102F300041FE514601904046FDF73CFE4946029055
:102F40004046FDF737FE314603905046FDF732FE0E
:102F50001E4C4946206006F10040FDF72BFE294635
:102F60006060A5600298FDF725FE01460198FDF717
:102F700019FD2946E0600398FDF71CFE01465846FE
:102F8000FDF70EFD3146206108F10040FDF712FE0D
:102F9000294660615846FDF70DFE01460398FDF78E
:102FA000FFFC2946A0610198FDF704FE0146029846
:102FB000FDF7F8FC3946E0613046FDF7FBFD206285
:102FC00005B0BDE8F08F00BF02000020540C0020C7
:102FD0002DE9F8434D4B0C460168013A1960808891
:102FE0009880072A30D8DFE802F004080F14191E71
:102FF0002226188820805A8803E0598821801A8860
:10300000524262809A881EE01988484220805A887D
:10301000F6E75988484220801A88F2E71988484222
:10302000208058880CE05A882280188808E0198887
:1030300021805A8803E05988484220801A885042EB
:1030400060809B885A42A280314B1A78002A5AD15C
:10305000B4F90000FDF75AFD8046B4F90200FDF70F
:1030600055FD0746B4F90400FDF750FD294D06460D
:1030700029684046FDF79EFDE96881463846FDF720
:1030800099FD01464846FDF78DFCA9698146304609
:10309000FDF790FD01464846FDF784FC09F006F96E
:1030A000696820804046FDF785FD296981463846DC
:1030B000FDF780FD01464846FDF774FCE96981464D
:1030C0003046FDF777FD01464846FDF76BFC09F0F9
:1030D000EDF8A96860804046FDF76CFD696980469F
:1030E0003846FDF767FD01464046FDF75BFC296A5F
:1030F00007463046FDF75EFD01463846FDF752FCB7
:1031000009F0D4F8A080BDE8F88300BF780C002057
:1031100002000020540C002070B5124D06462B789A
:10312000114C9BB102F060F82268B318984218D392
:103130000021297002F058F820600C4802780AB18A
:10314000531E03700A480121017070BD02F04CF853
:1031500021683231884204D30120287002F044F8FB
:10316000206070BD7E0C00208C0C0020810C0020A3
:103170007F0C002037B58DF805101F498DF80730FA
:103180000B788DF8040002A88DF80620C21812F8FA
:10319000044C0D46443CE0B20A2828D81749022BBB
:1031A00031F8104003D814B12046FFF7B5FF2B7853
:1031B000022B0BD9124D2D6802F016F8021B954216
:1031C00004D20D490F4B0020087018700E48027889
:1031D0000146012A00D074B9074B1878022801D89B
:1031E000421C1A7000230B7008490B7003E0322454
:1031F000022BD9D9DBE73EBD800C0020640001081A
:103200008C0C0020810C00207F0C00207E0C002004
:10321000014B1860704700BF840C002070B53D4B17
:1032200004465A7B3C4802B1012202704FF4007000
:1032300000F070F9002828D0384E394B3168987862
:103240000D68003018BF01206A68904748B13368A4
:10325000344D18680121C2682970904708B10221D5
:1032600029702E4D2B6818688268904728B12C4928
:103270008B7813B92B4A0220107029680B68986963
:10328000804710B1274900220A70202004F008FD71
:1032900060B12048244B827A0AB9C17A21B1204812
:1032A000C27A0AB9012100E0002119701D4B18787B
:1032B000022802D14C204E211DE0012807D14D21CA
:1032C00053204C220B46BDE87040FFF753BF164A0F
:1032D0001178012903D1532001464E2206E00E4BFE
:1032E0001878012804D15320014602464D23EAE70D
:1032F00024B153204D210A464423E4E70B4A1178B8
:1033000021B13220BDE87040FFF706BF084B1C70AA
:1033100070BD00BF1C1F0020830C0020840C002007
:103320000B1F0020820C0020880C0020810C002044
:103330007E0C0020014B1870704700BF810C0020EC
:103340000E4B1A78452A16D15888B0F56C7F12D1E9
:103350001979BE290FD193F8AD230020EF2A0CD1A3
:1033600013F8011B064A48409342F9D1D0F10100FD
:1033700038BF0020704700207047704700FC0108EC
:10338000B0FF0108C82314211E220380012381708D
:10339000C270037164214FF496722823C1800281A8
:1033A0004381704710B50446272005F075FE207054
:1033B000102005F071FE6070002005F06DFEA07019
:1033C000002005F069FE4FF4E133E07052206360A5
:1033D000A360E3602361207510BD00007FB51B4D25
:1033E0001B4C284604F092FC2146284604F0A8FC19
:1033F0001F3D04F1240001F085FD2E4604F1680014
:1034000005F026F916F8C40B02F05EF9304603F019
:1034100097FB681C03F052FC05F1B80000F05EFE5B
:1034200004F1280001F068FD04F14B0304F13800B9
:1034300005F1C20100930190029105F17800A11DF0
:10344000224605F1C00302F0D1FD7FBD331D0020EF
:10345000301A002008B5054BD02202FB0030044989
:1034600000F59E700AF0E0FE08BD00BF6019002064
:10347000141D0020254A452370B54FF46C7013705D
:10348000BE210023EF255080117182F8AD5382F8E0
:10349000AE331E461D4A985C0133B3F56C7F86EA55
:1034A0000006F7D182F8AE6308F012FC042600256E
:1034B000711E11F0FF061BD0342008F01DFC002403
:1034C0005CB1124A04F1006505F5FE30A15808F020
:1034D0003FFC0428054607D0EAE70D4808F062FCE7
:1034E00004280546EDD0E3E70434B4F56C7FE7D15A
:1034F00008F0FAFB042D02D1FFF722FF20B90A20C1
:10350000BDE8704001F0F4BE70BD00BF601900203E
:1035100000FC0108034B996808420CBF0020012001
:10352000704700BF60190020024B9A6810439860F2
:10353000704700BF601900202DE9F04FAA4AAB4D3B
:1035400085B010685168AA4C02AB03C34FF46C728B
:10355000002128460AF016FFD022002120460AF05A
:1035600011FF45200321287002206971FFF7DCFF5D
:103570002A232021FA22A5F8EE304FF4FA702B23EB
:1035800085F8F41040F24C41A5F8F220A5F8F600B9
:103590006E22212085F8053101F5487300274FF090
:1035A00001094FF4167685F8042185F8060140F2EA
:1035B000DC5240F27E40A5F816314FF47A73A5F83C
:1035C0001221A5F8F060A5F8141185F8AC7300F588
:1035D0002F71A5F8FA70A5F8F870A5F8FC7085F8B9
:1035E000E27085F8E37085F8E470A5F8E670A5F858
:1035F000E870A5F8EA7085F8ED7085F8EC9085F82C
:10360000077185F8387185F83A7185F8397185F850
:10361000107185F8187185F8197185F81A7185F897
:103620001B7185F81C91A5F8D00003F5CB70A5F8A7
:10363000D6006C30A5F8D8004FF4C870A5F8D210A9
:10364000A5F8D43040F2B4513223A5F8DE0005F5D8
:1036500090709B46A5F8DA10A5F8DC30A5F8E030AC
:10366000019285F81E71FFF79DFE1E21172355203C
:1036700040F6AC52E17263752173A3750B211423DC
:10368000AA81E0702D2208206171A3710E2163745C
:1036900050234FF0280862732074A2766420E171F1
:1036A000E3765A2178234FF00A0A22754122A37249
:1036B00084F8202021722077E177AF73277084F897
:1036C000018084F80280E77584F804B0A773277638
:1036D000E773677684F812A084F8098084F81E9056
:1036E00084F8237084F8247084F82570019904F11B
:1036F0002A00E18484F821B084F8227001F0D0FF20
:1037000004203C4A84F82E003B493C48152384F8A9
:103710003430A263E163206405F58471384827855D
:1037200084F82F8084F8308084F8449004F0C0FC42
:103730004FF44873A4F87430C8224FF4966140F2F5
:10374000D93040F643033E4684F8707084F87170B7
:1037500084F8728084F8739084F8767084F8B8A046
:1037600084F8B920A4F8BA10A4F8BC00A4F8BE30BC
:103770004FF47F724FF4FA61A4F8782007F1080340
:103780006A46A1F5FA70A4F87A10995CA4F87C0056
:103790000137FF2084F87E1084F87F000834082F5A
:1037A000E6D11348012480F8C04080F8C14080F879
:1037B000C240C430FFF7E6FD00230C4A00219818F0
:1037C0001033C02B0161F8D100240E4BD022E01839
:1037D0000749D0340AF028FDB4F51C7FF5D105B0B7
:1037E000BDE8F04FFFF746BEB4FE000860190020A8
:1037F000141D00209A99193FF6287C3F3D0A773F17
:103800007A0001089C1A002008B5FFF799FD18B945
:10381000BDE80840FFF790BE08BD0000024B9A6863
:1038200022EA00009860704760190020364B10B5FE
:103830009C68200409D4E10707D4220705D4E303D8
:1038400003D44FF40040FFF76FFE2F488268044610
:1038500002F42031B1F5203F03D14FF40030FFF7DF
:10386000DDFFA368DC0314D5180702D50820FFF795
:10387000D5FF25488268044612F4004F03D04FF468
:103880000040FFF7CBFFA168C90702D50120FFF771
:10389000C5FF1D488368044613F0080F0BD01A04B7
:1038A00003D54FF40040FFF7B9FFA268D30702D554
:1038B0000120FFF7B3FF144848F20103816848F282
:1038C00001040B40A342044603D14FF40040FFF72C
:1038D000A5FFA26848F24000104048F2400188422B
:1038E00002D14020FFF79AFF084804F069FA08481F
:1038F00005F056FD064805F0CFFC20B90448BDE8A8
:103900001040FFF74FBD10BD60190020681A00205D
:10391000801A002010B5FFF713FD10B90A2001F03E
:10392000E7FC0F4C0F4920464FF46C720AF07CFC08
:1039300094F8AC33022B02D9002084F8AC0394F83D
:10394000AC13D02202FB0143074803F59E710AF035
:103950006BFCFFF76BFFBDE81040FFF73FBD00BFFA
:103960006019002000FC0108141D002008B5FFF7B5
:10397000D1FF0F2014210122BDE8084007F098BBB9
:1039800008B5054B93F8AC03FFF764FDFFF772FD34
:10399000BDE80840FFF7EABF60190020014B9868B6
:1039A000704700BF60190020884203DB8242B4BF29
:1039B00011460146084670470023036170472DE910
:1039C000F041066904460136012E0D46066105D117
:1039D0000023616021608360BDE8F081D0F8008041
:1039E00008464146FCF7DCFF07463046FDF78EF8F7
:1039F00001463846FDF792F901464046FCF7D2FFF2
:103A00000646606031462846FCF7CAFF0146384644
:103A1000FDF7D0F8A168FCF7C5FF2660E060A06064
:103A2000BDE8F08110B504460069012807DD0138C2
:103A3000FDF76CF80146E068FDF770F910BD002055
:103A400010BD08B5FFF7EEFFBDE8084008F0FCBC6C
:103A500008B5FCF7D9FC04A3D3E90023FCF73AFD31
:103A6000FCF74AFF08BD00BF399D52A246DF913FD7
:103A70002DE9F041069C06460F46002B0CBF4FF087
:103A800020084FF03008204610F8013B0BB91546CE
:103A900003E0002AFBDD013AF6E7002D04DD3046A5
:103AA0004146B847013DF8E714F8011B11B1304613
:103AB000B847F9E7BDE8F081014B186801F048BB51
:103AC000980C00202DE9F04389B006460F4603927A
:103AD0001C46039A134613F8011B0393002900F0B8
:103AE0008A80252901D0304683E000200490557853
:103AF000911C302D039105D19578033203924FF03C
:103B0000010800E08046A5F13003D8B2092806D8A4
:103B1000284603A90A2204AB00F02AF905466C2DB9
:103B200005D10399012211F8015B039100E0002205
:103B3000642D2FD010D8582D3AD006D8002D5AD049
:103B4000252DC6D13046294653E0632DC1D13046DC
:103B50002178251DB8474AE0752D0DD0782D27D046
:103B6000732DB6D1251D2468304600943946049A39
:103B70000023FFF77DFF3AE0251D20680A2122B1CE
:103B8000002205AB00F07EF802E005AB00F0AAF8D9
:103B90002C4623E005AD04F104092068294612B142
:103BA00000F095F801E000F0C2F84C46009517E0EF
:103BB00004F104092068102142B1B5F158046342B0
:103BC00053EB040205AB00F05DF806E0B5F15803D5
:103BD0005A425A4105AB00F085F84C4605A80090C2
:103BE00030463946049A4346FFF742FF71E72C46B8
:103BF0006FE7B8476DE709B0BDE8F0830FB407B5CC
:103C0000094904AB0868094953F8042B0968019372
:103C1000FFF758FF064B186801F0B9FA0028F9D0F1
:103C2000BDE80E4004B07047940C0020900C0020BA
:103C3000980C0020034A044B044900201A600860D5
:103C4000704700BFB93A0008900C0020940C002087
:103C5000014B1860704700BF980C002070B50646F5
:103C6000B6FBF2F40846154614B12046FFF7F6FFFE
:103C700005FB1464024B195D00F8011B70BD00BF09
:103C800083000108F0B50124B0FBF4F58D4201D3A7
:103C90004C43F9E70026C4B1B0FBF4F504FB150072
:103CA000B4FBF1F41EB9002D01DC002CF4D1092D78
:103CB000EFB204DD002A0CBF5725372500E0302580
:103CC000ED1903F8015B0136E5E71C70F0BD002833
:103CD0000B4603DA2D22404203F8012B0A21002271
:103CE000FFF7D0BFF0B50124B0FBF4F58D4201D34E
:103CF0004C43F9E70026C4B1B0FBF4F504FB150012
:103D0000B4FBF1F41EB9002D01DC002CF4D1092D17
:103D1000EFB204DD002A0CBF5725372500E030251F
:103D2000ED1903F8015B0136E5E71C70F0BD0028D2
:103D30000B4603DA2D22404203F8012B0A21002210
:103D4000FFF7D0BFA0F13003DAB2092A01D8184634
:103D50007047A0F16101052901D857387047A0F1DB
:103D60004103052B01D8373870474FF0FF307047BB
:103D70002DE9F8430D6804460F4690469946002603
:103D80002046FFF7DFFF002806DB404504DC08FB88
:103D9000060615F8014BF3E73D602046C9F80060C0
:103DA000BDE8F883931E222B88BF0A22031E10B59C
:103DB0000C4603DA2D2001F8010B5842FFF74EFFA5
:103DC00000210170204610BD30B587B005460C4675
:103DD00003A800210C220AF0D5FA28460021FDF79D
:103DE000A5F820B128462949FCF7DCFD03E0284668
:103DF0002649FCF7D5FD2649FCF7DCFEFDF7A0F8C7
:103E0000054685EAE570A0EBE5700A226946FFF7F2
:103E1000C9FF002D01DB202300E02D2368468DF82B
:103E20000C300BF0E3F9012807D130228DF80D207A
:103E30008DF80E208DF80F200CE0022805D13021DE
:103E40008DF80D108DF80E1004E0032802D13020FB
:103E50008DF80D00694603A80BF0C6F803A80BF017
:103E6000C5F9C51EEDB22A4603A920460BF05CFA3F
:103E700000236355204607490BF0B6F803A92046F6
:103E800049190BF0B1F8204607B030BD6F12033A64
:103E900000007A44000B01082DE9F0410278034646
:103EA0000130202AFAD0092AF8D02D2A02D103465F
:103EB000414D04E02B2A08BF03464FF07E551E46B5
:103EC0000024334616F8010BA0F13007F9B2092996
:103ED0000DD83A492046FCF76DFE04463846FCF7FB
:103EE00015FE01462046FCF75DFD0446E9E72E2855
:103EF00017D1324F334616F8010B3038C2B2092AB7
:103F00000FD8FCF703FE3946FCF708FF01462046B0
:103F1000FCF748FD294904463846FCF74BFE0746A6
:103F2000E8E71878652801D0452839D15E782D2E2C
:103F300002D19F1C012605E02B2E01D05F1C00E062
:103F40009F1C00267B1E002713F8012F303AD1B2A8
:103F5000092903D80A2000FB0727F5E7B7F59A7F60
:103F600028BF4FF49A77B8464FF07E51B8F1070F4B
:103F700007D908461249FCF71DFEA8F108080146BA
:103F8000F4E707F0070737B108460C49FCF712FEC3
:103F9000013F0146F7E72EB12046FCF7BFFE04E0E3
:103FA0004FF07E512046FCF705FE01462846FCF7FF
:103FB00001FEBDE8F08100BF000080BF000020418D
:103FC00020BCBE4C014B00229A807047A00C002000
:103FD000034BB3F90400D0F1010038BF0020704753
:103FE000A00C0020014B187A704700BFA00C0020E5
:103FF000014B01221A727047A00C00200649074BA2
:104000000A68B3F90400137805214B439842D4BFE2
:1040100000200120704700BFAC0C0020A00C002045
:1040200010B50446FFF7EAFF002814BF2046002021
:1040300000F0010010BD0000074B084A1968B2F9F2
:1040400004004B780A78D118052251438842D4BF26
:1040500000200120704700BFAC0C0020A00C002005
:10406000024B9A88501C9880704700BFA00C00201B
:1040700070B5FFF7C3FF002824D0134C237A0BB987
:10408000A38070BD114EB578281C18BF0120FFF722
:10409000C7FF78B10E4901200A680E490E4B7070B7
:1040A00050890A681880588098805088D880E388A2
:1040B000591CE180FFF7C0FF00B91DB9BDE8704091
:1040C00000F01CBB70BD00BFA00C00200B1F002027
:1040D000B00C0020AC0C0020641F0020024B00221A
:1040E0001860024882807047AC0C0020A00C0020B1
:1040F000044B05491860054800230160C380037222
:10410000704700BFB00C0020A8000108A00C0020E0
:10411000044B9A8811B2142901DD143A00E0002200
:104120009A807047A00C002003280ED80B4B1B6808
:104130009A888A4209D2DB888B4206D9012202FA88
:1041400000F007490B781843087005490A780F2AD0
:1041500003D100200870FFF7DBBF7047AC0C0020D4
:104160009C0C002030B5784C87B0FFF763FDFFF75B
:104170004BFBFFF7CFFBA07B003018BF012001F005
:104180004FF894F8073133B1012B01D0092B02D13C
:104190008DF8003004E000218DF8001084F807113C
:1041A0006846FDF7BDF80220FFF7B4F910B1674883
:1041B000FEF74EFE6648FEF775FE022003F07AFD1C
:1041C000644D614AB5F9283002F1E200B2F8EE1010
:1041D00092F8ED2000F058FF10B9032001F088F8A4
:1041E0000A25192001F011F86C1E192001F00DF8B4
:1041F00014F0FF05F5D1544C01F0F2FA607904F1A6
:10420000100101F057FFFEF7C5FD04F5907005F0B1
:104210005DF960790E2801D0082803D101238DF8BB
:104220000B3001E08DF80B504B4C0121204605F07E
:1042300079F88DF807004020FFF76CF98DF8080039
:104240004FF40040FFF766F98DF804004FF400309A
:10425000FFF760F98DF806000120FFF75BF98DF894
:10426000050002F04DFB3B498DF8090091F8C22092
:1042700034F8423CC2F3800034F8401C8DF80A0048
:104280004FF47A724FF48040ADF80E30ADF8101054
:10429000ADF81220FFF73EF918B134F8464CADF8EE
:1042A0001240BDF80E00B0F5FA7F02D90023ADF838
:1042B0001230254991F80741B1F81221012CADF8CF
:1042C000142004D0092C01D1072400E0002401A807
:1042D0008DF80C40FDF7F2FC2048FFF709FF204C59
:1042E0002060FEF795FF1D48216803F0A3FD4FF401
:1042F0008070FFF70FF948B1134B1A4A03F590701D
:1043000093F81E11A2F1C30302F028FD4FF40060E0
:10431000FFF700F908B104F019FA00F04BFF124959
:10432000086009484279052A03D14FF4C87000F0AB
:10433000D1FC4FF47A7000F0EBFD0C4B0121002012
:104340005973587007B030BD60190020641A0020FE
:10435000461A0020141D0020801A0020681A002030
:10436000E81D0020D81D0020C00C00200B1F0020DD
:1043700008B5FFF7F7FE00F0E7F9FCE708B5034BD7
:10438000B3F9D40001F0ACFFFEE700BF60190020D4
:1043900008B500F0A5FC28B100F0C0FD80F00100D8
:1043A000C1B205E0022003F07BFC0028F4D001211B
:1043B00001F0010008BD0000044B1A6822B900F5A5
:1043C000F42000F590711960704700BFCC0C0020FC
:1043D000054A13683BB1C01A002804DB03F5F42139
:1043E00001F5907313607047CC0C00202DE9F04F5D
:1043F000AF4BB04AB3F90600D18C85B088420FDBD1
:10440000B0F5FA6F92F8254007DA451A6C43A1F52A
:10441000FA6694FBF6F4643403E0C4F1640400E04B
:104420006424A54FA34B97F9EC1093F82320B7F819
:1044300012C193F870504F4293F8716093F8243092
:1044400001920021BAB2029203930A46984FCB5FC1
:1044500040F2E6370093CCEB030303F2F31EBE45B4
:1044600003D8002BB8BF5B4201E04FF4FA73022A75
:10447000DFF850822CD025B1AB42CCBFC5EB030393
:1044800000236427DFF868A293FBF7FE6FF0630B4D
:104490003AF81E900BFB0E3B0EF1010E3AF91EA0EE
:1044A0000FFA89FECEEB0A0E0EFB0BFE9EFBF7FE0B
:1044B000F14428F80190DDF8048003FB08FE7F4BEF
:1044C0009EFBF3F3DB199BB2634393FBF7F712E018
:1044D00026B1B342CCBFC6EB03030023029F5F4368
:1044E000A8F80470039F002BB8BF5B427B43734F57
:1044F00093FBF7F764376F4B02EB030E9EF80190C6
:10450000642307FB09F898FBF3F9DFF8E88102F868
:1045100008909EF80B909EF815E007FB09F807FB42
:104520000EF798FBF3F9DFF8D08197FBF3F302F86D
:104530000890DDF80080624FE045D35503DA614B07
:10454000CF5A7F42CF5201320231032A7FF47EAF2D
:10455000594C4FF4FA62B4F81411FFF725FAB4F885
:1045600014614FF47A75801B4543C6F5FA63B5FBB9
:10457000F3F56421544895FBF1F36FF0630630F8CE
:10458000132006FB0355013330F9130013B2C01A90
:1045900045434E4B4B4C95FBF1F1587A8A18E2801B
:1045A000002838D04A4F4B4D3E882988721A10B2E5
:1045B000FFF74EFA074607F045FE0646384607F075
:1045C000B5FE0546B4F90200FCF7A0FA0746B4F9B7
:1045D0000000FCF79BFA31468046FCF7EBFA2946CF
:1045E00081463846FCF7E6FA01464846FCF7D8F91A
:1045F000FCF7A6FC314620803846FCF7DBFA29465A
:1046000006464046FCF7D6FA01463046FCF7CAF9A2
:10461000FCF796FC60800220FEF77CFF90B12E4CE8
:1046200006222378581CC3B2B3FBF2F1237002FBBD
:10463000113414F0FF0F05D1FEF7D2FBFEF7F2FBA9
:10464000264B18702548214C0278101C18BF0120F9
:10465000FEF7E4FDA178B1B9FFF79AFEA078012337
:10466000237010B9627B02B92270184C21781C4C5F
:1046700019B11C4B0020186002E02068FFF79CFE77
:104680002068FFF7A5FE04F041F804F02FFF20207A
:1046900003F006FB18B1124A106803F0EDFA124954
:1046A0008B680BB11148984705B0BDE8F08F00BF8B
:1046B000641F0020141D0020601900200CFEFFFF65
:1046C000271E0020321F00203A1F00200B1F002051
:1046D0002E1E0020F61D0020C40C0020B40C00206B
:1046E000B80C0020CC0C00200C1E0020EC1D00207B
:1046F000521F00202A1E0020241E0020024B9A7800
:104700000AB10020987070470B1F00200B4B1978DE
:104710001A4651B1987878B9597831B908480122C8
:104720009A700188074B19807047937823B902204B
:10473000FF21012206F0BCBC704700BF0B1F002008
:104740002E1E0020F61D002038B5904C03F0BCFB57
:10475000206803F0E3FB002800F0F081206803F0FC
:1047600085FC4FF48040FEF7D5FE20B1884C2578BB
:104770000DB9FFF7C3FF03F0AFFC4FF40070FEF775
:10478000C9FE98B1814A83491068884209D9824C90
:1047900023681D682A6A904718B9206801684C6A26
:1047A000A0477D4B1D682A68506980477B490022DD
:1047B000B1F81451B1F81641134679489B08115EBF
:1047C000A942C4BF63F07F03DBB2A142B8BF43F08C
:1047D00040030232082AF0D1724D734A2C782846E1
:1047E0009C4204D11578F92D03D8691C00E0002102
:1047F000117003704FF48040FEF78CFE68B167487B
:10480000674BB0F81211B0F8DC20B3F906408D1AEE
:10481000AC4202DD8B189C420CDB4FF48040FEF76B
:1048200079FED8B95E4C5D49B4F90600B1F814219F
:10483000904213DA5D4D00F037FF00F03DFFB5F810
:1048400046305BB1524C5A492078002800F00C8267
:104850000A78002A00F00882FFF758FF524B1C78B4
:10486000142C40F0C18052488478ECB14F4BB3F81F
:1048700046502DB94B490C785F2C01D1FFF73EFF14
:10488000464A92F81A01002800F0AE80474BB3F870
:104890004650002D40F0A88042490C787D2C40F015
:1048A000A380FFF72BFF9FE03E4D2978572911D1B8
:1048B0004FF47A7000F02CFB4FF48070FEF72AFE64
:1048C00008B102F0A9F9082003F0EAF9E0B9394C7F
:1048D000208019E00420FEF71DFEA8B12A785A2A8C
:1048E00012D1354B187820B11C70344B01221A704C
:1048F0000AE0334C257885F00101217009B10220CE
:1049000000E00320FEF716FD264805785D2D00F037
:10491000B2815B2D00F0B1815E2D00F0B0812348A3
:10492000B0F8465035B91F490C786F2C02D1FFF70B
:10493000EDFE15E0194A1B4B92F81A0118B115B992
:104940001D787E2DF3D01978972904D14FF4C870C3
:1049500000F0C0F904E0A72902D1154A012494739C
:1049600010480378BB2B03D11048818D8D1C04E0C7
:10497000B72B04D10D48838D9D1E858528E0BE2B65
:1049800020D10A4D6A8D941C21E000BFB80C002094
:104990001C1F0020404B4C00E81D00206019002027
:1049A000641F0020C70C0020B50C0020141D00203F
:1049B0000B1F00202E1E0020D00C0020C80C002051
:1049C000C60C0020BD2B0FD16B4D698D8C1E6C85E4
:1049D0006A4C94F8AC03FEF73DFDFEF74BFDFEF785
:1049E000C5FF6748002202700420FEF793FD0028EF
:1049F0002CD0644B1A788AB16348857875B16349C5
:104A00005E4AB1F90640B2F81401844206DD604DF9
:104A10002C781CB95F4932220A801C705C4B587C90
:104A200050B15D4B1D782DB95C4C227812B95948B4
:104A300032210180012008E0584D2C7834B1524ACF
:104A4000917819B9564B2970012018700023554CE4
:104A50001A4634F8020F40F2135501B2A942CCBFF6
:104A60000025012505FA03F5A0F21550B0F5C77F22
:104A70008CBF002001202A435D1C00FA05F0024390
:104A800040F2A4608142D4BF00210121981C01FAA8
:104A900000F103330A430C2B92B2DAD100233649DA
:104AA0003B4C01EB4300B0F846100A420CBF00201B
:104AB000012018550133152BF1D1627822B1022063
:104AC00003F0EEF868B914E04FF40070FEF722FD31
:104AD00078B1354C21680868836898470028EED182
:104AE00007E0294CE17839B900F0DEFD0120E070E3
:104AF00002E0254C0022E270254B234C987830B11F
:104B000021790022E27019B900F0CEFD0120207158
:104B1000202003F0C5F808B103F050F81C4B1A49E7
:104B20001A7B02B1012215488A724379082B01D001
:104B30000E2B44D1144A0021517240E01B4B1A68DD
:104B4000042A3CD8DFE802F00305080B34000120FA
:104B5000186019684A1C1A601868411C1960134BC8
:104B60001A68501C18604FF48070FEF7D3FCF8B13F
:104B700002F022FA23E000BF141D0020601900207B
:104B8000B50C0020C60C00200B1F0020641F002065
:104B90001C1F0020D20C0020C50C0020D00C0020CF
:104BA000C80C00206A1F0020E81D0020D40C002043
:104BB0003B4B00214FF400501960FEF7ABFC00F0B6
:104BC000F9FA3849384B8A891860384B1AB1196894
:104BD000411A00293CDB84181C6001F005F8FFF73E
:104BE00005FC00F0E7FA324B2F4A19681060441AAE
:104BF00018603048304A90F87630148053B12F490D
:104C0000CC780CB90A792AB12D482E4BC488198862
:104C10000A19C280202003F043F840B12748C37925
:104C20000BB9017A19B1047B0CB102F03DFF2648A3
:104C3000264A1C4B00F11E011468B3F8F62000F15F
:104C40002903A04701F05EFB01F0DAFA01F034FB22
:104C50001F48017819BB4FF40060FEF75BFCF0B110
:104C6000BDE8384003F096BD8D78002D3FF4F6ADD9
:104C7000FFF744FDF2E5012102E0022100E00321FB
:104C8000CCB2084B621E83F8AC23FEF7F3FBFEF7B1
:104C900041FE02202821224606F00AFA3FE638BDEE
:104CA000D40C002060190020B80C0020BC0C00209F
:104CB000C00C0020141D0020CA0C00200B1F002077
:104CC000321F0020F80D0020151D002008000020D4
:104CD0001C140020014B1880704700BFF00C00200E
:104CE000034B1888D0F1010038BF0020704700BF87
:104CF000F00C0020F8B51E4B0022196813461D4C1D
:104D00002588B5F5C87F1C4D01D10026EE501B4EFD
:104D1000EF5832F906C0184C6744EF5000250433B1
:104D200095538D5202320C2BE9D1124B1A88012A6D
:104D300018D1236803F1C8024FF4C87392FBF3F251
:104D40000A806268C83292FBF3F24A80A268C832D5
:104D500092FBF3F30A4A12889B1A8B8000F0A0FCA6
:104D6000FEF70EFE034801884A1E0280F8BD00BF10
:104D7000F40C0020F00C0020E40C0020481E002061
:104D800004000020F8B5354B0446188832280ED1AF
:104D90003349344D0A6834481688578893882188E7
:104DA00062882E806F80AB800180428001E0002805
:104DB00034D02B4D00222E681346284F2B493888BB
:104DC000322801D10025CD502948CD58175EED1964
:104DD000CD50002104331152B15202320C2B0D463A
:104DE000EBD11E480188012914D1224B224A02200E
:104DF00011701D70FEF79EFA1A4A1948118803684F
:104E000050889288198058809A80174B1988588842
:104E100021806080114B1A88511E19801748037831
:104E2000DBB10F4900220B6810490270086832227A
:104E300090FBF2F01880486890FBF2F05880896887
:104E40000F4891FBF2F201882046521A9A8000F036
:104E500027FCBDE8F840FEF793BDF8BDD20C00205A
:104E6000F40C0020F80C0020000D0020D80C0020CD
:104E7000481E0020C50C0020D00C0020C80C0020CB
:104E800004000020064B02881988891A198042887C
:104E90005988891A5980808899880A1A9A80704797
:104EA000481E00200F4B10B5596804460E4888472D
:104EB0000D480E4A01461278FEF78AF80C4803881E
:104EC00013B12046FFF716FF0420FEF723FB10B1B5
:104ED0002046FFF757FF07490868BDE81040FFF775
:104EE000D1BF00BFF81D0020481E0020040D002087
:104EF000F00C0020F40C0020014B1860704700BF3C
:104F0000F40C0020014B1860704700BF1C0D0020FE
:104F1000014B1880704700BF200D0020034B1888FC
:104F2000D0F1010038BF0020704700BF200D0020E5
:104F30002DE9F8433C4B3D48596888473B483C4A7B
:104F400001461278FEF744F83A480388002B42D015
:104F5000394C256800242F782646254635490A888D
:104F6000B2F57A7F08D1354B354A00201421E8503C
:104F700001FB0620FEF720FDDFF8B0802F4B38F94B
:104F80000400E9584FF014090A18EA502C4B09FBA9
:104F90000639FBF7BBFD01464846FEF710FD002031
:104FA00024F80800DFF88C802649B8F80020605209
:104FB000012A2FD14846FEF744FD8146DFB138462D
:104FC000FBF7A4FD01464846FBF7B0FF98B14FF44C
:104FD0007A73A8F80030154B1A4A18881188401ABD
:104FE0001880518858889288401A99885880881A61
:104FF0009880BDE8F883114B4FF47A72E858114B52
:1050000000F5FA7191FBF2F0E0520F210A20012223
:1050100006F04EF8013604350234032E9ED10549C0
:105020000A88501E0880D6E70C1E0020301E002083
:10503000600D0020200D00201C0D0020100D002010
:10504000240D0020140E00200146034B03480022CB
:105050001A70FCF721B900BF600D00200C1E002063
:1050600003780BB1054A1370417809B1044B1970EC
:10507000807808B1034A1070704700BF600D0020AF
:10508000040D00200C0D00202DE9F04106460846D5
:1050900014461D46FFF7D8FF002849D0254B0022B3
:1050A000022C1A7007D0072C01D024B10AE002208C
:1050B00002F008FE06E02048FCF79CF810B11F49FA
:1050C000022008701D4A13782BB90CB11C46E5E785
:1050D000022002F0F7FD3046FFF7C2FF022002F087
:1050E000DFFD10B1144C206880471549154C0A6843
:1050F0009047082002F0D4FDB8B1642795FBF7F67D
:105100003046FBF703FD804607FB165000B2FBF765
:10511000FDFC0D49FBF74EFD01464046FBF742FC06
:105120000A49FBF747FD206001E0002323600120CE
:10513000BDE8F081040D0020F81D0020FE0C0020C9
:105140000C1E0020000E00208988883C00002041B1
:1051500008B503681A68904708BD38B505460C467F
:1051600014F8011B19B12846FFF7F2FFF8E738BD24
:1051700008B503685968884708BD08B50368996889
:10518000884708BD08B50368DA68904708BD08B5C8
:1051900003681969884708BD08B503685A699047CC
:1051A00008BD7047024B1A68501C1860704700BF5A
:1051B000640D002010B5094A094913688C6810680D
:1051C0008342F8D1074A106811684FF47A7250434D
:1051D000001BB0FBF1F102FB031010BD640D0020B9
:1051E00010E000E0680D0020014B1868704700BF18
:1051F000640D002038B50446FFF7DCFF0546FFF7D5
:10520000D9FF401BA042FAD338BD10B504462CB1DB
:105210004FF47A70FFF7EEFF013CF8E710BD000095
:1052200030B587B005F0BEFF0121264806F03EFEEE
:10523000012144F61D2006F02DFE0120014606F056
:105240001DFE002506F056FE06AC4FF6FF736946BC
:105250001D4824F8183D8DF80250FCF7F3FC694610
:105260001A48FCF7EFFC69461948FCF7EBFC1948B3
:10527000426842F000714160FFF793FF01A806F019
:10528000AFFD019B1448154AB3FBF0F114481160BF
:1052900001684FF47A73B1FBF3F2124B501E124ABD
:1052A0005860F021072082F823109D6018600F4895
:1052B000FCF75EFAFCF74AFC6420FFF7A6FF07B094
:1052C00030BD00BF0700400000080140000C014055
:1052D000001001400000014040420F00680D002016
:1052E0008801002010E000E000ED00E000580040E0
:1052F00010B540F2DB146043841E2046FFF785FFA3
:105300001920FFF782FFF8E710B1034A034B1A6038
:1053100003480449C8607047EFBEADDEF04F00207F
:105320000400FA0500ED00E02DE9F04F89B0079385
:10533000754B07460692B3F90000B3F90220002826
:10534000B8BF4042002AB8BF524200248242B8BFD0
:10535000024605922546A146A0460494A24626464A
:105360006A49CB7813B90A79002A38D0022E36D090
:10537000674B6548EA5EDDF818B0295E02EB410034
:10538000CBF100015A46FEF70FFB6249DDF81CC065
:105390006B5E3CF90520C01A8318F879FA7E5843F1
:1053A00064214FF0050E90FBF1F06FF004015143C2
:1053B0000EFB02F20393FEF7F7FADFF878B1039BD6
:1053C000824654F80B00544942F210721818FEF746
:1053D000EBFA7A7C44F80B005043011304914B48DC
:1053E000C3781BB102790AB9022E2FD14649502049
:1053F00035F90180DFF828B100FB08F2BB5DDFF86A
:10540000389135F90B0092FBF3F154F809300A1A80
:10541000D01842494FF47A52FEF7C6FA35F90B100C
:1054200049F804000029B8BF4942B1F5207F02DDE8
:10543000002049F8040059F80420B9197D23887A1E
:1054400092FBF3FC00FB0CFE4FEAAE192F4B1A79CE
:10545000B2B1022E14D0DDF814B0DDF810C00BFB91
:1054600008F0CBF5FA7303FB0A020BFB09F003FB10
:105470000C034FF4FA7192FBF1F293FBF1F308E0A5
:10548000D97809B1022E02D14B46424601E0049B75
:1054900052462349DFF8A4B0695A16F80BC008B287
:1054A0000CFB00FB6FF04F0C9BFBFCFC94441D4A73
:1054B000CDF800C035F902C0A952CCEB00001A4A61
:1054C000DFF87CC0019054F80C10A05840180199E6
:1054D00002904018A15844F80C100199A150134AA9
:1054E0000434B15C202201FB00F090FBF2F1581A69
:1054F000009B0F49C21801366A520235032E7FF411
:105500002FAF09B0BDE8F08F321F00200B1F002025
:1055100002100020040E0020F0D8FFFF80C1FFFF22
:10552000C40D0020780D0020940D0020271E0020BF
:105530001E1E00208C0D00206C0D00202A1E002055
:10554000800D00202DE9F04F002585B006468946E4
:105550009246039307462C46022CDFF8388109D186
:1055600099F80500B8F904B01B300BFB00FC4FEABA
:105570006C1E2CE03E4B38F9140033F914105246DF
:1055800001EB4000CAF10001FEF70EFA394A039917
:1055900032F9143031F91420C01A374B8018D978F9
:1055A00079B999F8042038F914801B3208FB02F10C
:1055B0001B794FEA211E53B1727C50430EEB202E13
:1055C00005E096F807B00BFB00FC4FEA2C1E2B49B8
:1055D000DFF8C4C031F91430325DBCF80010C3EB01
:1055E0000E0802FB08F001FB08F2254BB97A4FEADE
:1055F000E01BD012EA5801FB00202249E8504FF48A
:1056000000120293CDF804C0FEF7CEF9029BDDF83C
:1056100004C01D4AE850BCF80030A9581B0945F8E1
:1056200002804FF6FF72B2FBF3F3C1EB080159435E
:10563000DFF868C0154B55F80C2055F80380891128
:105640004244E9505218397D0BEB60304A43104B0D
:1056500000EB222223F81420013445F80C80013796
:105660000435032C7FF478AF05B0BDE8F08F00BFA0
:1056700002100020040E00200B1F0020C40D00208B
:105680006C0D00200000E0FFB80D0020AC0D0020E4
:105690001E1E0020321F0020CA0C0020A00D00207A
:1056A0000023038043807047024B00221A605A6037
:1056B000704700BF8C0D0020024B00221A605A6018
:1056C0009A6070476C0D00200128034B14BF034AF9
:1056D000034A1A60704700BF0800002029530008E1
:1056E00045550008000000002DE9F84F384E0446EB
:1056F0003768384606F0A6FD0546384606F016FE21
:1057000076688046304606F09DFD8346304606F0BA
:105710000DFED4F80490064629464846FBF74AFA9F
:10572000A768824641463846FBF744FA0146504690
:10573000FBF736F9216882465846FBF73BFA4146AB
:1057400004464846FBF736FA3146FBF733FA014682
:105750002046FBF727F9314604463846FBF72AFA7C
:105760002946FBF727FA01462046FBF71BF90146BD
:10577000504606F067FE1749FBF71CFAFAF756FE8B
:1057800011A3D3E90023FAF7CFFF134B044618689F
:105790000D46FAF74BFE02460B4620462946FAF71D
:1057A000E7FC00220D4BFAF7BFFFFBF7A5F806F068
:1057B0007DFD81B20A0444BF00F5B47189B208B21C
:1057C000BDE8F88FAFF30080182D4454FB21094049
:1057D000CC0D00200000E144000E00200000244019
:1057E00010B5194C2088FBF791F91849FBF7E2F93D
:1057F00006F05CFD164B18802088FBF787F9014600
:105800001448FBF78BFA1449FBF788FA1349086030
:105810001348B0F87400FBF779F901461148FBF71B
:105820007DFAFAF703FE06A3D3E90023FAF752FE46
:10583000FBF762F80C4A106010BD00BFAFF30080A8
:105840003B597E90A9E7814004000020C903683FCE
:10585000CA0D00200AE81C4100401C46441E0020DE
:10586000141D002000006144601E0020AFF3008082
:105870002DE9F041044600680D460146FBF79AF910
:10588000D4F80480064641464046FBF793F90146AA
:105890003046FBF787F8A768064639463846FBF7D7
:1058A00089F901463046FBF77DF806F0CDFD002171
:1058B0000646FBF713FB70B920683146FBF72EFA5A
:1058C000314628606068FBF729FA31466860A068B5
:1058D000FBF724FAA860BDE8F0812DE9F04F0C68D1
:1058E000836889B0D0F800A0D0F80480064620462E
:1058F00003938B4606F0A6FC0746204606F016FDED
:10590000DBF804408146204606F09CFC0546204614
:1059100006F00CFDDBF8082004461046019206F064
:1059200091FC8346019806F001FD394602905846E5
:10593000FBF740F9394604900298FBF73BF95946CA
:1059400005904846FBF736F9029906904846FBF762
:1059500031F9294607905846FBF72CF90146504685
:10596000FBF728F9214683460698FBF723F9014601
:105970000598FBF717F801464046FBF71BF901466F
:105980005846FBF70FF8214683460498FBF712F9B7
:1059900001460798FBF704F801460398FBF70AF95C
:1059A00001465846FAF7FEFF3060029905F10040C3
:1059B000FBF700F901465046FBF7FCF82146834609
:1059C0000798FBF7F7F801460498FAF7E9FF014654
:1059D0004046FBF7EFF801465846FAF7E3FF214649
:1059E00083460598FBF7E6F801460698FAF7DAFFD2
:1059F00001460398FBF7DEF801465846FAF7D2FF56
:105A0000214670605046FBF7D5F82946044609F157
:105A10000040FBF7CFF801464046FBF7CBF80146C4
:105A20002046FAF7BFFF394604462846FBF7C2F87E
:105A300001460398FBF7BEF801462046FAF7B2FF8D
:105A4000B06009B0BDE8F08F80EAE073A3EBE073CB
:105A50008B4206DB002801DD401A704702D0401857
:105A600070470020704700002DE9F041524B86B08E
:105A70001A685B6802F1004203F1004301934F4B47
:105A80000646B3F900000092FBF740F800F1004031
:105A9000FAF7CCFC46A3D3E90023FAF71BFDFAF78B
:105AA0002BFF474C0290B4F90000FBF72FF803904E
:105AB000B4F90200FBF72AF80490B4F90400FBF7EC
:105AC00025F86946059003A8FFF707FF3D4B93F8BB
:105AD0004430012B16D13C48817869B93B4C4025B4
:105AE000226892FBF5F7D01BFBF710F80599FAF73F
:105AF00059FFFBF725FA2060344B4021186890FBD2
:105B0000F1F001E0324B1888FBF700F801460598E8
:105B1000FAF746FF05903046FAF7F4FF2D4907469D
:105B2000FAF740FF01463846FBF7F8F82A4D0746DA
:105B30002C6805982146FAF733FF01463846FBF7F3
:105B400039F801462046FAF72DFF244C28601D4DF8
:105B500007460398D4F8008006F0A8FB95F83010AB
:105B6000FFF772FF08EB000204982260D4F804806B
:105B700006F09CFB95F83010FFF766FF08EB00037A
:105B800038466360D4F8088006F090FB95F82F1033
:105B9000FFF75AFF1249134B0A684044A060186887
:105BA000B6180E60411C196006B0BDE8F08100BF58
:105BB000399D52A246DF913FCC0D00202E1E0020C1
:105BC000581E0020141D00200B1F0020FC0D00207B
:105BD000040000203661823CD40D0020381E0020D5
:105BE000E00D0020F40D00202DE9F04F87B0FFF705
:105BF0009FF9022002F054F8002800F0AD81AE4871
:105C0000FFF750F9FFF7D6FAAC4C05462768C71BDB
:105C10003846FAF777FFAA49C968FAF7CBFF8346F7
:105C2000A848256090F82E8000252C462E46A64ACE
:105C3000105FFAF76BFF5946FAF7BCFF03AB5851F8
:105C4000B8F1000F27D04046FAF760FF01464FF049
:105C50007E50FBF763F8DFF8B092824651464FF072
:105C60007E50FAF79DFE55F80910FAF7A3FF974901
:105C70000346085F0193FAF749FF5146FAF79AFF86
:105C800001460198FAF78EFE49F80500FBF758F92E
:105C90008F4A105303E08D498D4A605AA0528C4BB5
:105CA0000435E15E0234062C01FB0166BFD1894A4E
:105CB0006420138846435B43874803A996FBF3F6A9
:105CC000FFF70BFE082001F0EBFF20B1834803A98A
:105CD000FFF703FE07E0824803A9FFF7FEFD8048B7
:105CE0000146FFF7C5FD493E7E49B4B23B2CB1F8F1
:105CF000F00007D97B4E0820B6F8F25001F0D0FF33
:105D000030BB4FE0FAF7FEFE4FF07E518046FAF7C7
:105D100049FE01464FF07E50FBF700F8002406468E
:105D20006D4D404655F81410FAF744FF8146684817
:105D3000005FFAF7EBFE01464846FAF733FE3146BC
:105D4000FAF738FF45F814000234062CE8D1D1E701
:105D5000B6F8F200FAF7D6FE80462846FAF7D2FEE9
:105D60004FF07E51FAF71EFE01464FF07E50FAF7D3
:105D7000D5FF00240646594D404655F81410FAF751
:105D800019FF594A8146105FFAF7C0FE014648469E
:105D9000FAF708FE3146FAF70DFF45F81400023411
:105DA000062CE8D1514B4C4DB3F90000FAF7AEFE8A
:105DB000AC68014620460126FBF7B8F800B9064654
:105DC0004B4968684E73214606F03CFB494CD5F8B8
:105DD00008802060286800F1004668680146FAF7EC
:105DE000E9FE414605464046FAF7E4FE01462846EC
:105DF000FAF7D8FD06F028FB0146304606F022FBF4
:105E000060602068FAF712FB29A3D3E90023FAF7B0
:105E100061FBFAF771FD06F049FA374D288060689A
:105E2000FAF704FB22A3D3E90023FAF753FBFAF7AE
:105E300063FD06F03BFA6880082001F031FF2F4C2B
:105E400008B1264800E02648FFF74EFC1D4D208093
:105E50003846FFF709FE95F87620002A00F080808A
:105E60001D4B18689C6801465F68FAF7A3FE394627
:105E700006463846FAF79EFE01463046FAF792FD8E
:105E8000214606462046FAF795FE01463046FAF7C7
:105E900089FD06F0D9FA01462046FAF73FFF184976
:105EA0000446FBF72FF888B316480021018057E01D
:105EB0003B597E90A9E781403E1D0020E40D002063
:105EC0000C1E0020141D0020301E0020481E002043
:105ED000581E002004000020641E0020E80D002051
:105EE0000C00002060190020041E0020CA0D0020B4
:105EF0000B1F0020CC0D0020040E00202E1E0020C1
:105F00008FC2753CF80D0020080E0020204606F0D8
:105F100049FA274B1968FAF74DFE06F0C7F9B0F5B4
:105F2000617FA8BF4FF46170FAF76EFA1EA3D3E940
:105F30000023FAF7F9FBFAF7DFFC06F0F7F904465D
:105F400095F87600FAF7E2FD2146FAF733FE06F0FF
:105F5000ADF9184B188003E0174B188058809880D3
:105F6000164A5379012B164B07D0164819885A88C0
:105F70009B8801804280838011E01349B3F904209B
:105F8000B1F9000002EB4000032290FBF2F080B276
:105F90000C4A088019885B8890801180538007B074
:105FA000BDE8F08FAFF30080A2EB0FE5DD16964061
:105FB000601E0020F80D0020481E002060190020FF
:105FC000301E0020C40D0020D80D0020AFF300804B
:105FD00010B5054C00202188FBF7B4FF6188012033
:105FE000BDE81040FBF7AEBF1800002010B5094C0B
:105FF000206009480160094909480A60094A0A49BC
:106000001360029B039A03600848049B0A600360C4
:1060100010BD00BF1C0E0020F80E0020240E002032
:10602000F40E0020FC0E00202C0E0020F00E0020AC
:106030000A4B1A6802EBC002D379FF2B07D008493C
:106040000978994203D9074830F8130004E007287B
:10605000D4BF908840F2DC5000B270471C0E002084
:10606000601F0020641F0020054B1A6802EBC0006F
:1060700090F9063019420CBF01204FF0FF307047F5
:106080001C0E002010B500244FF48040FDF742FAAA
:1060900008B1054B00E0054B1868054A8188A152FC
:1060A0000234182CF0D110BDF80E0020240E002070
:1060B000881E0020F8B53A4B3A4E0546187006EB9C
:1060C000C0000F46384C417820202160FDF722FAAD
:1060D00008B101222260162D19D10024385900215F
:1060E000FAF7FCFE28B14FF48040FDF713FA50BBDD
:1060F00025E02E4A3B1916190FCB86E80F002C48D5
:10610000103401784A1CC02C0270E7D1EBE716F876
:10611000357006EBC506264BD6F804E01F70BEF1BD
:10612000000FE0D00024BC42DDDA204E20013618FA
:106130000EEB00010FC9013486E80F00F3E7082DCC
:106140001C4B23D124E01A4F3F78012FF7D91A4C6A
:1061500000261034BE42F2DA54F8100C4FF07C5195
:10616000FAF728FD4FF07C5144F8100C54F8140C49
:10617000FAF720FD4FF07C5144F8140C54F80C0C45
:10618000FAF718FD013644F80C0CE2E70E2D01D1A8
:10619000012000E000201874BDE8F840FFF772BF4E
:1061A000200E002020030108000F0020300E0020E8
:1061B000280E00200B1F0020380E0020F0B58C4662
:1061C000461C002300224CF803201033C02BF9D1C9
:1061D0000A4800EBC6014F6807B9F0BD0024074B21
:1061E00013F83620944208DA20010CEB0005391828
:1061F0000FC9013485E80F00F1E7F0BD2003010865
:10620000284B10B5186800284AD027490A78531E31
:10621000142B3DD8DFE803F00B3C3C24403C3C1CF5
:106220003C3C3C3C3C2C3C3C3C3C3C242C001F4833
:1062300001684A7832B11E4900204989BDE8104002
:10624000FBF780BE1B4B98780028F4D10146F5E798
:10625000174C0020E188FBF775FE01202189EDE74E
:10626000134C00202189FBF76DFE01206189E5E7D1
:106270000F4C0020E188FBF765FE01202189FBF728
:1062800061FE02206189FBF75DFE0320A189D5E74D
:106290002020FDF73FF918B1BDE81040FFF798BE88
:1062A00010BD00BF000F0020200E0020FC0E0020BB
:1062B000180000200B1F002010B50024064B187892
:1062C000A04208D90549204631F814100134FBF7E3
:1062D0002DFEE4B2F2E710BD280E0020701E002053
:1062E000064B1A780023D9B2914204D2044921F80E
:1062F00013000133F7E7FFF7DFBF00BF280E0020D0
:10630000701E00202DE9F74FA34B187803280FD9F2
:10631000A249A34CB1F904206FF06305002AB8BF6D
:106320005242A91AB4F904006432FDF73DFBA08083
:10633000994A1678012E1DD89A4E3478651E9A4CCB
:10634000142D00F2C981DFE815F0A400C701C701D0
:106350007B00B300C701C7015A01C701C701C701CC
:10636000C701C701D000C701C701C701C701C701E5
:106370005F00A1018D488A4B884F0168B7F806B0CD
:10638000B3F800805F88B3F904A0894C019100251F
:106390001034B542D0D20FFA8BF0FAF7B7FB54F8AD
:1063A000101CFAF707FC814638B2FAF7AFFB54F835
:1063B000081CFAF7FFFB01464846FAF7F3FA814654
:1063C0000FFA88F0FAF7A2FB54F80C1CFAF7F2FB6C
:1063D00001464846FAF7E6FA019A814692F900002A
:1063E00041420AFB01F0FAF791FB54F8041CFAF75A
:1063F000E1FB01464846FAF7D5FAFAF7A1FD6D4BE5
:1064000023F815000135C3E701210420FFF72CFE16
:10641000634D654C6E88704387B204202781FFF777
:1064200007FE3818208101210520FFF71DFE2B886B
:10643000584385B205206581FFF7FAFD2B1826E049
:1064400002210420FFF710FE554C0121A68870435D
:1064500087B20420FFF708FE6588534C00FB0572E5
:10646000042097B2FFF7E4FD3818208102210520AF
:10647000FFF7FAFD7043012186B20520FFF7F4FD16
:1064800000FB056105208DB2FFF7D2FD2B1863815B
:1064900022E101210520FFF7E7FD414A424E97889E
:1064A000784384B20520FFF7C3FD2018708113E103
:1064B000414900200D68FFF7BBFD404F95F90630BC
:1064C000B7F902607343322693FBF6F280182080FE
:1064D0000120FFF7ADFD95F90E10B7F900506943A3
:1064E00091FBF6F3C7186780F6E03549354E8A7898
:1064F000376812B9B888E08108E0284C3988B4F9C7
:1065000006007A88FDF750FA274BD881264D2E4F8A
:10651000E989284A3E681180347854B3264D022018
:10652000FFF786FD2B68B3F91010B3F91220FDF7C1
:106530003BFA2649264B0A68198854890EB2201A5C
:1065400002B2964203DA3E683278511803E003DD66
:106550003F683878091A19802D681D4F95F9163053
:10656000B7F90000642143430F4A93FBF1F6A419E5
:106570009480134D0C4BAF7A67B1084801880E4ADE
:10658000D9801981868817685E814488064D9C8170
:1065900003241FE00248F1E7280E0020321F0020EC
:1065A0001E1E0020200E002018000020FC0E0020DF
:1065B000300E0020701E00201C0E0020040E002053
:1065C0000B1F0020240E0020F40E00202C0E0020B3
:1065D000220E002007EBC40393F90600B5F906105C
:1065E0006426414391FBF6F6EE802046FFF720FD3E
:1065F00001343218EA800235072CEBD16CE0A54F4C
:10660000A54BB8781E6810B9B588E58108E0A349A4
:106610007288B1F906003188FDF7C6F9A04AD08129
:106620009F4C9C4B9F48E7899E7A0780012103205D
:106630001EB1FFF719FD994D02E0FFF715FD9A4DC8
:106640006E880221704387B20320FFF70DFD2D886D
:1066500000FB05710420E1800121FFF705FD704377
:10666000022186B20420FFF7FFFC00FB0562032035
:106670002281FFF7DDFC8A4CE388C018E08004200B
:10668000FFF7D6FC2789C519258125E0864A032412
:10669000978802212046FFF7E7FC7843012186B264
:1066A0002046FFF7E1FC804DC4F10603590835F898
:1066B00011207B4D00FB026086B225F81460204655
:1066C000FFF7B6FC331825F814300134072CE0D15D
:1066D000724F744AF98811802020FCF71BFF0028B4
:1066E00045D00020FFF7A4FC6D4F054638800120FF
:1066F000FFF79EFC6D4978800B7A002B37D06C4AEF
:106700006C4B14686C4A267806F00201CCB2D4B106
:106710001468B3F9001094F90E2094F906404A4326
:10672000322192FBF1F6B3F90230B2B26642734302
:106730006FF0310493FBF4F69419651993FBF1F1B2
:106740003D80561811E01168B3F9026091F90640D6
:106750003222664396FBF2F42D193D8091F90E101A
:10676000B3F900304B4393FBF2F680197880002692
:10677000514F4B4D3B68A85F03EB860233F926105F
:10678000B2F90220FDF710F9A8530236102EEFD10E
:10679000474C2168087800F00407FBB22BB9414A46
:1067A000464C1688277801231CE0454D2E780E2E86
:1067B0000AD0082E08D0434A02EBC60461780029AB
:1067C00014BF0225002500E0042500263E4F701965
:1067D00007EB4603C0B219890136FBF7B3FB042E61
:1067E000F4D1DCE7BB4209D22E4C36B234F9131097
:1067F0000133B142A8BF0E46B6B2F3E700242746E4
:106800002E490878874272D2234D31B22B685A88BC
:10681000914204DD2348951B235AEA1822524FF473
:106820008040FCF777FE1F4DC0B1284A264B106808
:10683000B3F906104389184A9942254905DD0968CC
:106840001268285F4988528804E012680B68285F44
:1068500091881A88FDF7A8F828533EE0DFF83880C1
:10686000285FD8F8003005EB040919885A88FDF72D
:106870009BF8164A144913682853B1F90600998900
:1068800088422ADA1020FCF745FED8F8002008BB21
:10689000108820E00B1F0020240E0020321F002053
:1068A00018000020701E00201E1E00201C1F00204B
:1068B000F00E0020040E00201C0E0020280E0020E8
:1068C000200E002020030108641F00202C0E002051
:1068D000F80E00209088A9F80000064883781BB9BC
:1068E00005490648625A22520137023488E7BDE85A
:1068F000FE8F00BF0B1F0020881E0020701E00208E
:10690000024B1868003018BF01207047000F0020AC
:1069100044F25063984203DDA0F50C40A038704764
:1069200003498842BCBF00F50C40A030704700BF4F
:10693000B0B9FFFF10B5FAF7E9F800210446FAF7FD
:10694000F5FA08B1204601E004F100400549FAF7E4
:10695000E5F90549FAF72EF905F074FC034B1860C8
:1069600010BD00BF8096184B35FA8E3C2C000020DD
:1069700010B5044C002320702361FEF735FC6061E4
:1069800010BD00BF78100020F8B51D4614460E4615
:10699000FAF7BCF86968FAF70DF93146FAF70AF91F
:1069A0002168F9F7FFFF2060FAF7CAFAED68074699
:1069B00005F10040FAF7C4FA06462846FAF7C0FA8D
:1069C000314602463846FCF7EFFFFAF79FF82060A1
:1069D000FAF7B6FAF8BD0000F8B5101A0C461F46D3
:1069E000FAF794F80546381BFAF790F8174B079E0C
:1069F0001968FAF7DFF8294604462846FAF7DAF864
:106A0000214607462046FAF7D5F801463846F9F7F9
:106A1000C9FF05F019FD0E49FAF7CCF8FAF7B6FAF6
:106A200006990860214605F1004005F00BFD094973
:106A3000FAF7C0F80849F9F7B5FFFAF781FA002824
:106A4000BCBF00F50C40A0303060F8BD2C00002029
:106A50002C7D8E3FA00CB34500A00C4610B504461B
:106A6000002003460D49CA5CA2B12E2A04D101338D
:106A700094B1C91800220A55084A0A21D25C484339
:106A8000A2F13001092901D8303880180E2B02D824
:106A90000133E7E710BD002010BD00BFDF0F00206D
:106AA0002DE9F843224B074648681D68381A0C4602
:106AB0009146FAF72BF82946FAF730F91D4920617B
:106AC0000A6880469078FAF71DF8F9F7AFFC16A32C
:106AD000D3E90023F9F7FEFC02460B4600201649D5
:106AE000F9F722FEF9F708FF2946F9F75BFF01469F
:106AF0002846FAF713F9A668054631464046F9F7E5
:106B00004FFF01462846FAF755F801463046F9F797
:106B100049FFD9F8081020616760A060FAF74AF8C9
:106B2000FAF70EFABDE8F883182D4454FB211940FA
:106B300014100020D80F00200000F03FAFF30080B9
:106B4000014B1860704700BFD80F0020F8B52D4BDF
:106B5000187810B1012850D10AE02B4B2B4A5878F5
:106B60002B4B02EB001149681868FEF70BFB41E064
:106B7000274D2868FEF70BFB00283ED0224C2178D9
:106B8000264601291ED1FEF72FFB06466069321A00
:106B9000632A35D92169042912D81C4F286807EBCC
:106BA00001135968FEF7EEFA607807EB0017B96831
:106BB0002868FEF7D2FA22696661511C21611CE047
:106BC000022018E022693AB96478104B286803EB78
:106BD00004114968FEF7D6FA33690B4C8B2B09D8A0
:106BE0000C4A0B48D15C0068FEF7B2FA21694B1CD5
:106BF000236102E00320FFF7BBFE034A0020506040
:106C0000F8BD00BF001000207810002060070108C8
:106C1000D40F0020D206010810B50B4CE37A8BB1DB
:106C20000A48017804290DD9094A0A4B10685168AD
:106C300018605960FFF77EFE0748084B0288012163
:106C40001A80217310BD00BF0B1F0020F81E00200A
:106C5000E01E0020C41E00202E1E0020EE0F00208B
:106C6000002370B51C460F480021195214206043C0
:106C70000D4A0E4E0E4D995200223250595335187E
:106C80000C4E6960AA60325035180B4E01346960B1
:106C9000AA6002333518022C32506960AA60E2D132
:106CA00070BD00BF1010002002100020940F0020C3
:106CB0009C100020380F00202410002070B50446DE
:106CC0000079F9F71FFF1E49FAF728F81D4D1E4EEF
:106CD0002860A07BF9F716FF1949FAF71FF8EE6054
:106CE00068606079F9F70EFF1849FAF717F8184D40
:106CF0002860E07BF9F706FF1149FAF70FF86860A2
:106D0000607EF9F7FFFE1349FAF708F8EE60A86015
:106D1000A079F9F7F7FE0D49FAF700F80E4D286053
:106D2000207CF9F7EFFE0649F9F7F8FF6860A07ECE
:106D3000F9F7E8FE0749F9F7F1FFEE60A86070BDCA
:106D40000000C842C00F00200000FA4400002041AB
:106D5000740F002000007A44840F0020F7B51F460E
:106D6000224B234D18600024C3686C70214800EB4F
:106D7000041675689D4207D00134E4B2042CF5D99D
:106D80001B4E0020707001E0194B5C701A4E002001
:106D900031701A49164D0A60FFF7EAFDFEF724FA32
:106DA00032780024A8603846A2420CBF0126032690
:106DB0006C60FFF783FF68780E4B214603EB0012EF
:106DC000009410205268334602F014FB0C4908600E
:106DD00030B94FF4807003B0BDE8F040FCF71EBD41
:106DE000012003B0BDE8F040FFF7C2BDA8100020AD
:106DF000781000206007010800100020D80F002044
:106E0000D40F002073B51D4B1D78032D32D12020E7
:106E100002F0BCF91A4E044638B102F071FB316839
:106E200020460969FEF7AEF909E032680090214674
:106E3000202012692B4602F0DDFA0446E0B1114D24
:106E40002868FEF795F930B12868FEF796F90146F3
:106E50002046FEF77DF92046FEF78AF90028EED09D
:106E6000084806682046FEF788F901463046FEF7D6
:106E70006FF9E4E7022000E028467CBD781000208E
:106E8000A8100020D40F0020F7B50368164C174D4A
:106E900023600968164E61600068FFF74BFD94E8B7
:106EA0000C0014480196009095E80300FFF794FD4C
:106EB0006B68114A61683668C81A1660F9F726FED1
:106EC0000E4A0F4F1168F9F775FEFAF739F829687D
:106ED000786020680B4A431A0B483B6001681660D3
:106EE0000A4BCA881A80FEBDF80F0020E01E002061
:106EF0005010002008100020F40F00202C0000206B
:106F0000AC10002064100020D80F0020A210002038
:106F1000264BF0B51D68024600F1100116781446A4
:106F2000AB195B78013203F00403DBB263B18A4230
:106F3000F4D10020F0BD13B10A225343DBB210F8A4
:106F4000011B30395B18DBB2211A0229F3DC002166
:106F5000844209D911B10A225143C9B210F8012B58
:106F6000303A8918C9B2F3E72E2E11D1013404202A
:106F700000220A2672432678AF197F7807F00407AB
:106F8000FFB217B1303A921901340138F1D100E063
:106F90000022074C6420614300FB021106240548CF
:106FA000B1FBF4F200FB0320F0BD00BFA401002000
:106FB00040420F00809698002DE9F04F9A4B8BB01D
:106FC0001868B8B9994C21784A1E032A00F26185E5
:106FD000DFE812F0F304F3043E0528052068FEF70D
:106FE000CCF8934904460B78012B00F0DF8008D3DE
:106FF000022B06D08C4C2068FEF7BAF80028EDD1A1
:10700000E0E7242C07D18B4B8B4A8C4C0021197064
:1070100011702170C5E02C2C02D02A2C40F0828007
:10702000854D844A2978864B157800205854854A26
:10703000B5B918781570472868D15978502965D1A5
:107040009878472840F01385D978472940F00F8574
:107050001B79412B40F00B850120107000F007BD1B
:10706000117801293AD1022D05D11846FFF750FFBA
:10707000754908604AE0032D07D11978532945D195
:10708000714802685342036040E0042D05D1184660
:10709000FFF73EFF6C4B586038E0052D07D11B7899
:1070A000572B33D168494A68504248602EE0062D7C
:1070B00007D119786548302994BF00210121C17298
:1070C00024E0072D04D1FFF7C9FC614A10701DE0D0
:1070D000092D1BD1FFF7C2FC5E4B16E0022915D12A
:1070E000072D0CD10120FFF7B9FC41F218425043A3
:1070F0004FF47A71584BB0FBF1F0188006E0082D80
:1071000004D10120FFF7AAFC544B1880494B4A498F
:10711000013500202A2C1D70087039D150480124F7
:1071200004703EE00D2C4E4A01D00A2C26D1147872
:10713000FCB1434C21786478A1F13000C3B2092B33
:1071400084BFA1F13703DBB2A4F1300003F00F02DA
:10715000C3B21101092B84BFA4F13703DBB2374C52
:1071600003F00F0289182078CBB2C21A514251EBBA
:1071700002043B4B002018707CB912E02E490B78BA
:107180000E2B03D82E48C45401330B70127842B929
:107190002A4B1A7854401C7003E02A4A10780128C0
:1071A00000D00020C00700F1338123E72D4B0022DF
:1071B000197808293FF61EAFDFE801F00A0511191A
:1071C00027607C96A000622801D1022105E01A7098
:1071D000B52C7FF40FAF1C78611C19700AE72249A7
:1071E000224A03261E7008701070214B0BE01F4EC0
:1071F0000421197032781E4BA1181878CAB21018E1
:1072000018701C4B32701C70F4E605211970174B76
:10721000174E1A783078A118CAB210183070164E6E
:107220001A703480E6E600BFD40F002078100020EA
:107230000010002075100020F00F00206E0F0020BD
:10724000DF0F00204C100020E01E00200B1F00204C
:10725000F81E0020B21E0020B61E00205C10002088
:107260002C0F0020DD0F002068100020D00F002020
:10727000DE0F0020350F0020700F00206C4906261D
:107280001E700A786B4BA6181878F2B21018187096
:10729000694B0A70198801EB0424A6B2B6F5007F89
:1072A00001D81E8003E000221A80644B1A7000246B
:1072B00063497FE35E495F4E0A783078A318DAB2FB
:1072C000101830705E4E0A7033885B4AC72B98BF27
:1072D0005C49108898BFCC545C1CA1B288423180B4
:1072E0007FF488AE072107E0514808261E70037816
:1072F000A3423FF47FAE0021504B6EE74D4E1A7013
:10730000337883427FF476AE4F4C207806283BD00A
:1073100005D8022813D003287FF46CAE23E012288E
:1073200047D030287FF466AE464A484C1679454A25
:10733000102E88BF102626702178002347E0414C8C
:10734000434E6368A06821697360424B4FF47A72C0
:107350003060414C91FBF2F6187840492680C872A3
:1073600001223F4923E037494A7912F0010004D055
:107370000E79F41E634253EB04003649087000286E
:1073800039D1364AD07236E02E4EF47A14F001012B
:1073900004D0B07AC21E534253EB02012D4E31701D
:1073A00009B92E4CE17227482E4990F82F200A7017
:1073B00021E024482C498669426942F210742B4B23
:1073C00096FBF4F00A80188001222949EFE70C327D
:1073D0008B4210DA12F8046C264812F8034C1E5443
:1073E000254E26489C5512F8014C16781C54244C06
:1073F0001E550133EBE71A490A78002A3FF4FAAD2B
:107400001B4B1E78002E3FF4F5AD00240C701C7051
:107410001C4CA068E060FDF7E7FEA060202000F0B3
:1074200049FC19490A78012A30D100232FE000BF16
:10743000D00F0020DE0F0020700F0020DD0F002095
:10744000BC0F0020B8100020350F0020F91E0020CE
:10745000E01E0020A1100020B21E00200B1F002003
:10746000DC0F0020F81E0020B61E00205C1000205B
:1074700074100020A01E0020CE1E0020E81E002058
:10748000FA1E002078100020A410002001237E4C5A
:107490000B70E07A00283FF4ADAD7C490A78042AED
:1074A0007FF6A8ADA77807B92773257B15B90FB16B
:1074B000FFF7B2FB764E05213378764F5C1C94FBC8
:1074C000F1F001FB10423270734E97F800C0734D1B
:1074D00006EB82020023724C72491F59DFF810E25A
:1074E0007148724E5F5097FBFEF1195006FB017018
:1074F000DFF8009203EB040A42F2107490FBF4F7F9
:107500001668BCB253F809701060C6EB0708404417
:10751000052643F8090090FBF6F00EFB01016448D4
:10752000BCF1010F25F8024F195005D1023CB4F50A
:10753000797F98BFCAF8001004331432082BCAD1DF
:10754000FDF752FE5B4D5C4C2A68801AF9F7DAFAB7
:107550005A49F9F7E3FB2060FDF746FE28602568ED
:107560004FF07E512846F9F7C3FC08B94FF07E551D
:10757000256006A907AC4A48514B0194009103C805
:107580000CCBFFF729FA069A64234E49B2FBF3F0BD
:107590000880079A3C4892FBF3F34B4C027B238014
:1075A0000AB90A80228049490C78002C36D0424F13
:1075B0004FF07E503968F9F7B1FB454D384E2B68D6
:1075C00004463068C01AF9F7A1FA2146F9F7F2FA31
:1075D000F9F7B6FC726869683E4D0746501AF9F72C
:1075E00095FA2968F9F7E6FA2146F9F7E3FAF9F787
:1075F000A7FC04B238480225B0F902303FB2E218C5
:1076000092FBF5F1B0F900208BB2B918334C91FB25
:10761000F5F291B263802180438001802B4B0120E1
:107620001F4C1870184B6168294A20681C7A5160F9
:1076300010601CB9DA79002A3FF4DCAC284E294DE1
:10764000294C01960095164F94E80C00FFF7C4F9F9
:1076500061687868254E081AF9F758FA1D4B1968C1
:10766000F9F7A8FAF9F76CFC70600A48226890F9FB
:1076700000303C68012BC4EB020131603CD0022B8E
:107680007FF4B8AC9FE000BF0B1F0020F81E002065
:10769000B4100020340F0020040F00200A10002036
:1076A000E01E00209410002018100020806967FF61
:1076B000640F0020901000201410002000007A4475
:1076C000C41E0020C01E0020CC1E0020A0100020E0
:1076D0006C1000202C0000205E10002020100020E4
:1076E0005010002008100020F80F0020AC100020DF
:1076F0008096980054100020002634463546DFF866
:1077000018C3AF4F5CF825B0CDF80CC05846F9F758
:10771000FDF93968F9F74EFAF9F712FCDFF8DC9257
:10772000A84934F80920DFF8DC82801A83B21FB23E
:10773000635238460497A44FF9F7E8F93968F9F726
:1077400039FAF9F7FDFB4FF0140A0AFB058A82B2F9
:107750009E4B0498196805923B4658445246FFF7E1
:1077600013F90599DFF8B4B2DDF80CC00A1824F853
:107770000B205CF8250051463A46FFF791F99449F1
:107780004FF4FA62FCF710F934F809303BF80420A2
:10779000313399B2622998BF0020801883B22BF848
:1077A00004308C4940F6B83218B2FCF7FDF858F8AE
:1077B0000610894A01352BF80400B1500234143602
:1077C000022D9CD116E4854F2D683E686C08B6F9F1
:1077D0000820A24228BF2246814C97B2268839B29F
:1077E00030B2814209DD794B7E491868F9F7E2F938
:1077F000F9F7A6FB8719BFB227807B4A7B4E146836
:107800003168661A3046FFF783F80028D8BF404237
:1078100041F293139842CCBF0020012050B3304670
:10782000F9F774F97249F9F7C5F904F07FFD0646D6
:107830002846F9F767F901463046F9F7BBF9F9F739
:107840007FFB6C4A6349108000B240F6B832FCF707
:10785000ABF8201848F6A044A04203DDA0F50C4088
:10786000A03804E00028BCBF00F50C40A0306249FD
:10787000086001E0604D2C605F4B1D68C5F50C5041
:107880002830F9F743F95A49F9F794F9064604F014
:10789000D9FC0990304604F049FD002508902C469B
:1078A0002E4638B2F9F732F908AA52F82610F9F73D
:1078B00081F980465148DFF80C91005FF9F726F90D
:1078C00001464046F9F76CF8F9F73AFB4FF47A7243
:1078D00024F809004A4900B2FCF766F881B20BB2FD
:1078E000DFF83C8124F8091018460493F9F70EF9E3
:1078F000D8F80010F9F75EF9F9F722FBDFF8D8A005
:107900004FF0140B0BFB06AB049A30491FFA80FCB6
:107910000968434610465A46CDF80CC0FFF734F8C4
:1079200042460346594639F904000493FFF7B8F874
:10793000049ADDF80C80801808EB000CDFF8DC807E
:107940001FFA8CF124F8081008B240F6B832214929
:10795000FCF72AF855F80A202A4B013628F80400CB
:10796000EA5002341435022E9BD11C480368197961
:1079700031B1214A64201468234A94FBF0F111804C
:10798000224C1B88206898420ED91749174B0A6869
:107990001C68101BFEF7BCFF42F210710028B8BF34
:1079A000404288427FF726AB194B1A4A01201C88B7
:1079B000154910700C80FFF71DBBFFF7C7F868E092
:1079C000C00F0020600F0020740F00201410002052
:1079D00030F8FFFF48F4FFFF24100020D80F0020EC
:1079E000A21000200000C8425010002064100020A7
:1079F000D30237396C0F0020F40F00202010002034
:107A000018FCFFFF380F00201C1E0020081000206B
:107A1000EE0F0020340F0020AC1000209C1000203E
:107A2000840F002062686078531C411CCAB26360F6
:107A30000523B2FBF3F003FB10216170FDF7D4FBCB
:107A4000154AA06015480023C372137001200BE093
:107A5000FDF7CAFBA36840F6C411C01A884218D9C2
:107A6000202000F02FF90420FEF782FF11E00C49DE
:107A70008A78522A7FF44AABCB784D2B7FF446AB01
:107A8000087943287FF442AB064A02211170FFF7C0
:107A90003DBB0BB0BDE8F08FF81E00200B1F00208F
:107AA000DF0F00204C1000203D4B2DE9F047B3F9CB
:107AB0000000F9F72BF83B49F9F77CF8044604F08D
:107AC00035FC0646204604F0BDFBDFF8EC90054689
:107AD000D9F80000344F90F80380B8F1000F2BD094
:107AE000324CB7F90210B4F802A00FFA8AF2881AE1
:107AF000FEF70EFFC8F100014246FBF755FFB4F850
:107B0000008000EB0A03B7F900000FFA88F7C01BEA
:107B10006380FEF7FDFED9F80010CA785142FBF7EA
:107B200043FF00EB080297B22780B4F90200F8F790
:107B3000EDFF804638B206E0B7F90200F8F7E6FF3D
:107B40008046B7F90000F8F7E1FF294607464046AE
:107B5000F9F730F8314681463846F9F72BF80146F7
:107B60004846F8F71DFF1249F9F7D8F8F9F7E8F990
:107B7000104C314620804046F9F71CF8294606464D
:107B80003846F9F717F801463046F8F70BFF084971
:107B9000F9F7C4F8F9F7D4F96080BDE8F08700BFC1
:107BA0002E1E002035FA8E3C9C1000201010002064
:107BB0000000204102100020D80F002038B5254CCD
:107BC000E37A2246002B3ED02348017804293AD993
:107BD0002248817A79B1E179002939D12048214BB5
:107BE000012221721970011DE271FFF74DF91E4942
:107BF0000220087038BDC37AE171C3B11B4A106816
:107C0000408900F06DF890B1237A002B20D11548FF
:107C10001749037017480A684B680125011D026067
:107C200043602572FFF730F90F48057038BD0D48E5
:107C3000084B02780021197252B901210170BDE888
:107C40003840FFF70DB80023D3711372064A137042
:107C500038BD00BF0B1F0020F81E00201C1F002095
:107C6000C41E002028000020340F0020D80F002060
:107C7000E01E0020B81E0020074B1A68811A002958
:107C800008DB064A1178042904D900F5123000F502
:107C9000F8721A60704700BF300F0020F81E0020F5
:107CA000034B196808420CBF00200120704700BF39
:107CB00080110020024B1A6810431860704700BF03
:107CC00080110020024B1A6822EA000018607047F9
:107CD00080110020014B1868704700BF8011002000
:107CE000094BB3F90020002AB8BF5242824209DA98
:107CF000B3F902100029B8BF49428142ACBF00204D
:107D00000120704700207047321F002010B54478D2
:107D10000078002303FB03F11939614301F6C41114
:107D20005943414340F6C41291FBF2F1034A22F851
:107D300013100133072BEDD110BD00BF521F0020DF
:107D40002DE9F04384780A276743C678C4F1640CB0
:107D50001A4D5FFA8CFCC6F1640800231A1B12B29C
:107D6000002A04DCB8BF204602DB012000E06046A8
:107D700002FB02F9404309FB06F999FBF0F040448D
:107D800042434FF00A0992FBF9F2B81882B26A80B6
:107D90000888B1F8029012B2C0EB090902FB09F29F
:107DA0000A334FF47A7992FBF9F29BB28018782B60
:107DB00025F8020FD2D1BDE8F08300BF381F0020A4
:107DC000014B1860704700BF0C120020074B196868
:107DD0000B7A032B09D8DFE803F00202040600F057
:107DE000F1BB00F037BA00F01BBB70470C1200204B
:107DF00008B5037A032B12D8DFE803F00202070C60
:107E00000A490B4A00F0E6FB08E00849084A00F07E
:107E100029FA03E00549064A00F00AFB28B90820C0
:107E2000FBF7FCFC02480022026008BD601F002036
:107E3000A4110020174B10B5186004460023608978
:107E4000154A98520233242BF9D1144801600820B6
:107E5000FBF760FB10B12046FFF7CAFF4FF48030FC
:107E6000FBF758FB20B120460D490E4A00F098F967
:107E70000120FBF74FFB28B109480A49BDE8104033
:107E800000F09CB94FF40040FBF744FB0028F3D10D
:107E900010BD00BF0C120020641F0020A0110020A4
:107EA000601F0020A4110020037A032B09D8DFE80B
:107EB00003F00202040600F0C5BB00F0FFB900F0B9
:107EC000D5BA00207047000010B5114C00230820DF
:107ED0002370FBF71FFB20B10E480068FFF7E4FF9B
:107EE00020704FF48030FBF715FB094C10B100F007
:107EF0004DF92070217849B14FF40070FBF70AFB6F
:107F000020B1054A136818680168884710BD00BF92
:107F1000A81100200C120020A0110020054B197898
:107F200029B9054A1368C01AC143C80F7047012018
:107F3000704700BFA8110020101200200E4A0F4BFE
:107F4000127802F0030202EB800223F8121003EB16
:107F5000C00233F830105388CB189188D2885B1850
:107F60009918074A8BB222F81030042118B290FBFE
:107F7000F1F398B2704700BF9C110020AA110020B5
:107F800084110020F8B540F20120FBF7C3FA28B1B4
:107F9000FAF7B0F80746FAF7B9F800E0012700242D
:107FA000204B1878A0423BD91F49204A0B682BB9B7
:107FB00012681F49508921F814002EE01568072C1B
:107FC00094BF2E5D264617483146984705464FF424
:107FD0000070FBF79FFA38B137B116480168304698
:107FE0000B682946DA699047A5F2EE26B0B240F256
:107FF000DC51884202D90D4D2B685D8948F20100A1
:10800000FBF788FA0A4E10B926F8145005E020460E
:108010002946FFF793FF26F814000134E4B2BFE7C6
:10802000F8BD00BF601F0020A41100200C1200202A
:10803000641F0020A011002010B5064C237843B126
:10804000054801680A6813689847FFF79BFF0020FE
:10805000207010BDA8110020A0110020024B1A783A
:10806000501C1870FFF78EBF9C11002008B500F55A
:108070009C400D4B203018604FF40070FBF74AFA1B
:1080800020B10A490A6810680369984748F201005C
:10809000FBF740FA18B9BDE80840FFF7CDBFBDE8CF
:1080A0000840FFF7DBBF00BF10120020A011002026
:1080B000F8B505460F46441E14F8011F49B1054E98
:1080C000304606F0B7FF0028F6D0861B631BBB5571
:1080D000F2E7F8BDB007010810B5204B1A681C463E
:1080E000107C38B121680B7C5BB1591E1C4B33F8F6
:1080F00011001BE04FF40030FBF70CFA0028F1D11F
:1081000010BD4FF40030FBF705FA78B1F9F7C6FF60
:10811000124A80B211684B7C012B07D102B2B2F532
:108120007A7FC8BF002000F57A7080B20D4A002126
:10813000D08000B24FF47A72A0F57A70FBF734FC6D
:10814000F8F7E4FC0849F8F7E9FD0849F8F732FDCB
:10815000F8F71CFF0649088010BD00BF0C12002074
:10816000641F0020EE1D002000007A4400C07F4400
:10817000621F0020014B33F811007047641F00207C
:10818000014B01221A70704714120020034B18781B
:1081900010B100221A700120704700BF1412002095
:1081A00008230B700AB1024810600120704700BF1D
:1081B000758100080846FAF753B80000084B10B55F
:1081C00004460B604FF40040FBF7A4F908B1082007
:1081D00020700120FBF79EF908B10C21217010BD21
:1081E000B5810008034B53F82100410801F577726F
:1081F00090B270472012002038B50446FCF7DAFF31
:10820000104B40F6C4111A68821A8A421A460E4B65
:1082100001D9002119701B7810600BB90F2C10D1F7
:108220000A4800210170084A4BB1094D182B1D4422
:1082300005F8014C03D101230370117038BD0133DF
:10824000137038BD181200201C1200201D120020CF
:1082500050120020024B032143608360417370473A
:10826000A0860100F7B50025074605230E461446F3
:108270000D490E4A0095082001F0BCF879890C4B95
:10828000A1F57772186051002B460A4A99500433C1
:10829000302BFAD10CB1084921600C220030327029
:1082A00018BF0120FEBD00BFF9810008A0860100B3
:1082B0006C12002020120020E5810008344B10B51C
:1082C0001A780AB9002010BD00201870314B997D32
:1082D0000A07F7D4587819782F4A00F0070441EAC2
:1082E00004211160997801F03F04640144EAD00050
:1082F0005060DC78A00040EA9110197901F0010487
:1083000040EA84209060587900F00F04E40144EAC8
:108310005101D160997901F07F04240144EA1010E1
:108320001061DC79600040EAD111187A00F0030492
:1083300041EA44215161597A01F01F04A40144EA41
:10834000900090619C7AE00040EA5111D161187B65
:10835000D97A00F0070441EA04211162597B01F047
:108360003F04640144EAD00050629C7BA00040EAD4
:108370009110D97B01F0010440EA842090621B7CBB
:1083800003F00F00C30143EA5101D162012010BD87
:108390001D1200205012002020120020024B53F822
:1083A0002100C0F3CF007047A012002010B5044692
:1083B000FCF700FF154B1A68811AB1F57A6F1A465F
:1083C000134B01D9002119701060187820B9A82C1E
:1083D0001AD1104B187006E0022802D10E4A147010
:1083E00001E0242801D80D490C540B490130C3B2D7
:1083F0000878074A4100481D8342137004D10023C6
:108400000449137001220A7010BD00BFE012002061
:108410009C12002096120020701200207112002081
:108420004FF4E133012143608360417370470000E2
:1084300037B5002300930D461446094908204FF430
:10844000E132012300F0D6FF064908600CB1064A6C
:108450002260102300302B7018BF01203EBD00BFEA
:10846000AD830008981200209D830008124B10B5C0
:108470001A780AB9002010BD1049002018704B78F6
:10848000012BF7D10E480278102A01D91021017072
:1084900001780C4A0023D8B2023288420AD212F87C
:1084A000010C12F8024C40EA0424074840F823402B
:1084B0000133F0E7012010BD961200207112002058
:1084C0007012002074120020A0120020114B012213
:1084D00010B51A700446FCF76DFE0F4A014610688D
:1084E00011600B1A0D4841F288318B4203600C4B2E
:1084F00001D900221A7018780A49E4B20F280C54E6
:1085000003D109490120087010BD054A431C1370AE
:1085100010BD00BF1E1300203413002018130020CC
:108520001C130020211300201D1300201E4B2DE9D9
:10853000F0411A781AB31D4C1D4D2678077895F82E
:1085400000C002231B4A03F10108D45C44FA06F47C
:1085500004F00F04E5B2BD420BD20B2D09D8D55C57
:1085600012F8082005EA0C0502EB0525124A42F82C
:1085700024500233102BE5D10B4B00221A700078E7
:1085800088420ED90D4A107860B10D4B0A481A780E
:1085900050F8211002B1490801F5777398B2BDE88F
:1085A000F0810020BDE8F0811D130020E4120020BE
:1085B0002013002021130020E81200201E130020A9
:1085C0001F1300204FF4E1330121436083604173A6
:1085D0007047000013B5037A14465BB1012B13D129
:1085E000124A03201070124A0720107011480370BD
:1085F0000C2308E00D4A022010700D4A0320107071
:108600000C48037007230B70002100914FF4E132F6
:1086100008200949012300F0EDFE084A10600CB162
:10862000074B2360003018BF01201CBDE41200205E
:10863000201300201F130020CD84000838130020D1
:108640002D850008014B1878704700BF1D130020CE
:10865000014B1860704700BF40130020034B18689F
:108660000178D1F1010038BF00207047401300208D
:10867000034B186801784A1E534253EB02007047BF
:108680004013002008B54FF40060FAF743FF20B113
:108690000420BDE8084000F065BE08BD084B18780E
:1086A00060B108490A68537813B1074A117D01E0A7
:1086B00006488178081C18BF0120704701207047C8
:1086C0003C130020401300201C1F00200B1F002023
:1086D00008B5FFF7C3FF18B1BDE8084000F074BA51
:1086E000FFF7C6FF18B1BDE8084000F0A7BC08BD01
:1086F00008B5FFF7B3FF08B100F0A4F8FFF7B8FF23
:1087000018B1BDE8084000F039BB08BD0D4B10B5ED
:108710001878B0B1FFF7C2FF0B4904460A788242CD
:108720000FD050B1FFF79AFF08B100F0A3F8FFF7A0
:108730009FFF20B100F040FB01E0FFF7D9FF024BA3
:108740001C7010BD441300203D13002008B501210A
:10875000042000F013FE0C4B1870FFF793FF0B4939
:108760000870FFF77BFF18B10948006800F064F853
:10877000FFF77EFF18B1064A106800F017FBBDE84E
:108780000840FFF7C3BF00BF3C1300204413002084
:108790004013002008B5094B187870B1FFF77EFF31
:1087A00058B1FFF75BFF08B100F0A8F8FFF760FFD2
:1087B00018B1BDE8084000F013BC08BD4413002008
:1087C00038B5064C05465E212068FCF7C1FC2068E0
:1087D0002946BDE83840FCF7BBBC00BF5813002059
:1087E000024B5E211868FCF7B3BC00BF5813002091
:1087F00010B50A4C5E280146206805D15D21FCF7C2
:10880000A7FC20683E2105E05D2903D1FCF7A0FC10
:1088100020683D21BDE81040FCF79ABC58130020A9
:1088200010B50446C0B2FFF7E3FFC4F30720BDE86C
:108830001040FFF7DDBF0000014B1860704700BF1C
:108840005013002010B5084B084C19782068FCF72D
:10885000A3FC074920680968FCF794FC2068042100
:10886000BDE8104000F0C2BC4D130020581300209A
:108870004813002013B5042000F088FC154C014675
:108880002060A0B14279144B81681A70134A1160BC
:108890004FF41651FCF776FC20680221FCF77CFCB3
:1088A0002068042102B0BDE8104000F08DBC0C4BE4
:1088B000186802238278042000924FF4165200F0C8
:1088C00099FD054B41792060044A80681970106059
:1088D00002B010BD581300204D1300204813002093
:1088E0005013002008B5044B1868FCF741FCD0F188
:1088F000010038BF002008BD581300202DE9F041C9
:10890000FFF7F0FF002800F04081FCF76DFCA04B62
:108910001A68811A7C2940F2388118609D480478D1
:10892000651C0570002404F12406F0B2FFF748FF2F
:10893000994B33F91400F8F7E9F8984A054610887E
:10894000F8F7E4F801462846F8F7E8F99449F8F70B
:1089500031F9F8F7F5FA013400B2FFF761FF032CA3
:10896000E1D13020FFF72CFF8E49B1F90000FFF76D
:1089700057FFFFF735FF8748067816F0030629D121
:10898000894D1020FFF71CFF2B68642493FBF4F241
:1089900010B2FFF745FF2120FFF712FF296891FB76
:1089A000F4F004FB101484EAE473A3EBE47318B24C
:1089B000FFF736FF1420FFF703FF7C4AB2F90000EF
:1089C000FFF72EFF1C20FFF7FBFE3046FFF728FFC6
:1089D000FFF706FF6F490878430740F0B080744DF9
:1089E0000220FFF7EDFEB5F900300A2593FBF5F004
:1089F000FFF716FF0220FAF78DFD002847D06D4FD4
:108A00006D4E3878347840F63401B4FBF0F26B4C9C
:108A10004A4321882A2391FBF0F800FB1810B2FB8F
:108A2000F3F24FEA001399B241EA022C1FFA8CFECE
:108A3000C2F303224EEA02080620FFF7C1FE0FFA36
:108A400088F0FFF7EDFE20883F78431C9AB292FB36
:108A5000F7F107FB1120367820806E24744315232C
:108A600094FBF3F43A206427FFF7AAFEB4FBF7F671
:108A70003046FFF7D5FE3B20FFF7A2FE07FB16426C
:108A800091B24C1D94FBF5F000B2FFF7C9FE202017
:108A9000FFF706F9002850D0494C1320FFF790FE4D
:108AA0002568484F002DB8BF6D4295FBF7F630B2F0
:108AB000FFF7B6FE1B20FFF783FE23680A26002B74
:108AC000B8BF5B4293FBF6F142F2107591FBF5F2F1
:108AD00005FB121000B2FFF7A3FE2320FFF770FE84
:108AE0002368002BACBF4E205320FFF799FE1220C5
:108AF000FFF766FE61680029B8BF494291FBF7F2B3
:108B000010B2FFF78DFE1A20FFF75AFE60680028AA
:108B1000B8BF404290FBF6F696FBF5F305FB1361F8
:108B200008B2FFF77DFE2220FFF74AFE6268002AA6
:108B3000ACBF45205720FFF773FEFFF751FE1548E5
:108B40000378282B21D100240470FCF74DFB4FF44F
:108B50007A753C24B0FBF5F61720FFF731FEB6FB23
:108B6000F4F5B5FBF4F104FB1152100200B2FFF76B
:108B700057FE1820FFF724FE04FB156318B2FFF719
:108B80004FFEBDE8F041FFF72BBEBDE8F08100BF0E
:108B9000541300204C130020581E00200400002015
:108BA00000007A44DC0D0020080D00202E1E00205D
:108BB000EC1D0020010000205C190020461300205D
:108BC000E01E0020A08601004FF4165070470A46B0
:108BD00010B50021044605F0D5FB7C238E20E02152
:108BE0007D2223706070E17084F82B2010BD0A464E
:108BF00010B50021044605F0C5FB7C238A20A02186
:108C00007D2223706070E17084F82B2010BD00007D
:108C10002C2108B50448FFF7DAFF04482C21BDE8F1
:108C20000840FFF7E4BF00BFA81300206413002032
:108C30002DE9F041314B32481978324AC07A9176A9
:108C40001346002856D0042901D9332400E03224E9
:108C50002D48DC7605682D4CEE0F95FBF4F85E721E
:108C60002B4E5FFA88F806FB085706256F4342F241
:108C70001072B7FBF2FC02FB1C7740681F7390FB7D
:108C8000F4F43F0AE4B25F73C70F06FB04006843C5
:108C9000B0FBF2F5642102FB1502E8B201FB04000F
:108CA000D873000A18741B485A74120A9A740288FE
:108CB0005FFA8CFC01FB08CC2420B2FBF1F14143AC
:108CC00015488AB2110ADA71028814481972DA74E6
:108CD000110A0288124819755A75110A028883F818
:108CE0000AC04FEA1C2C83F80BC09F7399751A7742
:108CF000BDE8F0812D21D176BDE8F081F81E00207D
:108D00000B1F002064130020E01E0020A08601003D
:108D10006079FEFFB61E0020C01E0020B21E00209B
:108D2000CC1E0020124BA52199711249D22009783E
:108D300058730A20484383F82000000A83F8210072
:108D40000D48002200789A701A71DA719A731A72BB
:108D5000DA735A721A74DA775A75CA0798771875DF
:108D600001D580221A71142119765976704700BFF7
:108D7000A8130020D41300205C19002010B5084B64
:108D8000084C19782068FCF707FA07492068096839
:108D9000FCF7F8F920680421BDE8104000F026BA7D
:108DA000D5130020A413002098130020014B186055
:108DB000FFF72EBFD813002013B5042000F0E6F90A
:108DC000144C01462060A0B14279134B81681A709F
:108DD000124A11604FF49641FCF7D4F92068012142
:108DE000FCF7DAF92068042102B0BDE8104000F079
:108DF000EBB900904FF496420123042000F0FAFAF8
:108E0000054B42792060054980681A70086002B0FD
:108E100010BD00BFA4130020D5130020981300201C
:108E2000044B1A7822B9044B0131186003480170D1
:108E3000704700BF5D13002060130020A0130020C6
:108E400001482C21FFF7ECBF64130020034B2C21B9
:108E50001A78501C18700248FFF7E2BFD4130020A4
:108E6000A813002008B5FFF75DFFBDE80840FFF735
:108E7000DFBE00008A2808B508D08E2810D10F4B1D
:108E80001A78501C1870FFF7E1FF09E00C49202008
:108E90000B785A1C0A70FEF703FF08B1FFF7D0FFEA
:108EA000084801784B1CDAB2027007480449028076
:108EB000024A0B7811784380818008BDD6130020C8
:108EC000E113002094130020EE1D002010B5054C86
:108ED0002068FCF74DF918B12068FCF74EF9F6E769
:108EE00010BD00BFA413002070B5154D06462868BC
:108EF000FCF73EF9012821D90228124C03D0FFF7D4
:108F0000E5FF012204E022780F4B1AB11E60002217
:108F1000227070BD1868361AB6F57A6F0ED301212B
:108F200028682170FCF729F904462868FCF725F920
:108F3000802C03D1BDE87040FFF79CBF70BD00BF1F
:108F4000A4130020300000209C1300201A4938B5DB
:108F50000C781A4B44B901220A7018680221FCF7F8
:108F60001BF9174B1C7038BD1648027852B91648C9
:108F70000A70026001211868FCF70EF9BDE838405C
:108F8000FFF7A4BF511EC9B201700D4A19B911787B
:108F9000481C107007E00C4C1578206810F8011B75
:108FA0004D1915702060094A10780130107018684A
:108FB000BDE83840FCF7CCB85D130020A4130020B6
:108FC0005C130020A013002060130020E013002099
:108FD000024B187880F00100704700BF5D1300203D
:108FE00038B5FCF7E7F8104D104A2B680446C01A54
:108FF000904202D9FFF736FF2C60FFF7E9FF10B16E
:109000002046FFF771FF0A490B6863B1094D2878C4
:10901000094D28B12A6840F6B733A11A994202D9FE
:10902000FFF794FF2C6038BD901300203F0D030024
:10903000601300205D130020DC1300204FF49640E5
:109040007047000010B500230C245C430549DAB2D8
:10905000615C814203D00133042BF5D11A461046DE
:1090600010BD00BF34000020037A002023B15A1E37
:1090700001301340C0B2F9E70A7A22B1511E013320
:109080000A40DBB2F9E7984294BF00200120704704
:10909000004870476400002000230549DAB2595C9B
:1090A000814203D00133092BF7D11A46104670478D
:1090B000B90701082DE9F74F167C81460F46144683
:1090C000032E3FD80C237343204A02EB030A9AF87D
:1090D000081019EA010F32D0D05C00251C4A2B0180
:1090E000D15C814203D00135EDB2042DF6D14FEAB7
:1090F000051B402002EB0B080192FAF70BFA019ACC
:1091000020B912F80B00831E012B18D9797B19B1F5
:1091100098F80C20114212D07868D8F804309842A0
:109120000DD3B968D8F80820914208D801362570C7
:10913000C4F80880C4F804A0E760267403E0013690
:10914000F6B2BDE700242046BDE8FE8F34000020C3
:10915000C407010870B50A4C06460D4614220021CA
:10916000204605F00FF904210C220648064B05F0B5
:109170009FF9304629462246BDE87040FFF79ABF66
:1091800008140020340000206990000800220D4BD4
:109190000C2101FB0233197A814211D00132D2B283
:1091A000042AF4D10022074B0C2101FB0233197A67
:1091B000014005D10132D2B2042AF4D108467047E9
:1091C000586870473400002010B50023064A0C246C
:1091D00004FB03225468844203D00133042BF5D1ED
:1091E0000022517210BD00BF340000200023074A46
:1091F0000C2101FB03225168814203D00133042B6F
:10920000F5D1002200205072704700BF34000020CA
:1092100038B5002205461D4811014318405CA8429C
:1092200004D00132062AF6D1002038BD184C042D96
:109230000FCB84E80F001BD007D8012D0FD0022DD3
:1092400021D114490B68996810E0102D15D0202DFC
:1092500009D0082D17D12046FEF7B8FD11E00D48C2
:10926000026851680CE00B490B681969616007E0FE
:10927000FFF72EFA6060A06003E006480268D1683C
:10928000A160204638BD024838BD00BF040801086F
:10929000F8130020F4130020214B10B518600120B2
:1092A000FFF7B6FF01460120FFF754FF08B9002081
:1092B00010BD0220FFF7ACFF01460220FFF74AFF76
:1092C0000028F4D01020FFF7A3FF01461020FFF77D
:1092D00041FF04464FF48070FAF71CF908B1002CE6
:1092E000E5D00820FFF794FF01460820FFF732FF82
:1092F00004460820FAF70EF908B1002CD7D0042054
:10930000FFF786FF01460420FFF724FF04464FF4D1
:109310000060FAF7FFF808B1002CC8D0012010BD9A
:10932000F4130020F8B50F4600240D4BE05C002339
:109330000B4E1D01715D7219814203D00133062B62
:10934000F6D100221146FFF705FF80680178B94287
:1093500004D01034602CE8D10020F8BD0120F8BD05
:109360000408010810B50446FFF752FF01462046E5
:10937000FFF7F0FE003018BF012010BD38B50546DC
:109380000C46FFF745FF01462846FFF7E3FE28B1EC
:109390004368187A04420CBF0020012038BD000049
:1093A000F8B505460020FFF74DFE104E0C272B7830
:1093B0000F4C07FB0060E15C01720120FFF742FEE9
:1093C00007FB00626878235C02201372FFF73AFE05
:1093D000AA7807FB0061A05C08720320FFF732FE49
:1093E000EB7807FB0061E25C0A72F8BD34000020F4
:1093F000B90701082DE9F04F87B01F4681460E4698
:1094000014469DF840B0FFF703FF0DF1080E054626
:10941000034600F1100C18685968724603C20833FD
:1094200063459646F7D1287B08B9039404944846CF
:1094300002A9FFF78FFE054640B141684B683BB17A
:10944000484602A92A46FFF735FEF4E7002432E039
:10945000826890F800A092F80080B8F1030FF5D868
:10946000DFE808F002061012CDF800B0144802E060
:109470001448CDF800B0224631463B46F9F77AF958
:1094800004460BE0002000E00120314622465B4606
:10949000F8F760FF39460446FBF77EFE002CD5D076
:1094A00084F804800848696840F82A404C602046E7
:1094B0004946FFF789FE204607B0BDE8F08F00BFA0
:1094C0000038014000440040E413002038B5064C49
:1094D00005462060FFF764FF284600F0FFFF206884
:1094E000BDE8384000F0E0BEF4130020034B1878CC
:1094F00008B100F0E1BD01F089B800BF1C140020E4
:1095000010B504462046FBF742FE18B90A20FBF7C7
:109510007CFEF7E710BD0000232801D100F0CCBD90
:10952000044B19680A7D824202D10120FBF7ECBE90
:10953000704700BFF413002010B5441E14F8011F3B
:1095400021B1034B1868FBF703FEF7E710BD00BF1E
:10955000541400200148FFF7EFBF00BFF0090108D5
:1095600010B50748FFF7E8FF0024064B06481A1914
:10957000E15852680C34FAF741FBC02CF5D110BD0C
:109580002E0A01080C090108440A010870B5FBF70E
:109590002BFE244C244B4FF47A71B0FBF1F11A7876
:1095A00022482378FAF72AFBFEF794FB0546204869
:1095B000204902682048B2FBF1F1FAF71FFB0024B2
:1095C0001E4B53F8241051B1012000FA04F0284238
:1095D00002D01B48FAF712FB0134E4B2F0E7022094
:1095E000FEF75EFB68B1174A174B1178174853F81E
:1095F0002110FAF703FB1648017A11B11548FAF762
:10960000FDFA154C1548FFF797FF2488F8F76EFA16
:109610000246134821464FF46C73BDE87040FAF7D8
:10962000EDBA00BF010000205C1900204C0A0108BF
:109630008801002040420F008A0A0108A018010892
:10964000A80A0108FE0C0020CC090108AC0A010898
:10965000F81D0020B60A0108CA0C00201C0D0108E4
:10966000BA0A010838B50C680546204605F0BEFD6B
:10967000024628682146BDE8384005F0E7BD0000F5
:1096800037B5037904460D46052B34D8DFE803F0DF
:1096900003060A0D1114816809782DE0806890F99D
:1096A000001029E08368198826E08268B2F900106A
:1096B00022E0816809681FE0806869460068FAF75F
:1096C00083FB01461148FAF799FAF5B1E068F7F71C
:1096D0001DFA6946FAF778FB01460D48FAF78EFA4B
:1096E0002069F7F713FA6946FAF76EFB0146084856
:1096F000FAF784FA09E000210648FAF77FFA25B163
:109700000548E1682269FAF779FA3EBDB30A010813
:10971000B20A0108F00A0108EC0A010808B5064877
:10972000FFF70AFF054B1868FFF7EAFE0020BDE8C7
:109730000840FBF7E9BD00BFF30A010854140020FC
:1097400008B50748FFF7F8FE064B93F8AC03F9F7A6
:1097500081FEF9F78FFEBDE80840FFF7DFBF00BFCD
:10976000020B0108601900207FB5044605F03EFD9C
:10977000082825D100231F49E25C086885186E7807
:1097800006F00301022908BF203AE2540133082BF6
:10979000F1D10025665D1848314605F04BFC28B133
:1097A00001356019314605F045FC18B11348FFF743
:1097B000C3FE1DE0082DEDD120461149FEF778FCCF
:1097C0001048FFF7B9FE00230F4A04A9981890F833
:1097D00008218818084A995C0133082B00F80C1CF2
:1097E000F2D100208DF80C0001A90848FAF706FA1A
:1097F0007FBD00BFA4010020B00701080C0B0108C9
:10980000681A00202C0B010860190020470A010883
:1098100008B5FDF7F7FA022801D0032804D1034860
:10982000BDE80840FFF788BE08BD00BF410B010836
:109830002DE9F041054605F0D9FC0446FAF7AEF8EB
:10984000064694B92A48FFF777FE2A4951F82410B2
:1098500049B1012202FA04F2324202D02648FAF754
:10986000CDF90134F1E7254821E028462449224674
:1098700005F0ECFC58B92348FFF75EFE224C54F883
:10988000041F0029EFD01C48FAF7B8F9F7E72B7846
:109890002D2B04D10135013C4FF0010801E04FF0C0
:1098A00000080026134850F8267027B91748BDE86D
:1098B000F041FFF741BE28463946224605F0C6FC76
:1098C000A0B9012000FA06F0B8F1000F03D0F9F7B3
:1098D000A5FF0F4802E0F9F727FE0E48FFF72CFE20
:1098E0000D483946BDE8F041FAF788B90136D9E7A5
:1098F000670B010864080108A80A01081C0D01088B
:109900007D1601087A0B0108600801088F0B010819
:10991000A90B0108B30B0108470A010810B504465A
:109920000848FFF709FE084A084809490023036070
:1099300013700B70FCF7A6FB2046BDE81040FFF744
:10994000FFBE00BFBC0B01081D14002050140020F6
:109950001C14002008B50448FFF7EEFDF9F7ECFDF4
:10996000BDE80840FFF7DABED40B01082DE9F0434B
:1099700089B0044605F03AFCC6B2002E6AD17A4896
:10998000FFF7DAFD794C20690021F7F7A7FA38BB19
:10999000013677483146FAF731F9206904A9FAF718
:1099A00013FA01467348FAF729F9606904A9FAF72E
:1099B0000BFA01466F48FAF721F9A06904A9FAF7F2
:1099C00003FA01466B48FAF719F9E06904A9FAF7B6
:1099D000FBF901466848FAF711F910340C2ED2D180
:1099E0000025664C2F46A8464FF000091034B145BB
:1099F00014DA404654F8101CF6F7D4FF54F80C1C47
:109A000080462846F6F7CEFF54F8081C054638462F
:109A1000F6F7C8FF09F101090746E7E75848CDF80E
:109A2000048002950397FFF787FD002401A82358BF
:109A3000544923F00040F7F779FA5349534A043464
:109A4000002814BF10460846FFF776FD0C2CEDD118
:109A50004F4871E020464F49052205F0F7FB38B921
:109A6000424B0022C1181030C0280A61F8D177E0BB
:109A700020464949042205F0E9FB054620460DBB76
:109A8000202105F0D7FA00286AD0461C304605F0A0
:109A9000ADFB2C460746414850F824500DB94048CC
:109AA0004AE030462946FAB205F0D0FB40B92046DC
:109AB0003C49FCF783FB3C482946FAF79FF847E00E
:109AC0000134E8E704F014FB461E0B2E074643DC86
:109AD0002046202105F0AEFA054640B1451C284637
:109AE000FAF7DAF9214B3F01D851012400E004468E
:109AF0002846202105F09EFA054640B1451C28461F
:109B0000FAF7CAF91949013401EB061250612846E7
:109B1000202105F08FFA054640B1451C2846FAF78A
:109B2000BBF9124B013403EB061188612846202152
:109B300005F080FA18B91D48FFF7FEFC10E001306F
:109B4000FAF7AAF9094A032C02EB0616F061F2D1E2
:109B50001748FFF70BFF03E016480C21FAF74EF801
:109B600009B0BDE8F08300BFF50B010860190020C3
:109B7000200C0108260C0108470A0108741900206E
:109B80002A0C01080AD7233CF10B0108ED0B010850
:109B90001C0D0108390C01083F0C0108B008010830
:109BA000440C0108701900205C0C01086F0C0108BE
:109BB0005B0F0108A90C0108F8B5074605F016FB74
:109BC000044638B91A491B4B4A791B48511E53F8B1
:109BD000211028E038461949224605F037FB60B9C4
:109BE0001748FFF7A9FC174C54F8041F19B1164881
:109BF000FAF704F8F8E7154805E000250D4B53F88F
:109C0000256026B91248BDE8F840FFF795BC3846F4
:109C10003146224605F01AFB01350028EED10448F2
:109C2000314645710B48BDE8F840F9F7E7BF00BF82
:109C300060190020B0080108D10C01087D16010848
:109C4000E50C0108AC080108A80A01081C0D010870
:109C5000440C0108F80C01082DE9F047064605F010
:109C6000C5FA054620B1012819D133782A2B16D11F
:109C70004748FFF761FC002414266643454F4648D9
:109C8000F159F9F7BBFFB8192946FFF7F9FC013480
:109C90004248FFF751FC742CEED1BDE8F087304606
:109CA0003D2105F0C7F9002857D0441C204604F098
:109CB0001FFA82462046FAF7EFF8002705461424DB
:109CC0007C43DFF8D09054F80980404605F08EFAC6
:109CD00041460246304605F0B9FA002835D14C44D9
:109CE000E068F6F713FF01462846F7F715F9002854
:109CF00029D02069F6F70AFF01462846F7F702F94E
:109D0000002820D020792279052818BF5546052A39
:109D10000FD8DFE802F003030606090CA1680D70F6
:109D200007E0A268158004E0A068056001E0A16872
:109D30000D6041461A48F9F761FF20460021BDE851
:109D4000F047FFF79DBC174803E00137742FB6D1E9
:109D50001548BDE8F047FFF7EFBB044614256543FF
:109D60000C4F314655F80780404605F041FD50B193
:109D700009484146F9F742FF78190021FFF780FCB6
:109D80000648F9F73BFF0134742CE7D1BDE8F087B2
:109D90000A0D0108C0180108E40E01081C0D010895
:109DA0001F0D01082A0D01084F0D010810B50446CA
:109DB000204605F01BFA10F0FF0F07D10B490C48A5
:109DC00091F8AC13BDE81040F9F718BF204604F035
:109DD0008FF9022808D8054B064C83F8AC03F9F735
:109DE00049FBF9F797FDE3E710BD00BF60190020BC
:109DF0006C0D01085B0F010870B5044605F0F6F91B
:109E000008B9204830E020461F4905F067FE0024CD
:109E10002646254678B12CB1012C06D104F068F90C
:109E2000064602E004F064F90546002016490134B4
:109E300005F054FEEEE70B2D05D914480C21BDE8C2
:109E40007040F9F7DBBE012C08DC114A114832F9E9
:109E500015202946BDE87040F9F7D0BEA6F57A7303
:109E6000B3F57A7F04D90C48BDE87040F9F7C6BE57
:109E70000A4829463246F9F7C1FE054820F8156020
:109E800070BD00BF820D0108250F0108BC0D01083F
:109E9000881E0020E20D0108FA0D01081C0E0108C1
:109EA00038B5054605F0A2F9C0B268B904461249B2
:109EB000124801EB4402B2F8462021460134F9F77A
:109EC0009DFE152CF3D138BD284604F011F9142855
:109ED00004460BDC2021284605F0ACF804F008F914
:109EE000054B03EB4404A4F8460038BD0448152193
:109EF000BDE83840F9F782BE141D0020350E010878
:109F0000410E01082DE9F043584885B0584CF9F747
:109F100075FE5848FFF7C4FF6279574B511E5748EA
:109F200053F82110F9F76AFE20690021F6F7D6FFF1
:109F3000002858D10025266900213046F6F7CEFFCB
:109F400000284CD101354E482946D4F81490D4F855
:109F50001880E769F9F752FE30460021F6F7C8FF8E
:109F600010B14848F9F74AFE69463046F9F72CFF28
:109F700001464548F9F742FE48460021F6F7B8FF8A
:109F800010B14048F9F73AFE69464846F9F71CFF18
:109F900001463D48F9F732FE40460021F6F7A8FF9A
:109FA00010B13848F9F72AFE69464046F9F70CFF28
:109FB00001463548F9F722FE38460021F6F798FFAA
:109FC00010B13048F9F71AFE69463846F9F7FCFE39
:109FD00001462E48F9F712FE10340C2DABD12C4857
:109FE000691CF9F70BFEF9F7D9FC2A4C064654F820
:109FF000041F19B12848F9F701FEF8E70D46274874
:10A0000050F8251049B1012202FA05F2324202D07D
:10A010002348F9F7F3FD0135F1E7154B214ACE1836
:10A0200096F808418B5C04A801310519082905F848
:10A03000103CF2D100241C4869468DF80840F9F71D
:10A04000DDFD14256543194E1948A959F9F7D6FDC8
:10A0500000217019FFF714FB01341648FFF76CFA62
:10A06000742CEED105B0BDE8F08300BF670E010887
:10A07000601900205B0F0108B0080108970E010865
:10A08000A20E0108250F0108B30A0108470A0108BA
:10A09000AA0E010860080108BC0E01086408010846
:10A0A000CA0E0108B0070108D70E0108C018010840
:10A0B000E00E01081C0D0108F0B56D4B87B01A7851
:10A0C0007AB96C4C0120187002212068FFF77CF8E7
:10A0D0002068F9F7BDFD6848FFF72EFA6748FFF7DB
:10A0E0002BFA644C2068FBF743F8002800F0BD8091
:10A0F0002068FBF742F809280146614A01D03F2851
:10A1000051D1002517685F4C2E462FB15E4821685B
:10A110003A4605F09BF810B9254606B926465B4934
:10A120000C348C42F1D3C6B13468D5F800E03B461C
:10A13000E05C1EF8031081420DD1534A41B92D2B2A
:10A1400006D820244E48D45401330360D15404E08F
:10A15000D0540133ECE74A490B60494A14681CB1FA
:10A16000AE4201D13C4612E04948FFF7E5F9AE4264
:10A1700009D856F80C0BFFF7DFF93E4B0921186898
:10A18000FAF7E6FFF3E73D48FFF7D6F900243C4B2A
:10A1900018688442A5D237493B4A0868115DFAF72E
:10A1A000D7FF0134F3E713682BB9042838D13648B8
:10A1B000FFF7B4FB59E00C2801D136488CE70A2997
:10A1C00001D00D2948D12E4D3348FFF7B5F92E4C5B
:10A1D0002A6832480023A35404930090294903A815
:10A1E00010220C23039403F087FF054638B1006862
:10A1F00004F0FCFF411CAA686018904702E0284860
:10A20000FFF79AF9002130221F4804F0BBF81849E3
:10A210001B4B0A7800201860002A7FF45FAF24E00F
:10A220000C28CAD07F2903D15BE72F2B3FF659AF0B
:10A230001F297FF656AF7E293FF653AF13B9202969
:10A240003FF44FAF104C581CE1540A4A0C4B1860B5
:10A250001068FAF77DFF44E77F29E6D10A4C581EC3
:10A260000021106021540F4839E707B0F0BD00BF4E
:10A270001C14002054140020EA0E0108220F0108CB
:10A28000501400200C0901081D140020CC090108FD
:10A29000270F01082C0F01081C0D01086596000806
:10A2A000370F0108580F010837B505460220FEF7A1
:10A2B0006DFF064C0146206030B90090AA6802206C
:10A2C0000323FFF797F820603EBD00BF5414002021
:10A2D000F8B5174E174C184D0746C1B230682170BB
:10A2E000FAF736FF22782B78C7F3072182EA0300BA
:10A2F000287030682170FAF72BFF21782A783068AF
:10A3000081EA0203C7F307412B702170FAF720FF9F
:10A310002078297880EA0102390E306821702A708D
:10A32000FAF716FF2B78207880EA03012970F8BD30
:10A33000601400205C14002058140020F8B50D4E65
:10A340000D4D0E4CC1B2074630682970FAF700FF78
:10A350002A782378391282EA030020702970306845
:10A36000C9B2FAF7F5FE23782A7882EA0300207052
:10A37000F8BD00BF601400205B14002058140020BA
:10A38000054B10B5044621461868FAF7E1FE03486C
:10A3900002785440047010BD60140020581400204E
:10A3A000034B04491A78885C01321A70704700BF69
:10A3B000591400207C14002010B5FFF7F1FF04466B
:10A3C000FFF7EEFF04EB002080B210BD10B5FFF7E1
:10A3D000F3FF0446FFF7F0FF04EB004010BD000060
:10A3E00038B5044624200D46FFF7CAFF4D20FFF77D
:10A3F000C7FF002C0CBF3E202120FFF7C1FF064BFA
:10A40000002228461A70FFF7BBFF04480078BDE819
:10A410003840FFF7B5BF00BF581400206514002076
:10A4200001460020FFF7DCBF01460120FFF7D8BF3F
:10A43000014B1878FFF7A4BF5814002070B50546EB
:10A4400008460E46FFF7ECFF2C467219D0B2E3B275
:10A45000984204D014F8010BFFF792FFF5E770BDA6
:10A4600010B5441E14F8010F10B1FFF789FFF9E78A
:10A4700010BD00002DE9F843002701240025144BEE
:10A48000187885421CDA1349134B15F801800C2209
:10A4900002FB0830406804F0A9FE81460CB13F1869
:10A4A0000CE026464E4509DA0B4A0C2101FB082335
:10A4B0005868805DFFF764FF0136F3E70135DEE79A
:10A4C00024B1F8B2FFF7ACFF0024D7E7BDE8F8836A
:10A4D0005A140020671400206C000020F7B5474D87
:10A4E000FF2115220746284603F04CFF00230220D7
:10A4F0002B70FDF7D5FB012418B102206C70A870F9
:10A5000003240420FDF7CCFB68B13C4E03214FF43B
:10A5100000503155651CF8F7FDFF18B10422725543
:10A52000023400E02C460220FDF7BAFB48B1334B61
:10A5300005201E190621072518557170B5700334C2
:10A5400004E00820FDF7ACFB0028F0D12020F8F74C
:10A55000E1FF18B1294B08221A5501344FF48070DD
:10A56000F8F7D8FF30B125480A2601190B25065502
:10A570004D700234224A214B5079082801D00E2810
:10A5800002D10C261E5501340D2104201955651CDD
:10A59000F8F7C0FF18B1194811224255A51C1849F7
:10A5A000132391F83921154E6C1C101C18BF012083
:10A5B0007355F8F7AFFF10B114203055AC1C114B98
:10A5C000114A00211C7011607A680024002100915A
:10A5D00001200323FEF70EFF20B94FF496423CB949
:10A5E0000124F3E7084C2368002BEDD12060EBE752
:10A5F00003B0BDE8F040FEF74BBD00BF671400207C
:10A60000601900205A14002060140020F8B5B54CE1
:10A610002068FAF7ADFD002800F03D852068FAF7C4
:10A62000ACFDB14A0346117871B9B0F1240463421C
:10A6300053EB040111700029E9D1AC4A9478002C45
:10A64000E5D1FEF769FFE2E7012904D14D280CBFEF
:10A650000223002321E0022904D13C280CBF03235C
:10A6600000231AE003290FD140284FF0000101D93F
:10A670001170CCE79E489F4C03709F482170017079
:10A680009E490B70042308E0042908D19B499C488B
:10A690000C78037063400B7005231370B7E705292E
:10A6A000B5D19448924C017822788A42934A07D9CE
:10A6B00014785C401470934A53544B1C0370A6E703
:10A6C0001078984240F0E2848D4B19787B2900F095
:10A6D0001F8300F2C5806E2900F0718360D868295D
:10A6E00000F0328325D8652900F0068219D8642944
:10A6F00040F0C7840720844CFFF792FEE620FFF766
:10A700003FFE6079FFF73CFE0020FFF739FE94F82A
:10A710001B017E4B7E4A00280CBF1046184600F0F5
:10A7200061BC662900F06682672940F0AA847948F6
:10A730000BE36B2900F0218323D8692900F00983FA
:10A740006A2940F09E841020FFF76AFE6748724C29
:10A75000C07AFFF715FE71490878FFF711FE2068EF
:10A76000FFF7B6FD6068FFF7B3FD6D4AB2F9000070
:10A77000FFF7E4FD6B4BB3F90000FFF7DFFD6A4A1A
:10A780001AE36C2900F00B836D2940F07A840620CF
:10A79000FFF746FE65490868FFF79AFD644A0BE338
:10A7A000732900F079833CD8702900F03783C0F01A
:10A7B0001783712900F04583722940F06284524C5E
:10A7C0001620FFF72DFE0020FFF7B8FDB4F9D000EA
:10A7D000FFF7B4FD574DB4F9D200FFF7AFFDB4F960
:10A7E000D400FFF7ABFDB5F9BA00FFF7A7FD0020D5
:10A7F000FFF7A4FD0020FFF76BFDB5F928000A2341
:10A8000090FBF3F0FFF79AFD94F80401FFF7B8FD11
:10A8100094F80601FFF7B4FD94F80501FFF7B0FDC9
:10A8200069E3762900F043830DD8742900F0218371
:10A83000752940F026842F20FFF7F2FD3E48FFF7F0
:10A840000FFE00F021BC772900F01683782940F034
:10A850001884384C3820FFF7E3FD04F1400507E287
:10A86000D02900F07D8300F2CA80CA2900F005815A
:10A870006CD8A42900F0E48310D8A02940F001840A
:10A880000C20FFF7CDFD2D492D4C0868FFF720FD6A
:10A890002C4A1068FFF71CFD2068A3E3C82900F0CC
:10A8A000DE80C92940F0ED83FFF77AFD0F4B1A4C8B
:10A8B000D872FFF775FD19490870FFF787FD206012
:10A8C000FFF784FD6060FFF777FD154A1080FFF702
:10A8D00073FD144B18801C48017841F00204047089
:10A8E000DAE000BF60140020641400200B1F002079
:10A8F000BC140020661400205914002058140020B5
:10A90000651400207C140020601900201C000080C9
:10A910001400008018000020E01E0020F81E002017
:10A92000B21E0020B61E00205C100020501E002029
:10A93000DC0D0020141D0020D0210108E8F7FF1FC6
:10A94000F0F7FF1FECF7FF1FA4100020CD2900F047
:10A95000118322D8CB2900F0A180CC2940F091832B
:10A96000FFF71EFDCC4CE077FFF71AFD84F82000BE
:10A97000FFF716FD84F82300FFF712FD84F824008A
:10A98000FFF70EFD84F82500FFF70AFD84F821008B
:10A99000FFF706FD84F822007EE0CE2900F0F48265
:10A9A000CF2940F06E83FFF707FDFFF705FDBB4C95
:10A9B000B94DA4F8D000FFF7FFFCA4F8D200FFF7D0
:10A9C000FBFCA4F8D400FFF7F7FCA5F8BA00FFF7EA
:10A9D000F3FCFFF7FBFCFFF7EFFC0A235843288545
:10A9E000FFF7DEFC84F80401FFF7DAFC84F80601C7
:10A9F000FFF7D6FC84F80501FFF7D2FC4CE0D5291F
:10AA000000F094810FD8D22961D0C0F07882D32988
:10AA10006DD0D42940F035839F4C0020FFF700FD16
:10AA200004F1400556E1F02900F0CF820CD8D62978
:10AA300044D0EF2940F02583FFF7BEFC964CA0855B
:10AA4000FFF7BAFC608527E0FA2900F0A582FE290D
:10AA500040F017830820FFF7E3FC0024ADE2002458
:10AA6000FFF7AAFC8E4A10530234102CF8D10020B4
:10AA7000FFF7D6FCFDF784FB06E38A4C04F10A05D8
:10AA8000FFF78EFC01346070FFF78AFCE072FFF77D
:10AA900087FCAC426075F3D100208BE20024824831
:10AAA00001788C42F8D2814D655DFFF785FC7A4ACA
:10AAB000013402EB4505A5F84600F0E70024FFF756
:10AAC0007BFC7B4A10530234102CF8D1E4E7794C1C
:10AAD000A478002CE0D1FFF763FC7049022881F8CC
:10AAE000AC0388BF81F8AC43F8F7C4FC3FE2FFF742
:10AAF00063FC714B1880CFE7704D0B20FFF790FC83
:10AB0000B5F90000FFF71AFCF6F7F0FF00B2FFF707
:10AB100015FC0220FDF7C4F805460420FDF7C0F837
:10AB200004460820FDF7BCF8820042EA44012943AC
:10AB300020208CB2FDF7B4F844EAC00084B21020A3
:10AB4000FDF7AEF844EA001318B2FFF7F7FB594AD5
:10AB50001079D17884009378907944EA41011943BF
:10AB600041EAC0045179537A44EA411040EA83141F
:10AB70005348C17944EAC113047A417A43EA042371
:10AB800043EA4124D379117A44EA8324927A44EA4D
:10AB9000C123417B43EA0234827B44EA4133017C96
:10ABA00043EA8234027944EA0143417C43EA0214D5
:10ABB000827C44EA4143C17C43EA8244007D44EA0A
:10ABC000C142394B42EA00540020197803468B42B7
:10ABD0000AD2364D01225D5D02FA05F525421CBF01
:10ABE0009A4010430133F2E72C4CFFF771FB94F8C5
:10ABF000AC0381E11220FFF713FC32490C88B4F555
:10AC0000806F314CB4F9000008D8FFF797FBB4F916
:10AC10000200FFF793FBB4F904000EE0082590FB57
:10AC2000F5F0FFF78BFBB4F9020090FBF5F0FFF7AE
:10AC300085FBB4F9043093FBF5F0244CFFF77EFB61
:10AC4000B4F90000FFF77AFBB4F90200FFF776FBD6
:10AC5000B4F904001E4CFFF771FBB4F90000FFF7D4
:10AC60006DFBB4F90200FFF769FBB4F90400B6E12B
:10AC7000B4F97800FFF762FBB4F97A00FFF75EFBE6
:10AC8000B4F97C00FFF75AFB94F87E000834FFF714
:10AC900077FBAC42ECD1F7E1141D002060190020D5
:10ACA000641F0020131D00205A1400206714002088
:10ACB000881E00200B1F00201C1E0020CA0C002034
:10ACC0001C1F002004000020581E0020C40D00207E
:10ACD000041E0020FFF770FBA4F87800FFF76CFB60
:10ACE000A4F87A00FFF768FBA0F57A7107288AB20A
:10ACF00098BF84F87F00B2F57A7F98BFA4F87C00F3
:10AD0000FFF74EFB84F87E000834AC42E2D1BBE191
:10AD10000820FFF785FB0024B44AA31893F87F00AE
:10AD20000834FFF72DFB402CF6D1ADE10020FFF7F2
:10AD300077FB0024FFF734FBAC4AA3180834402CFF
:10AD400083F87F00F6D19FE1A9481021FFF776FB39
:10AD50009AE1A84801784C0004F0FE00FFF760FB80
:10AD60000024A44A13789C4280F08E81A24830F9D6
:10AD70001400FFF7E3FA0134F3E70520FFF750FB77
:10AD80009E4BB3F90000FFF7D9FA9D48B0F90000D7
:10AD9000FFF7D4FA9B490A7802F00100ACE09A4C24
:10ADA0000620FFF73DFBB4F90000FFF7C7FAB4F93E
:10ADB0000200FFF7C3FA954AB2F900000FE107203D
:10ADC000FFF72EFB92480078FFF7DAFA0020FFF732
:10ADD000B5FA904BB3F90000FFF7B0FA0020FEE09F
:10ADE000824C0720FFF71CFBE07FFFF7C9FA94F8BD
:10ADF0002000FFF7C5FA94F82300FFF7C1FA94F892
:10AE00002400FFF7BDFA94F82500FFF7B9FA94F88B
:10AE10002100FFF7B5FA94F822006DE01E20FFF73D
:10AE2000FFFA7D4C04F10A0501346078FFF7A8FAB7
:10AE3000E07AFFF7A5FA607DFFF7A2FAAC42F3D102
:10AE400022E176490A78540004F0FE00FFF7E8FAA0
:10AE50000024724803789C4280F016817049634850
:10AE6000625C013400EB4203B3F94600FFF766FA77
:10AE7000EFE7FFF7FFFA07E1684900240878FFF7DA
:10AE8000CFFA664A1078844280F0FE80644B185DE9
:10AE9000FFF776FA0134F4E70820FFF7C1FA01243E
:10AEA000E0B20134FFF76CFA092CF9D1ECE0FFF7BE
:10AEB00077FA06461220FFF7B3FA0EB9594902E0B5
:10AEC000102E03D158490D684C6801E00024254636
:10AED0003046FFF755FA2846FFF7FAF92046FFF704
:10AEE000F7F9524A1068FFF7F3F90020FFF726FA46
:10AEF0000020FFF723FA0020FFF742FAC4E0FFF733
:10AF00004FFA0546FFF762FA0746FFF75FFA064673
:10AF1000FFF75CFA0446FFF74FFAFFF74DFAFFF729
:10AF20003FFA65B93F484249012207604660CD714A
:10AF30000A73002C3FF4B0AD3C4B1C60ACE5102D07
:10AF40007FF4AAAD3848076046600CB137490C6001
:10AF50003548384B0222011D1A70FBF795FF9BE51F
:10AF60003348817800297FF497ADF8F7E5FAF8F7D0
:10AF7000D1FC91E52E4CA378002B7FF48DAD4FF4DE
:10AF8000C870F9F7A7FE87E52948817800297FF482
:10AF900083AD012282737FE5254B9C78002C70D114
:10AFA000254991F8AC03F8F755FAF8F763FAF8F782
:10AFB000B1FC2046FFF734FA66E02048005F023417
:10AFC000FFF7BCF9082CF8D15EE0084C0420FFF72D
:10AFD00027FAB4F92C00FFF7B1F9B4F92A00FFF70A
:10AFE000ADF951E0FFF774F94EE000BF141D0020E9
:10AFF000701E0020601F0020641F0020C01E002063
:10B00000CC1E0020A4100020040E00202E1E0020C4
:10B010005C190020621F0020131D00205A1400201C
:10B0200067140020C41E0020B81E0020541E0020FB
:10B030000B1F0020340F002060190020EE1D00209F
:10B04000154C23789800411CC8B2FFF7E9F9207825
:10B05000FFF796F90024104A13789C4214D20F4847
:10B06000005DFFF78DF90E49085DFFF789F90D4A7C
:10B07000105DFFF785F90C4B185DFFF781F901347E
:10B08000E9E70020FFF7D0F9FFF7D2F907490020E0
:10B090000870FFF7BCBAF8BDF91E0020A01E002002
:10B0A000CE1E0020E81E0020FA1E0020641400209E
:10B0B0002DE9F0410746884616460024B4420ED0DA
:10B0C0000025BD4205D040460135FAF79EF8EDB2A5
:10B0D000F7E73C200134FAF798F8E4B2EEE7BDE870
:10B0E000F08100000F4B1A6842F0010018605968A7
:10B0F0000D4A0A405A60186820F0847121F48032A9
:10B100001A60186820F4802119605A684FF41F01F2
:10B1100022F4FE0058609960044B4FF000629A6080
:10B12000704700BF001002400000FFF800ED00E093
:10B13000164A174B516801F00C00042803D0082868
:10B1400005D0144801E014490868186011E05168FE
:10B150005068C1F383410231C00301D40F4A06E0B5
:10B1600052680D4812F4003F026818BF520851435C
:10B170001960064B0A485A68054BC2F30311415C3B
:10B180001A6822FA01F21A60704700BF00100240EC
:10B190008801002000127A008401002000093D008F
:10B1A000740100201FB50023574C4FF4E0110093A9
:10B1B000019302930391226842F480332360A169D2
:10B1C00041F01002A261504C236803F40031019158
:10B1D000009A531C0093019919B9009AB2F5A06F17
:10B1E000F1D12168484B11F4003401D0022416E05B
:10B1F0001A6842F0010119600094434B1C6804F086
:10B200000202019200994C1C0094019A1AB900990B
:10B21000B1F5A06FF1D11B6899073BD501243B49DB
:10B2200002940A6842F010030B600C6824F00302D9
:10B230000A600B6843F002040C60A1F58053596862
:10B2400059605A685A605C68314A44F480615960B8
:10B25000146824F0704111602E4C2F490C605C681A
:10B2600024F47C145C60146844F000441460946816
:10B2700024F400449460043A9268120449BF274AB7
:10B280004FF4E0120A604FF48012039202990129F0
:10B2900001D119E0FEE702291AD168B10398B0F58F
:10B2A000801F02D14FF4A01205E0039BB3F5E01F0D
:10B2B00002D14FF400120392134B5968039841EAEC
:10B2C000000242F4803002E0596841F46010586096
:10B2D0000D4B1A68184642F08071196002680A4BDB
:10B2E0009201FBD5596821F0030058605A6842F07A
:10B2F00002015960044B586800F00C02082AF9D189
:10B30000FFF716FF1FBD00BF0010024000200240E3
:10B310000410014000127A0084010020001BB700D5
:10B3200008B5154B98420BD101214FF4805000F025
:10B33000C9FD4FF480500021BDE8084000F0C2BDB7
:10B340000E49884207D14FF48040012100F0C6FD2C
:10B350004FF4804009E00A4A90420BD14FF400407C
:10B36000012100F0BBFD4FF400400021BDE8084082
:10B3700000F0B4BD08BD00BF0030014000380040FF
:10B38000003C00400B8810B54C88028823438C8811
:10B3900002F441522343CC8823430C8923434C8934
:10B3A00023438C892343CC89098A23431A4393B2CC
:10B3B0000380828B22F400631A04130C83830182BE
:10B3C00010BD038819B199B241F0400303E023F0A6
:10B3D00040010A04130C0380704781817047808903
:10B3E00080B27047038919420CBF002001207047CA
:10B3F000426810B522F470230A6823F4807444EA8A
:10B4000002030C7943EA04224260CB688A688468AC
:10B410001A43084B234013434A7943EA42038360AB
:10B42000097CC26A4B1E22F47002D9B242EA015270
:10B43000C26210BDFDF7F1FF836811B143F0010155
:10B4400001E023F0010181607047836811B143F48A
:10B45000807101E023F4807181607047836843F05C
:10B460000801816070478068C0F3C000704783683E
:10B4700043F00401816070478068C0F3800070472A
:10B48000836811B143F4A00101E023F4A0018160BD
:10B490007047092970B54FF003040CD94C430725B8
:10B4A0001E3C05FA04F503FA04F3C66826EA05050E
:10B4B0002B43C3600BE04C43072505FA04F503FA60
:10B4C00004F3066926EA050545EA03040461062A31
:10B4D0004FF005030DD8013A53431F2202FA03F23D
:10B4E00001FA03F1446B24EA020242EA01034363D6
:10B4F00070BD0C2A0DD853431F22233B02FA03F2DE
:10B5000001FA03F1046B24EA020242EA0103036335
:10B5100070BD53431F22413B02FA03F201FA03F1CB
:10B52000C46A24EA02021143C16270BD40F0BF60E8
:10B53000024B40F40031D960704700BF00ED00E0DD
:10B54000C37810B503B3164CE168CB43C3F30224B0
:10B550004178C4F1040201FA02F10F2222FA04F246
:10B560008478037822400A43110103F16043CAB290
:10B5700003F5614181F800230078012200F01F03E8
:10B58000410902FA03F007E00078012200F01F03EE
:10B59000410902FA03F02031024B43F8210010BDAB
:10B5A00000ED00E000E100E030B5048C24F001057E
:10B5B0002C04250C0584048BA5B225F0F3052A4341
:10B5C00042EA0313114A048C9042A4B29DB215D0F2
:10B5D00002F50063984211D0B0F1804F0ED0A3F570
:10B5E000983290420AD002F58063984206D003F563
:10B5F0008062904218BF24F00A0401D124F00204B2
:10B6000044F0010421430583018430BD002C014036
:10B6100030B5048C24F010052C04250C0584048B13
:10B62000058C24F440742405240D44EA022242EAE5
:10B630000333144AADB290429BB212D002F50062BD
:10B6400090420ED0B0F1804F0BD0A2F598329042CC
:10B6500007D002F58062904203D002F580629042EA
:10B6600007D125F0200242F0100545EA011189B208
:10B6700004E025F0A00545F010052943038301846B
:10B6800030BD00BF002C0140224A038890429BB28B
:10B6900012D002F5006290420ED0B0F1804F0BD074
:10B6A000A2F59832904207D002F58062904203D012
:10B6B00002F58062904203D14A8823F0700313435D
:10B6C000154A904208D002F58062904204D023F4DB
:10B6D0004073CA889BB2134303808B880A88838592
:10B6E0000C4B028598420FD003F5006290420BD0BC
:10B6F00002F54063984207D003F58062904203D080
:10B7000002F58063984201D1097A01860122828282
:10B71000704700BF002C014000100040038C70B542
:10B7200023F001021404250C0584068C8388028B07
:10B730009CB222F073052B040D881A0C26F0020629
:10B7400033042A434E880D891B0C3543ADB22B437D
:10B75000134DA8420FD005F50065A8420BD005F5A2
:10B760004065A84207D005F58065A84203D005F5DD
:10B770008065A8420ED123F008064B898D881E43B0
:10B7800026F004032B43CE898D8924F4407435437D
:10B79000ADB22C43C988848002838186038470BD46
:10B7A000002C0140038C30B523F010021404250C4A
:10B7B0000584038C8288048B23F0200324F4E6455F
:10B7C0002C040D88240C44EA05241D042B0C0D893F
:10B7D00092B243EA05134D88A4B243EA0513124D11
:10B7E0009BB2A84203D005F50065A84215D14D894A
:10B7F00023F080039BB243EA05134FF6BF751D404B
:10B800008B8822F4406245EA0315ABB28D8942EA87
:10B810008502CD8942EA850292B2C988828004837A
:10B820000187038430BD00BF002C0140038C30B57C
:10B8300023F480721404250C0584038C8288848B85
:10B8400023F4007324F073052C040D88240C2C437E
:10B850001D042B0C0D8992B243EA05234D8843EA5F
:10B860000523124D9BB2A84203D005F50065A842FE
:10B8700015D14D8923F400639BB243EA05234FF6AB
:10B88000FF351D408B8822F4405245EA0325ABB2B8
:10B890008D8942EA0512CD8942EA051292B2C98821
:10B8A000828084838187038430BD00BF002C0140E7
:10B8B000038C30B523F480521404250C0584038CCA
:10B8C0008288858B94B225F4E64215042A0C0D88F3
:10B8D00023F4005342EA05221D042B0C0D8992B279
:10B8E00043EA05334D8843EA05330A4D9BB2A8422B
:10B8F00003D005F50065A84205D18D8924F4804464
:10B9000044EA8514A4B2C98884808283A0F84010D8
:10B91000038430BD002C014000214FF6FF7383806B
:10B920000180C18041800172704700230380438001
:10B930008380C380038143818381C3817047002357
:10B940000122038043808280C38003817047038883
:10B9500019B199B241F0010303E023F001010A0497
:10B96000130C03807047B0F8443029B16FEA4343A9
:10B970006FEA53418AB201E059044A0CA0F844200E
:10B98000704783899BB20AB1194301E023EA0101A0
:10B9900081817047038B23F0080213041A0C1143B2
:10B9A00001837047038B23F4006213041A0C42EAEC
:10B9B00001218BB203837047838B23F008021304A9
:10B9C0001A0C114381837047838B23F400621304A4
:10B9D0001A0C42EA01218BB283837047818470473D
:10B9E000038B23F00C0213041A0C0283038B9AB20C
:10B9F000114301837047038B23F4406213041A0C34
:10BA00000283038B9AB242EA01218BB2038370470F
:10BA1000838B23F00C0213041A0C8283838B9AB25B
:10BA2000114381837047838B23F4406213041A0C03
:10BA30008283838B9AB242EA01218BB2838370475F
:10BA4000F8B50B880D4604464988AA8843B92B8966
:10BA5000FFF7AAFDE9882046BDE8F840FFF7C0BF20
:10BA6000042B08D12B89FFF7D3FDE9882046BDE8D8
:10BA7000F840FFF7C0BF082B0E462F89008C3BD142
:10BA800020F480731804030C2384A08B83B223F06A
:10BA9000F30343EA0717374B208CBFB29C4280B2B6
:10BAA00047EA020212D003F500639C420ED0B4F1C3
:10BAB000804F0BD0A3F598339C4207D003F58063E9
:10BAC0009C4203D003F580639C4207D120F40070B0
:10BAD00040EA06218BB243F4807305E020F4206035
:10BAE00041F4807140EA0103E9882046A28323845F
:10BAF000BDE8F840FFF78CBF20F480531804030C16
:10BB00002384A38B208C23F440731B051B0D43EA75
:10BB1000022242EA0733174A80B294429BB212D003
:10BB200002F5006294420ED0B4F1804F0BD0A2F522
:10BB30009832944207D002F58062944203D002F515
:10BB40008062944207D120F4005040EA063291B25C
:10BB500041F4805205E047F6FF52024041F4805123
:10BB60000A43E9882046A3832284BDE8F840FFF712
:10BB70005ABF00BF002C0140808E80B27047008FFA
:10BB800080B27047808F80B27047B0F8400080B2BA
:10BB90007047038A828911EA030092B203D01142EE
:10BBA0000CBF002001207047C9438AB2028270474F
:10BBB000038A30B50D460446EA8898B220F4405115
:10BBC00011432182A3892889A98823F4B05340EA2C
:10BBD0000102688923F00C0102430804030C1A4394
:10BBE00091B2A181A08AAA8983B223F4407187B05F
:10BBF0001143A18201A800F0F3F81848A3898442F8
:10BC00000CBF0498039819B200294FF019032A6851
:10BC100003FB00F001DA510000E09100B0FBF1F10C
:10BC20006423B1FBF3F21201100903FB1011A08988
:10BC300000B2002806DAC9003231B1FBF3F303F099
:10BC4000070005E009013231B1FBF3F303F00F0007
:10BC5000024390B2208107B030BD00BF00380140E0
:10BC6000838919B199B241F4005303E023F40051E0
:10BC70000A04130C83817047C1F3421310B50124E9
:10BC800001F01F01A34204FA01F101D10C3004E0DC
:10BC9000022B01D1103000E01430036812B143EAE6
:10BCA000010201E023EA0102026010BD838A9BB217
:10BCB0000AB1194301E023EA010181827047090AB0
:10BCC000012303FA01F3DA4391B2018070470000C7
:10BCD000034A044B02F188305A605860704700BF35
:10BCE0002301674500200240024B1A6942F08000A0
:10BCF0001861704700200240014BD860704700BFB8
:10BD000000200240084BDA68D20709D4D8684007FF
:10BD100008D4D96811F0100F0CBF0420032070471D
:10BD200001207047022070470020024010B50446F1
:10BD3000FFF7E8FF012806D11CB1FFF7E3FF013C44
:10BD4000F8E7052010BD002C08BF052010BD00003D
:10BD500073B5002306464FF400500D460193FFF7DC
:10BD6000E5FF04281AD10E4CAAB2206940F0010167
:10BD700021614FF400503280FFF7D8FF042808D12A
:10BD800002360196019B2D0C1D804FF40050FFF7E9
:10BD9000CDFF216941F6FE720A4022617CBD00BFE1
:10BDA0000020024038B505464FF43020FFF7BEFFB3
:10BDB000042812D1094C236943F002002061656117
:10BDC00021694FF4302041F040022261FFF7AEFFBD
:10BDD000216941F6FD730B40236138BD002002400C
:10BDE000204B10B55A6802F00C01042903D0082931
:10BDF00005D01D4B01E01D4C2368036011E05C6819
:10BE00005968C4F38342941CC90301D4184A06E05C
:10BE100016495B680A6813F4003F18BF5208544380
:10BE20000460104B5968C1F3031212498C5C02681C
:10BE300022FA04F242605C68C4F302240C5D22FA28
:10BE400004F484605C68C4F3C224095D22FA01F240
:10BE5000C2605B680849C3F38133CB5CB2FBF3F289
:10BE6000026110BD0010024000127A00840100201F
:10BE700000093D00900100208C010020044B5A690C
:10BE800009B1104301E022EA00005861704700BF89
:10BE900000100240044B9A6909B1104301E022EA04
:10BEA00000009861704700BF00100240044BDA693F
:10BEB00009B1104301E022EA0000D861704700BFD9
:10BEC00000100240044BDA6809B1104301E022EA95
:10BED0000000D860704700BF00100240044B1A6990
:10BEE00009B1104301E022EA00001861704700BF69
:10BEF00000100240024B5A6A42F08070586270474C
:10BF00000010024008B50B4B984207D14FF40010C7
:10BF10000121FFF7E3FF4FF4001006E04FF480002B
:10BF20000121FFF7DBFF4FF480000021BDE808404E
:10BF3000FFF7D4BF00540040F0B58688044687B0B0
:10BF400026F03F000D46010401A80E0CFFF748FF44
:10BF50002C4A0399B1FBF2F087B23E43A6802388B6
:10BF600023F0010213041A0C22802B68264A934204
:10BF70000AD85B00B1FBF3F0013783B2BFB227846C
:10BF8000032B98BF042320E0EE884BF6FF72964205
:10BF900004D103225343B1FBF3F305E019225343C9
:10BFA000B1FBF3F141F4804399B20A054FF4967264
:10BFB00008BF41F00101504341F400434FF47A714E
:10BFC00090FBF1F0421C91B22184A383228891B2AC
:10BFD00041F001032380208820F4816222F00201D5
:10BFE0000B04AA886989180C41EA02032989AA89E5
:10BFF000184380B241EA0203208098B2208107B042
:10C00000F0BD00BF40420F00A086010041F288331E
:10C01000002103604BF6FF724FF480438180C280A1
:10C020000181418183817047038819B199B241F040
:10C03000010303E023F001010A04130C038070479D
:10C04000038819B199B241F4807303E023F480713D
:10C050000A04130C03807047038819B199B241F4A4
:10C06000007303E023F400710A04130C038070478B
:10C07000038819B199B241F4806303E023F480612D
:10C080000A04130C0380704783889BB20AB11943DA
:10C0900001E023EA01018180704701827047008A34
:10C0A000C0B2704712B141F0010101E001F0FE01A0
:10C0B0000182704702684FF6FE73134003602D4BF8
:10C0C00000219842016041608160C16022D02A490C
:10C0D000884229D0294B984230D02949884237D00C
:10C0E000284B98423ED0284B984206D153F8681C02
:10C0F00041F4700043F8680C70472449884206D127
:10C1000051F87C0C40F0706241F87C2C7047204B59
:10C11000984206D153F8042C42F00F0143F8041C56
:10C1200070471C49884206D151F8183C43F0F00092
:10C1300041F8180C7047184B984206D153F82C2C34
:10C1400042F4706143F82C1C70471449884206D1B0
:10C1500051F8403C43F4704041F8400C7047104B9C
:10C16000984205D153F8542C42F4702143F8541CE2
:10C17000704700BF080002401C000240300002402F
:10C1800044000240580002406C000240800002401F
:10C19000080402401C0402403004024044040240EF
:10C1A0005804024070B506688C680D6A26F4FF4298
:10C1B00022F070060A6945EA04034C6913438A6950
:10C1C0002343CC6913431C434B6A44EA03028B6A42
:10C1D0001A4332430260CB680A6849684360826050
:10C1E000C16070BD0023036043608360C36003616E
:10C1F00043618361C361036243628362704719B123
:10C20000016841F0010303E002684FF6FE7313403A
:10C210000360704703680AB1194301E023EA010192
:10C220000160704741607047406880B2704700000D
:10C23000C3004CBF014B024B5860704700040240E2
:10C240000000024000B540F6D87320F00042C3F66B
:10C2500049739A4283B0014615DDB2F1FF4F03DB0B
:10C26000F4F79EFB03B000BD694600F095FB00F0BB
:10C270000302012A009801990ED0022A07D082B940
:10C2800000F0A0FDEEE7002100F09CFDEAE700F0E1
:10C2900099FD00F10040E5E701F040FC00F10040AD
:10C2A000E0E7012201F03AFCDCE700BF30B5C0F363
:10C2B000C754A4F17F031E2B83B0014621DC581C18
:10C2C0001DDBCD0F162B0CDD21F07F4323F4000086
:10C2D00040F40000963C00FA04F005B1404203B07F
:10C2E00030BD114850F825402046F4F75BFB019023
:10C2F00021460198F4F754FB20F0004121B90020B9
:10C30000EDE7F4F71DFEEAE720F07F4222F4000398
:10C31000C0F3C75043F40001C0F1960221FA02F0C5
:10C32000002DDCD0DAE700BFB022010800B540F6EE
:10C33000D87320F00042C3F649739A4283B0014695
:10C3400016DDB2F1FF4F03DBF4F72AFB03B000BDAB
:10C35000694600F021FB00F00300012815D00228F7
:10C360000BD0B8B900980199012201F0D7FBEDE795
:10C370000021002201F0D2FBE8E700980199012298
:10C3800001F0CCFB00F10040E0E70098019900F0DB
:10C3900019FDDBE70098019900F014FD00F1004061
:10C3A000D4E700BF70B58AB0064600F09BF8224C77
:10C3B000054694F90030013303D0304601F0B0FD5A
:10C3C00010B928460AB070BD304601F05BFD4FF051
:10C3D0007E51F4F7ABFD0028F3D0184A0121002567
:10C3E0003046019200910895F4F720F802460B467A
:10C3F0001348CDE90423CDE9022301F011FC94F99F
:10C400000030CDE90601022B0BD0684601F006FC96
:10C4100038B1089850B9DDE90601F4F76DFA054620
:10C42000CFE701F089FE21210160F2E701F084FEEF
:10C43000089A0260EFE700BFA0010020B8220108BF
:10C44000C022010800F002BA70B58AB0054600F0BB
:10C450004FFC224C064694F90030013308D02846A0
:10C4600001F05EFD20B128460021F4F741FD10B92E
:10C4700030460AB070BD1A4A0121284600260091B4
:10C4800001920896F3F7D2FF2478CDE90401CDE9B3
:10C4900002017CB900220023CDE90623684601F0A1
:10C4A000BDFB88B10898A0B9DDE90601F4F724FACC
:10C4B0000646DDE70020002102460B46F4F734F97A
:10C4C000022CCDE90601E9D101F036FE21230360FB
:10C4D000E8E701F031FE08990160E5E7A0010020DE
:10C4E000C4220108F8B520F00043B3F17E5F044692
:10C4F00013D00BDCB3F17C5F14DAB3F10C5F00F303
:10C50000A48040F6DB70C3F6C970F8BD0146F4F7AD
:10C5100047FA0146F4F702FCF8BD002840F30E810B
:10C520000020F8BD0028C0F20E8101464FF07E5079
:10C53000F4F736FA4FF07C51F4F73CFB044600F078
:10C54000D7FB4EF60871064620F47F65C3F611014D
:10C550002046F4F72FFB47F60471C3F64F21F4F79A
:10C5600021FA2146F4F726FB41F24611C3F6245185
:10C57000F4F716FA2146F4F71DFB40F6A821C3F69E
:10C580004E61F4F70FFA2146F4F714FB4BF29001D9
:10C59000C3F6A661F4F704FA2146F4F70BFB4AF65A
:10C5A000AB21C3F62A61F4F7FDF92146F4F702FB4B
:10C5B0004CF22E610746C3F69D512046F4F7FAFA75
:10C5C00043F26131C3F63071F4F7EAF92146F4F72A
:10C5D000F1FA45F22D71C4F20101F4F7E3F92146B5
:10C5E000F4F7E8FA4DF23911C4F21901F4F7D8F969
:10C5F0002146F4F7DFFA4FF07E51F4F7D3F9014604
:10C600003846F4F78BFB3146F4F7D4FA25F00F05E2
:10C61000074629462846F4F7CDFA01462046F4F7A6
:10C62000BFF9294604463046F4F7BCF901462046D6
:10C63000F4F774FB01463846F4F7B4F92946F4F7E9
:10C64000B1F90146F4F7AEF9F8BD0146F4F7B2FAD4
:10C650004EF60871C3F611010546F4F7ABFA47F63A
:10C660000471C3F64F21F4F79DF92946F4F7A2FAB5
:10C6700041F24611C3F62451F4F792F92946F4F732
:10C6800099FA40F6A821C3F64E61F4F78BF92946D2
:10C69000F4F790FA4BF29001C3F6A661F4F780F933
:10C6A0002946F4F787FA4AF6AB21C3F62A61F4F774
:10C6B00079F92946F4F77EFA4CF22E610646C3F664
:10C6C0009D512846F4F776FA43F26131C3F6307192
:10C6D000F4F766F92946F4F76DFA45F22D71C4F2C4
:10C6E0000101F4F75FF92946F4F764FA4DF23911C4
:10C6F000C4F21901F4F754F92946F4F75BFA4FF044
:10C700007E51F4F74FF901463046F4F707FB014636
:10C710002046F4F74FFA014642F26810C3F2A23005
:10C72000F4F73EF901462046F4F73AF9014640F69F
:10C73000DA70C3F6C970F4F733F9F8BD40F6DB7070
:10C74000C4F24900F8BD4FF07E51F4F72BF94FF0D9
:10C750007C51F4F72FFA4EF60871C3F61101044626
:10C76000F4F728FA47F60471C3F64F21F4F71AF9E3
:10C770002146F4F71FFA41F24611C3F62451F4F7AB
:10C780000FF92146F4F716FA40F6A821C3F64E61D8
:10C79000F4F708F92146F4F70DFA4BF29001C3F6CD
:10C7A000A661F4F7FDF82146F4F704FA4AF6AB2146
:10C7B000C3F62A61F4F7F6F82146F4F7FBF90646CA
:10C7C000204600F095FA4CF22E610546C3F69D51C5
:10C7D0002046F4F7EFF943F26131C3F63071F4F714
:10C7E000DFF82146F4F7E6F945F22D71C4F20101B4
:10C7F000F4F7D8F82146F4F7DDF94DF23911C4F217
:10C800001901F4F7CDF82146F4F7D4F94FF07E5131
:10C81000F4F7C8F801463046F4F780FA2946F4F7F1
:10C82000C9F942F26811C3F2A231F4F7B9F801462E
:10C830002846F4F7B7F80146F4F7B4F8014640F695
:10C84000DA70C4F24900F4F7ABF8F8BDF8B521F09E
:10C850000044B4F1FF4F034617DC20F00045B5F16A
:10C86000FF4F064611DCB1F17E5F42D08F1707F013
:10C87000020040EAD37775B9022F35D0032F08D1D3
:10C8800040F6DB73CCF2490303E01846F4F78AF86C
:10C8900003461846F8BDD4B1B4F1FF4F2DD0B5F121
:10C8A000FF4F14D02C1BE4153C2C18DC002952DB64
:10C8B0001846F4F733FA01F0E5FA01F0B7F9012F61
:10C8C00046D0022F35D0002F25D10346E1E7002EB8
:10C8D00040F6DB731CDBC3F6C9731846F8BD40F69F
:10C8E000DB70C3F6C970EAE740F6DB73C4F24903B4
:10C8F000CFE7BDE8F84001F099B9B5F1FF4F2FD06F
:10C90000022FF1D0032FBBD0012F34D00023C0E77A
:10C91000CBF6C973BDE74BF62E51C3F2BB31F4F72A
:10C9200041F840F6DB71C4F24901F4F739F80346E7
:10C93000AFE74BF62E51C3F2BB31F4F733F80146A3
:10C9400040F6DB70C4F24900F4F72AF80346A0E78A
:10C9500000F100439DE714F13C0FA9DA0020AEE797
:10C96000022F13D0032F0CD0012F40F6DB7305D01C
:10C97000C3F649738DE74FF000438AE7CBF649735E
:10C9800087E74CF6E433CCF2160382E74CF6E43347
:10C99000C4F216037DE700BF2DE9F04F40F6D873CF
:10C9A00020F00044C3F649739C4289B006460D4608
:10C9B00040F38B804CF6E331C4F216018C4226DC46
:10C9C0004FF478610028C3F6C97140F32B81F3F767
:10C9D000E7FF4FF47D6224F00F04C3F6C97294425E
:10C9E000064600F0818044F24341C3F23571F3F70B
:10C9F000D7FF014628603046F3F7D2FF44F24341A7
:10CA0000C3F23571F3F7CCFF0127686061E04FF4A2
:10CA10007867C4F24937BC4240F38180B4F1FF4FDC
:10CA20005BDA4FEAE459A9F18609A4EBC954204620
:10CA3000F4F786FAF4F76AF80246014620460592B2
:10CA4000F3F7AEFF4FF08741F4F7B4F80746F4F779
:10CA500077FAF4F75BF80146044638460694F3F794
:10CA60009FFF4FF08741F4F7A5F800210790F4F7F6
:10CA700035FA002800F0F6800327204600210DF14A
:10CA80001808013FF4F72AFA40B158F8044D002184
:10CA90002046013FF4F722FA0028F6D1924B0220FB
:10CAA0000090019305A83B4629464A4600F066FAE5
:10CAB000002E07460DDA95E80C0002F1004103F163
:10CAC000004229606A60474203E000232860002793
:10CAD0004B60384609B0BDE8F08F0146F3F760FFC0
:10CAE000002768602860F4E74FF48841C3F235718D
:10CAF000F3F756FF4AF20831C2F685610446F3F7B0
:10CB00004FFF014628602046F3F74AFF4AF20831FA
:10CB1000C2F68561F3F744FF01276860D9E701F0A9
:10CB2000B1F94FF68411C3F622718046F4F742F84A
:10CB30004FF07C51F3F736FFF4F702FA0746F3F7AC
:10CB4000E5FF4FF47861C3F6C9718346F4F732F814
:10CB500001464046F3F724FF44F243418146C3F2C5
:10CB600035715846F4F726F81F2F8246514648463D
:10CB70001FDC5E4B7A1E53F8223024F0FF029A42EB
:10CB800017D0F3F70DFF8046C5F8008041464846B0
:10CB9000F3F706FF5146F3F703FF002E686098DABB
:10CBA00008F1004800F10041C5F8008069607F424B
:10CBB0008FE7F3F7F5FEE3158046C0F3C750191A67
:10CBC0000829E1DD4FF48841C3F2357158460393DB
:10CBD000F3F7F0FF824651464846F3F7E1FE04467C
:10CBE00021464846F3F7DCFE5146F3F7D9FE4AF2F8
:10CBF00008318146C2F685615846F3F7DBFF4946A6
:10CC0000F3F7CEFE824651462046F3F7C9FE039B5A
:10CC1000C0F3C7528046981A192841DCC5F8008035
:10CC2000A146B3E7F3F7BEFE4FF47D6724F00F048F
:10CC3000C3F6C977BC42064616D044F24341C3F25C
:10CC40003571F3F7AFFE014628603046F3F7A8FED2
:10CC500044F24341C3F23571F3F7A4FE4FF0FF37BE
:10CC6000686036E7032719E74FF48841C3F235714E
:10CC7000F3F798FE4AF20831C2F685610446F3F7ED
:10CC800091FE014628602046F3F78AFE4AF20831F9
:10CC9000C2F68561F3F786FE4FF0FF37686018E74C
:10CCA0004FF42341C2F685615846F3F783FF80466F
:10CCB00041462046F3F774FE814649462046F3F785
:10CCC0006FFE4146F3F76CFE43F232110446C2F2A6
:10CCD0008D415846F3F76EFF2146F3F761FE824619
:10CCE000514648464DE700BF4C230108CC220108BD
:10CCF00020F00042B2F1FF4FF8B50446034646D299
:10CD0000002A42D0002852DBC415B2F5000F09D228
:10CD100010F4000553D15B0001351902FBD5C5F1B4
:10CD20000100241823F07F417F3C21F40006E20734
:10CD300046F4000048BF400043004FF080720027D7
:10CD400060109A423C462CDD5B004FF4000218252F
:10CD5000A61851089E4205F1FF3502DCB4189B1B52
:10CD6000BF185B0062189A4202DC9B1A54187F18A5
:10CD70005B004A08013DEBD113B107F001017F18B8
:10CD80007C1004F17C5303EBC0542046F8BD0146EF
:10CD9000F3F710FF01462046F3F704FE0446204651
:10CDA000F8BD4FF0007403F17F431746CCE701460E
:10CDB000F3F7F6FD0146F3F7B1FF0446E5E701207E
:10CDC000AFE700BF2DE9F84320F00046B6F1485F19
:10CDD00005460F465BDAF4F7B3F8002800F0CA8086
:10CDE00029462846F3F7E6FE4DF24E71CAF6475142
:10CDF0000446F3F7DFFE47F2F641C3F20F11F3F7F3
:10CE0000D1FD2146F3F7D6FE4FF27C21C3F29341C8
:10CE1000F3F7C6FD2146F3F7CDFE40F60151C3F20C
:10CE2000D071F3F7BFFD2146F3F7C4FE40F6613140
:10CE3000C3F6B621F3F7B4FD2146F3F7BBFE4AF67D
:10CE4000AB21C3F62A51F3F7ADFD2146F3F7B2FE4D
:10CE5000804620464FF07C51F3F7ACFE4146064633
:10CE60002046F3F7A7FE394604462846F3F7A2FE0C
:10CE700001462046F3F794FD01463046F3F790FD56
:10CE800001464FF07E50F3F78BFDBDE8F883014675
:10CE9000F3F790FE4DF24E71CAF647510446F3F790
:10CEA00089FE47F2F641C3F20F11F3F77BFD2146ED
:10CEB000F3F780FE4FF27C21C3F29341F3F770FD4C
:10CEC0002146F3F777FE40F60151C3F2D071F3F734
:10CED00069FD2146F3F76EFE40F66131C3F6B621D7
:10CEE000F3F75EFD2146F3F765FE4AF6AB21C3F684
:10CEF0002A51F3F757FD2146F3F75CFE49F69913E3
:10CF0000C3F699639E428046A3DD0020C3F64870B5
:10CF1000864227DC06F17F464FF07E503146F3F71C
:10CF20003FFD814620464FF07C51F3F743FE3146EA
:10CF3000F3F736FD414606462046F3F73BFE3946F9
:10CF400004462846F3F736FE01462046F3F728FD4F
:10CF500001463046F3F724FD01464846F3F720FD2D
:10CF6000BDE8F8834FF000090026C3F63879C3F610
:10CF70009066D7E74FF07E50BDE8F8832DE9F04F7B
:10CF8000DFB00C930C9D224B689C0A91691ED61E43
:10CF900048BF161D834653F82400F71027EAE773AD
:10CFA0000890049104980D93089DDC43DDF834C08B
:10CFB00002EBC40241190792C0EB0C0750D47E1853
:10CFC000699BC7EB06090136002F03EB870522ACEE
:10CFD00009F0010AC0F2FE822868F3F797FD0137D5
:10CFE000B74220604FF004083AD0BAF1000F26D0C3
:10CFF000002FC0F2F18255F80800F3F787FD0137E2
:10D00000B74244F8080008F1040818D128E000BF2E
:10D010006426010855F80800F3F778FD013708F198
:10D02000040944F8080013D455F80900F3F76EFD1D
:10D030000137B74244F8090009F1040810D0002F65
:10D04000E8DA0020013708F1040944F80800EBD5BC
:10D0500001370020B74244F8090009F10408EED175
:10D06000089A002AC0F2458508990C9E8D004AABAB
:10D070005C19039549AF02944FEA860A049A002A84
:10D08000C0F296820DF1880808EB860555F8041C5D
:10D09000AAF10403DBF80000C3F38009F3F78AFD6B
:10D0A00001460020F3F77EFC0424043D54458046ED
:10D0B0002BD0B9F1000F0DD055F8041DDBF804009A
:10D0C000F3F778FD01464046F3F76CFC082454451D
:10D0D00080461AD055F8041C5BF80400F3F76AFD8B
:10D0E00001464046F3F75EFC0434804655F8081CC0
:10D0F0005BF80400F3F75EFD01464046F3F752FC8F
:10D100000434083D54458046E4D1029847F8048F22
:10D1100001368742B2D1039F0EA9CE190996089E07
:10D12000B2005EAB9D18002E029255F8509C7DDD3A
:10D130000DF5947C4FF06E5148460DACA7180CEBE2
:10D140000205F3F737FDF3F7FBFEF3F7DFFC4FF0D3
:10D1500087410190F3F72EFD01464846F3F720FC86
:10D16000F3F7EEFE0EAC20600198014655F8040D71
:10D17000F3F718FCBC428146C7F3800156D0E9B1F1
:10D180004FF06E51F3F716FDF3F7DAFEF3F7BEFC3E
:10D190004FF087410190F3F70DFD01464846F3F744
:10D1A000FFFBF3F7CDFE019A0FAC2060114655F856
:10D1B000040DF3F7F7FBBC42814637D04FF06E51B8
:10D1C0004846F3F7F7FCF3F7BBFEF3F79FFC4FF08D
:10D1D00087418046F3F7EEFC01464846F3F7E0FB53
:10D1E000F3F7AEFE4146606055F8040DF3F7DAFB45
:10D1F0004FF06E518146F3F7DDFCF3F7A1FEF3F734
:10D2000085FC4FF087418046F3F7D4FC0146484641
:10D21000F3F7C6FBF3F794FE4146A06055F8040D02
:10D22000F3F7C0FB0834BC428146C7D10799484692
:10D2300000F0A2FE4FF078510546F3F7BBFC00F07A
:10D2400025FE4FF08241F3F7B5FC01462846F3F77F
:10D25000A7FB0746F3F774FE8146F3F757FC014638
:10D260003846F3F79DFB07990746002940F33981BB
:10D27000721E0EAC079D54F82230C5F1080043FA27
:10D2800000F101FA00F0C5F107041B1A43FA04F497
:10D290000DF1380C89444CF82230002C55DD002E5D
:10D2A00009F1010940F39481029D0EABDDF808C03D
:10D2B00053F8042B281F0DF1380E00250EEB0C013E
:10D2C000C0F3800022B1C2F5807243F8042C01251E
:10D2D0008B4226D060B10F9A0433002D40F0F380CA
:10D2E00022B1C2F5807543F8045C01258B4218D049
:10D2F00053F8042B002D40F0EC80C2F5807012B181
:10D3000043F8040C012553F8042B002D40F0DB807A
:10D31000C2F58070002AE9D001258B4243F8040C45
:10D32000E6D1079900290DDD012900F0E2800229EC
:10D3300008D1701E0DF1380E5EF8202002F03F0378
:10D340004EF82030022C00F0E08038460021F3F740
:10D35000C5FD002800F0F3800898751EA84225DC62
:10D36000029B0DF1380E0EEB03010B46DDF824C0D5
:10D3700053F8042DCCEB0100011F6345C1F380007D
:10D3800011D030B153F8041DDDF824E00A43734591
:10D3900009D0099F53F8040D53F8041D0243BB4202
:10D3A00042EA0102F6D1002A40F01A81089F0EAD30
:10D3B000781E55F82020002A40F0108105EB8004EB
:10D3C000012354F8041D01330029FAD0F018771C0A
:10D3D00087420B9075DCDDF810E00D9D0B9B0C9CDB
:10D3E0000EEB0702DDF808C0699F991B06EB0509E3
:10D3F0004AA8A61922AB07EB890900EB0C05571CBC
:10D400008A0003EB8601029506920591002659F8E1
:10D41000040FF3F77BFB059CA051049800285EDB0A
:10D4200022AD05EB8702AAF10403C3F3800452F88E
:10D43000041CDBF800000394141FF3F7BBFB014648
:10D440000020F3F7AFFA4FF00408D04505462DD081
:10D45000039971B154F8041DDBF80400F3F7AAFB3B
:10D4600001462846F3F79EFA4FF00808D0450546D6
:10D470001CD054F8041C5BF80800F3F79BFB014632
:10D480002846F3F78FFA08F10408054654F8081CFB
:10D490005BF80800F3F78EFB01462846F3F782FAA3
:10D4A00008F10408083CD0450546E2D1DDF808E063
:10D4B000069804364EF8045F01378642CDF808E03E
:10D4C000A5D10B9E2CE6C2F1FF0243F8042C0125E6
:10D4D0000CE7C2F1FF0543F8045C012513E70025C2
:10D4E000E4E75ED1701E0DF1380E5EF820301C129C
:10D4F000D3E6711E0DF1380C5CF82100022C00F00F
:10D500007F024CF821207FF420AF39464FF07E5047
:10D51000F3F746FA0746002D3FF417AF07994FF08F
:10D520007E5000F029FD01463846F3F739FA0746E8
:10D5300038460021F3F7D2FC00287FF40DAF0294A7
:10D54000079C38466142CDF8109000F015FD4FF071
:10D5500087410546F3F7E0FC002800F0D2824FF047
:10D560006E512846F3F726FBF3F7EAFCF3F7CEFA01
:10D570004FF087410746F3F71DFB01462846F3F7B6
:10D580000FFAF3F7DDFC0EA941F826003846F3F751
:10D59000D7FC079A013608320EAC079244F82600F1
:10D5A00034E04FF07C51F3F7B7FC58B90024CCE6D7
:10D5B0004FF00008029847F8048F013687427FF445
:10D5C0005DADA8E50224002E09F101093FF76CAE1C
:10D5D0000025A6E6002002E5002010E50123F5E67F
:10D5E000079A0EAE56F82530083ACDF810900294FE
:10D5F0000792002B40F08E8206EB85042E4654F8ED
:10D60000045D013E083A002DF9D007924FF07E509C
:10D61000079900F0B1FC002E0446C0F2AC804FEA3E
:10D62000860AC6EB867B0EAF4FEA8B095744C9F1D9
:10D6300000034AA9386801EB0A08C3F3800BF3F72B
:10D6400065FA2146F3F7B6FA4FF06E51C8F80000BC
:10D650002046F3F7AFFAA9F104096FF0030ACA45AF
:10D66000054631D0BBF1000F0BD057F8040CF3F78F
:10D670004DFA2946F3F79EFA6FF0070A48F8040CB2
:10D680001AE057F80A00F3F741FA2946F3F792FA3D
:10D690004FF06E5148F80A002846F3F78BFAAAF1CA
:10D6A000040405463859F3F731FA2946F3F782FAAC
:10D6B000AAF1080A48F8040028464FF06E51F3F723
:10D6C00079FACA450546DCD1701CDFF84C94DDF8C8
:10D6D00020A0039000270596BAF1000FC0F2058242
:10D6E000002FC0F20282002600241AF0010F3546F6
:10D6F00020D0D8F80010D9F80000F3F75BFA014603
:10D700002046F3F74FF90125AA45044626DB0426F7
:10D71000BD420FDD22E0BB4520DC58F8021059F86D
:10D720000200F3F747FA01462046F3F73BF9BD4202
:10D73000044613DC58F8061059F80600F3F73AFAD5
:10D7400001462046F3F72EF905F1010B06F104021C
:10D750000235DA45044602F10406DCDA5EABDDF898
:10D760000CC003EB87010137674541F8A04CA8F1D5
:10D770000408B1D1059E689C032C16D8DFE814F08C
:10D7800085011F011F011B0000230299002900F0E1
:10D790000B81379C369804F100420A9C00F1004549
:10D7A00003F1004325606260A360049D05F007005B
:10D7B0005FB0BDE8F08F002EE6DD06F1FF3836AF32
:10D7C00007EB88094D4655F804290DF1D40AD5F820
:10D7D00008B0104659460192F3F7E4F880464146F6
:10D7E0000198F3F7DDF801465846F3F7DBF85545A5
:10D7F000C9F38003A860C5F8048044D0BBB155F8D4
:10D800000429D5F808B0104659460192F3F7CAF832
:10D810000199804608464146F3F7C2F8014658464A
:10D82000F3F7C0F85545C5F80480A8602BD02C4606
:10D8300054F80439D4F808B0184659460193F3F760
:10D84000B1F8804641460198F3F7AAF801465846D8
:10D85000F3F7A8F8C4F80480A06055F804BC251FAD
:10D86000D5F8088058464146F3F79CF8044621460F
:10D870005846F3F795F801464046F3F793F85545B7
:10D880006C60A860D3D1012E7FF77EAF4D4655F86E
:10D8900004B9C7EB090ED5F808A058465146AEF1B9
:10D8A0000409F3F77FF8804641465846F3F778F8C5
:10D8B00001465046F3F776F8BD42C9F38009C5F832
:10D8C0000480A86043D0B9F1000F15D055F804A921
:10D8D000D5F8089050464946F3F764F8804641462B
:10D8E0005046F3F75DF801464846F3F75BF8BD4252
:10D8F000C5F80480A8602AD02C4654F804A9D4F8AE
:10D90000089050464946F3F74DF880464146504648
:10D91000F3F746F801464846F3F744F8C4F80480A4
:10D92000A06055F8049C251FD5F80880484641465C
:10D93000F3F738F8044621464846F3F731F8014634
:10D940004046F3F72FF8BD426C60A860D4D1013691
:10D9500007EB860708353E467A1B131F56F8041D51
:10D960000020C3F38007F3F71DF8AE4203463FF4EF
:10D970000CAF3FB156F8041DF3F714F8AE4203465E
:10D980003FF403AF184656F8041C341FF3F70AF8A7
:10D99000083E54F8041CF3F705F8AE42F3D102999F
:10D9A000034600297FF4F5AEDDF828C03699379894
:10D9B000CCF80010CCF80400CCF80830F5E60023D1
:10D9C000002E29DB36AF751C07EB85042546E21BCC
:10D9D00055F8041DA2F1040E0020CEF38008F2F7E2
:10D9E000E1FFBD42034617D0B8F1000F06D055F84D
:10D9F000041DF2F7D7FFBD4203460DD0184655F877
:10DA0000041C2C1FF2F7CEFF083D54F8041CF2F75B
:10DA1000C9FFBD42F3D103460299002967D003F143
:10DA20000040DDF828C01946CCF800003698F2F71F
:10DA3000B7FF002E034621DD36AF07EB8606F51B48
:10DA40002A1F3799C2F38007F2F7ACFF37ACB44214
:10DA5000034613D037B16168F2F7A4FF38ACB44283
:10DA600003460BD0184654F8041FF2F79BFF54F8F6
:10DA7000041FF2F797FFB442F5D10346029909B1AA
:10DA800003F100430A9C63608FE6002E40DB36AF53
:10DA9000013607EB86000546C21B55F8041D002021
:10DAA000141FF2F77FFFBD42C4F38006034615D072
:10DAB00036B155F8041DF2F775FFBD4203460DD08F
:10DAC000184655F8041C2C1FF2F76CFF083D54F85B
:10DAD000041CF2F767FFBD42F3D10346029909B176
:10DAE00003F100430A9C23605FE6002436E61846F3
:10DAF00097E7DDF830E0900003904FEA8E0AFFF7D9
:10DB00000ABB2846F3F71CFA0EAB43F826007DE566
:10DB10000023E3E72E4679E5702601082DE9F84356
:10DB200020F00043B3F1485F04460F46904603DA05
:10DB3000F3F706FA002859D021462046F3F73AF8C1
:10DB400021460546F3F736F84CF6D311C2F62E718E
:10DB500006462846F3F72EF842F63471C3F2D72171
:10DB6000F2F71EFF2946F3F725F84EF61B71C3F2B4
:10DB70003861F2F717FF2946F3F71CF840F6015118
:10DB8000C3F65011F2F70CFF2946F3F713F848F6E5
:10DB90008901C3F60841F2F705FF8146B8F1000F8D
:10DBA00027D04FF07C513846F3F704F849468046B9
:10DBB0003046F2F7FFFF01464046F2F7F1FE2946F4
:10DBC000F2F7F8FF3946F2F7EBFE4AF6AB210546CD
:10DBD000C3F62A613046F2F7EDFF01462846F2F718
:10DBE000E1FE01462046F2F7DBFE04462046BDE892
:10DBF000F88301462846F2F7DDFF4AF6AB21C3F66B
:10DC00002A61F2F7CDFE3146F2F7D4FF01462046F5
:10DC1000F2F7C8FE04462046BDE8F88300207047AE
:10DC200000210020C7F6F871704700BF2DE9F041D0
:10DC300020F00045B5F1A14F044606460DDBB5F1D5
:10DC4000FF4F00F39C80002840F6DB7440F3D48043
:10DC5000C3F6C9742046BDE8F0814FF6FF73C3F6E2
:10DC6000DF639D4200F3A280B5F1445FC0F28E8075
:10DC70004FF0FF3721462046F2F79CFF01468046D1
:10DC8000F2F798FF46F6D711C3F685410546F2F73D
:10DC900091FF4DF65921C3F64B51F2F783FE294609
:10DCA000F2F788FF46F63531C3F68851F2F77AFE6F
:10DCB0002946F2F77FFF42F66E61C3F6BA51F2F7DA
:10DCC00071FE2946F2F776FF44F62511C3F612617C
:10DCD000F2F768FE2946F2F76DFF4AF6AB21C3F66C
:10DCE000AA61F2F75FFE4146F2F764FF4AF2212192
:10DCF0008046CBF615512846F2F75CFF4FF26B11C8
:10DD0000C3F66E51F2F74CFE2946F2F753FF48F284
:10DD10009571C3F69D51F2F743FE2946F2F74AFF8B
:10DD200048F63861C3F6E351F2F73AFE2946F2F7B6
:10DD300041FF4CF6CD41C3F64C61F2F731FE294666
:10DD4000F2F738FF7B1C0146404658D0F2F72AFE16
:10DD50002146F2F72FFF494B53F82710F2F720FE28
:10DD60002146F2F71DFE0146454850F82700F2F71C
:10DD700017FE002E3DDB04462046BDE8F08101463B
:10DD8000F2F710FE04462046BDE8F0814FF2CA21AA
:10DD9000C7F24911F2F706FE4FF07E51F3F7C6F8CD
:10DDA00000283FF465AF2046BDE8F08100F06AF836
:10DDB0004FF6FF71C3F697718D4204464FF6FF721E
:10DDC00028DCC3F62F72954246DC0146F2F7EAFDE5
:10DDD0004FF07E51F2F7E4FD4FF0804105462046BA
:10DDE000F2F7E0FD01462846F2F798FF00270446C7
:10DDF00040E700F100442DE7CBF6C9742AE7F2F7BB
:10DE0000D1FD2146F2F7D6FE01462046F2F7C8FDC5
:10DE100004461FE7C4F21B02954214DC4FF07F5109
:10DE2000F2F7BEFD4FF07F5105462046F2F7C2FEE5
:10DE30004FF07E51F2F7B6FD01462846F2F76EFF2D
:10DE40000227044616E700202146CBF68070F2F741
:10DE500065FF032704460DE74FF07E51F2F7A0FD62
:10DE60004FF07E5107462046F2F79CFD01463846AA
:10DE7000F2F754FF01270446FCE600BF9C26010888
:10DE8000AC26010820F00040704700BFF8B520F034
:10DE90000046F50D7F3D162D014604461BDC002D86
:10DEA000074620DB4FF6FF73C0F27F0343FA05F607
:10DEB00006420ED04FF2CA21C7F24911F2F772FDA5
:10DEC0000021F3F733F818B1002C1BDB27EA060416
:10DED00021460846F8BDB6F1FF4FFAD3F2F762FDCE
:10DEE00001460846F8BD4FF2CA21C7F24911F2F7C0
:10DEF00059FD0021F3F71AF80028E9D0002C07DBC0
:10DF00000024E5E74FF4000040FA05F56719DDE766
:10DF10000021CBF68071002E18BF0C46D8E700BF59
:10DF200008B902207047B0F1004FFAD0A0F5000206
:10DF30006FF001439A4201D80420704700F1FF417D
:10DF40009942F9D94FF6FE73421EC0F27F039A42FE
:10DF500001D80320704700F100414A1E9A42F8D9C7
:10DF6000B0F1FF4F05D010F5000F14BF00200120C5
:10DF700070470120704700BF38B530F000440346B9
:10DF800002460D460FD0B4F1FF4F0ED2B4F5000F8C
:10DF900011D3E40D6419FE2C33DC002C1BDD22F0C0
:10DFA000FF4141EAC453184638BD0146F2F7FAFC76
:10DFB0000346184638BD4FF09841F2F7FBFD43F693
:10DFC000B041CFF6FF718D42034612DBC0F3C75458
:10DFD0000246193CDEE714F1160F21DA4CF25032FA
:10DFE000954219460EDC44F26020C0F6A25000F0C3
:10DFF00023F844F26021C0F6A251F2F7DBFD03469C
:10E00000D1E719464FF2CA20C7F2491000F014F8C0
:10E010004FF2CA21C7F24911F2F7CCFD0346C2E71D
:10E0200022F0FF4304F1190043EAC0504FF04C5175
:10E03000F2F7C0FD0346B6E701F0004120F00040D2
:10E04000084370472DE9F041274C84B02568074606
:10E05000D5F84841002C41D066681F2E1CDD2348AE
:10E0600010B94FF0FF301FE04FF4C87003910292D7
:10E070000193AFF3008003990446029A019B0028A4
:10E08000EFD0D5F84861002060602660C5F84841AF
:10E09000C4F88801C4F88C01656847B9A81C01352B
:10E0A00044F820106560002004B0BDE8F081012034
:10E0B00000FA05F0D4F8886104EB85080643022FC6
:10E0C000C8F88820C4F88861C8F80831E6D1D4F8C7
:10E0D0008C3143EA0002C4F88C21DFE705F5A67411
:10E0E000C5F84841B8E700BFC42701080000000098
:10E0F00000210A2201F0C4BD2DE9F84FDDF828B057
:10E1000081468A4698469AB193B11646002503E0A7
:10E110000FD0651CAE420BD97419640808FB04A724
:10E1200048463946D8470028F2DA2646AE42F3D8A8
:10E1300000273846BDE8F88F40F2D053C2F2000302
:10E1400018687047114B124A70B5981A831018D08E
:10E15000591E02EB83040D4654F8042D01F001060C
:10E16000904775B126B154F8040D8047013D08D0A1
:10E1700054F8043D9847013D54F8041D8847013D7B
:10E18000F6D1BDE8704004F025BB00BFEC270108C4
:10E19000E8270108F8B5204F204C381B871017D00E
:10E1A0007A1E2368012502F001069847AF420FD07E
:10E1B0002EB154F8041F02258847AF4208D060688A
:10E1C00080470235A268261D90470834AF42F6D139
:10E1D000134F144C04F0F8FA3B1B9F1018D07D1E0F
:10E1E000216805F0010601258847AF4211D02EB104
:10E1F00054F8040F02258047AF420BD06268904765
:10E200000235A368261D98470834AF42F6D1F8BD01
:10E21000F8BDF8BDF8BD00BFE0270108E027010800
:10E22000E8270108E02701080F2A2DE9F00340F252
:10E23000A18041EA00039B0740F09E800C68A2F198
:10E24000100504604B68AC4643608C68BCF10F0F4E
:10E250008460CC68C5F30015C46000F1100301F1BF
:10E2600010042BD975B12568ACF1100C1D606568E0
:10E270005D60A5689D60E5681034DD601033BCF119
:10E280000F0F1BD9276804F110061F60676803F1A0
:10E2900010055F60A768ACF1200C9F60E768DF6045
:10E2A00024691C61776806F110046F60B768203339
:10E2B000AF60F668BCF10F0FEE60E3D8A2F1100872
:10E2C00028F00F0302F00F0403F1100C032C00EBF5
:10E2D0000C0301EB0C0851D9211F4FEA9109444668
:10E2E00008EB890C54F8046BC8EB0C010CF1040C1E
:10E2F0001D46644545F8046BC1F3800112D029B175
:10E3000054F8041B644545F8041B0BD0274657F806
:10E31000041B2E4646F8041B64686C603C1D351DCA
:10E320006445F3D109F1010C4FEA8C0902F00302B4
:10E3300008EB09014B44D2B10D789A18DC4303F87D
:10E34000015B1419934204F0010410D02CB111F8B0
:10E35000014F03F8014B934209D04D781C4604F855
:10E36000015B8D7802315D70631C9342F5D1BDE88D
:10E37000F00370470346DEE70346DDE741462246E9
:10E38000D9E700BFF0B48407034600F08D80541E27
:10E39000002A00F08780E507CEB211D41A4602F8B1
:10E3A000016B13461546920710D0621E002C79D0DF
:10E3B00003F8016B14469A071D4607D0013CEDE7B0
:10E3C000034603F8016B9A071D46F7D1032C52D977
:10E3D000CEB246EA06270F2C47EA07432DD9A4F10F
:10E3E000100217460F2FC2F300162B606B60AB6054
:10E3F000EB6005F1100216D93EB1103F1360536077
:10E400009360D36010320F2F0DD9203F02F1100618
:10E41000136053609360D360136153619361D36160
:10E4200020320F2FF1D8A4F1100222F00F0204F0D5
:10E430000F041032032C15441DD9271F3E462A46CF
:10E44000032E42F8043BC7F380070DD927B1043EE1
:10E45000032E42F8043B07D9174647F8043B083E11
:10E4600053603A1D032EF7D8231F23F00302131D18
:10E4700004F00304ED18ACB1C9B2EA432C1905F855
:10E48000011BA318A54203F001020BD01AB105F835
:10E49000011BA54206D02B4603F8011B69705D1CC9
:10E4A000A542F8D1F0BC7047054614468EE700BF80
:10E4B0002DE9F04F89B014468046019202EB4202EA
:10E4C000A508500004F0030418F0030F02919946C8
:10E4D00003950694079040F0D6800699002940F0F5
:10E4E0005A82019A151F18BF01250095029D062D1D
:10E4F00040F2CF80DDF808C0019F64464FEA5C0619
:10E50000072C07FB068A40F0E281DDF81CC008EB0F
:10E510000C06009B002B40F0FB81D8F80010DAF8C5
:10E520000030C8F80030CAF800100198DDF804A0E7
:10E5300008EB00054946002205952F460495344610
:10E54000CAF1000A91460D46A74240F213812B46BC
:10E550004D469946002D00F0C183DDF810B00299B8
:10E56000CBEB070AC8EB0B025245A8BF5246DDF8B9
:10E5700004C0002A0CFB018B3ADD009BB91A022B68
:10E58000404640F0D28210F8015B91F800C002953D
:10E5900000F801CCDDF808C00B468A18CD4303F81B
:10E5A00001CBAD180130934205F0010520D04DB1EB
:10E5B00010F8015C497800F8011C03F8015B013098
:10E5C000934215D0014611F8015C93F800C018463B
:10E5D00001F801CC00F8015B11F8015B93F801C070
:10E5E000034601F801CC03F8015B01319342EAD103
:10E5F0000199C6EB0B03341B581AA04228BF2046D2
:10E6000000282FDD009DC0EB0B02022D40F053824D
:10E610001578FB433978381807F8015B874203EB1C
:10E620000005134603F8011B05F001011AD039B1AA
:10E6300055783A7807F8015B874203F8012B11D02F
:10E640003D781E781A46394601F8016B02F8015BE5
:10E650005B787D780F4607F8013B8742134603F845
:10E66000015BEDD1019D5545C0F08C81DDF804C002
:10E67000A4457CD2C4EB0B0818F0030FB4FBFCF4E8
:10E6800002943FF42AAF029D0223062D00933FF629
:10E6900031AFDDF804C00CFB058A08EB0C015145D5
:10E6A00065D2019CDDF804B065420434009E0294FA
:10E6B0000091CDF810A04F46DDF80090C14509D873
:10E6C0004DE0D9F800002168C9F8001020604445E9
:10E6D000A14644D909EB050420464946B84700281D
:10E6E0003DDD002EEDD0012E00F0A7831BF804E0E5
:10E6F00094F800900BF1FF310BEB04000246234627
:10E7000001F0010C002902F8019B03F801EBDEDDAA
:10E71000BCF1000F09D0407894F801E001390029DC
:10E7200002F801EB03F8010BD1DD93F800A092F899
:10E730000090944618460CF801AB00F8019B92F843
:10E7400001E093F801A0023962460346002902F86D
:10E7500001AB03F801EBE8DC4445A146BAD8DDF88B
:10E7600000C0049BDC449C45CDF800C0A4D309B094
:10E77000BDE8F08F38464146A84700280BDC8CE006
:10E78000206832682260306056444FF001095444DA
:10E79000A7423FF6DCAE20464146A8470028C0F21B
:10E7A0009A83F4D1009B002BEAD00099012935D03F
:10E7B000DDF804E0207896F800C00EF1FF31224623
:10E7C000334601F00109002902F801CB03F8010BDF
:10E7D000DADDB9F1000F09D0107893F800C00139E3
:10E7E000002902F801CB03F8010BCDDD93F800B04E
:10E7F00092F800E0944618460CF801BB00F801EBD3
:10E8000092F8019093F801B002396246034600295C
:10E8100002F801BB03F8019BE8DCB5E7214633466B
:10E82000DDF80CE053F8042B51F8040B0EF1FF3C1B
:10E8300041F8042C0CF0010243F8040C04310433B9
:10E84000BCF1000FA0DD72B151F8040C53F8042C98
:10E850000CF1FF3C41F8042C43F8040C0431043360
:10E86000BCF1000F90DD53F8042C51F8049C0846CD
:10E8700041F8042C1A4643F8049C50F8043B52F823
:10E88000041BACF1020C40F8041C011D42F8043CCE
:10E89000131DBCF1000FE6DC76E714D1009A002AC4
:10E8A0007CD104983B680268DDF810C0CCF80030D9
:10E8B0003A60DDF810E0DDF804900EEB090CCDF8BD
:10E8C00010C04FF00109DDF804E077443CE60298FF
:10E8D0000199431E282801FB038600F2AB803446D1
:10E8E000454651462846C847002821465046C0F2B2
:10E8F0009580C84700283FF70CAE28462146C847F8
:10E90000009B34EA200A28BFAA46002B3FF405AE3C
:10E9100000994246012900F04781DDF804C012F851
:10E92000015B9AF800400CF1FF3102F8014C5746A8
:10E9300001F001000132002907F8015B7FF7F5AD16
:10E9400058B13D7812F8013C013902F8015C0132FE
:10E95000002907F8013B7FF7E8AD12F8014C3B783E
:10E96000384602F8013C00F8014B12F8014B7D7863
:10E97000023902F8015C07460132002907F8014B11
:10E98000EBDCD2E5019D4046BAFBF5F12A464B4649
:10E99000FFF78EFD6AE602240094A7E5009801289F
:10E9A00000F03B81DDF810E0DDF804B039789EF826
:10E9B00000000BF1FF3B724602F8011B3B460BF0D7
:10E9C0000101BBF1000F03F8010B7FF772AF59B1E2
:10E9D000117818780BF1FF3BBBF1000F02F8010B27
:10E9E00003F8011B7FF765AF92F800C093F8009021
:10E9F0001046194600F8019B01F801CB92F801E09E
:10EA000093F801C0ABF1020B02460B46BBF1000FBD
:10EA100002F801CB03F801EBE6DC4AE7C84700281F
:10EA2000FFF677AD28462146C84735EA200A28BFB9
:10EA3000A2466EE5019AC40802FB04F408EB040543
:10EA40004FEA440B29464046CDF810B0C84708EBC2
:10EA50000B07002839462846C0F23481C8470028F1
:10EA600040F33182C4F1000B0AEB0B0751463846E4
:10EA7000C8475444002821465046C0F21781C84771
:10EA8000002840F31882049806EB0B04371A21463D
:10EA90003846C847002831462046C0F2FB80C847A8
:10EAA00000283FF71EAF38463146C84736EA2004F3
:10EAB00028BF3C4615E73946134653F8042B51F856
:10EAC000045B8008013841F8042C00F0010243F88F
:10EAD000045C0431043300287FF7C4AD6AB151F8F7
:10EAE000045C53F8042C013841F8042C43F8045C0E
:10EAF0000431043300287FF7B5AD51F8046C53F8A6
:10EB0000042C0D4641F8042C43F8046C1A4652F8C4
:10EB1000041B55F8046B023845F8041C131D291D0D
:10EB2000002842F8046CE8DC9CE50B4653F8045BD3
:10EB300050F8041B920802F1FF3C40F8045C021DEF
:10EB40000CF0010543F8041C0433BCF1000F7FF7FF
:10EB50004FAD7DB152F8041C53F8040C0CF1FF3C8E
:10EB600042F8040C43F8041C04320433BCF1000FD7
:10EB70007FF73EAD52F8045C53F8040C114642F89E
:10EB8000040C43F8045C184650F8042B51F8045B5D
:10EB9000ACF1020C41F8042C031D0A1DBCF1000F5E
:10EBA00040F8045CE6DC23E55746039952F8043B41
:10EBB00057F8040B013942F8040C01F0010447F83E
:10EBC000043C04323B1D00297FF7AFAC6CB152F816
:10EBD000045C53F8047C013942F8047C43F8045C7B
:10EBE0000432043300297FF7A0AC52F8045C53F8D8
:10EBF000040C144642F8040C1F4643F8045C57F812
:10EC0000042B54F8045B023944F8042C3B1D221DEC
:10EC1000002947F8045CE8DC87E404993B46DDF80A
:10EC20000C9053F8042B51F804EB09F1FF3041F834
:10EC3000042C00F0010243F804EC043104330028F2
:10EC40007FF737AE6AB151F804CC53F8042C013881
:10EC500041F8042C43F804CC0431043300287FF736
:10EC600028AE53F8042C51F804EC894641F8042CE2
:10EC70001A4643F804EC59F8043B52F8041B0238D6
:10EC800049F8041C42F8043C131D002809F1040152
:10EC9000E7DC0EE6C8470028FFF623AE38463146CB
:10ECA000C84737EA200428BF34461AE6C847002878
:10ECB000FFF6E9AE38462146C84737EA200A28BFA2
:10ECC000A246E0E6C8470028FFF6CCAE40463946EB
:10ECD000C84738EA200528BF3D46C3E60298019C94
:10ECE000059D04FB008A5545BFF441AD019FDDF849
:10ECF00014B03C1D009ECDF800B0DDF804B07D429C
:10ED00000494CDF808A01F46DDF80090C84509D34B
:10ED10004CE0D9F800002168C9F800102060444593
:10ED2000A14643D909EB050420464946B8470028C7
:10ED30003CDD002EEDD0012E41D01BF804E094F80C
:10ED400000900BF1FF310BEB04000246234601F06B
:10ED5000010C002902F8019B03F801EBDFDDBCF197
:10ED6000000F09D0407894F801E00139002902F839
:10ED700001EB03F8010BD2DD93F800A092F80090AC
:10ED8000944618460CF801AB00F8019B92F801E09C
:10ED900093F801A0023962460346002902F801AB4C
:10EDA00003F801EBE8DC4445A146BBD8DDF800C020
:10EDB000029BDC449C45CDF800C0A5D3D7E4DDF828
:10EDC0001090234609EB0402DDF80CE053F8041B15
:10EDD00052F804CC0EF1FF3042F8041C00F001019F
:10EDE00043F804CC04320433002898DD61B152F8B2
:10EDF000049C53F8041C013842F8041C43F8049C9A
:10EE00000432043300288ADD53F8041C52F804EC61
:10EE1000944642F8041C194643F804EC5CF8043BA1
:10EE200051F8042B02384CF8042C41F8043C0B1D1B
:10EE300000280CF10402E7DC71E7029A234612195C
:10EE4000DDF80C9053F8041B52F804CC09F1FF30A4
:10EE500042F8041C00F0010143F804CC04320433EE
:10EE600000287FF734AC69B152F804EC53F8041C65
:10EE7000013842F8041C43F804EC0432043300283F
:10EE80007FF725AC53F8041C52F8049C944642F8D2
:10EE9000041C194643F8049C5CF8043B51F8042B0D
:10EEA00002384CF8042C41F8043C0B1D00280CF1EE
:10EEB0000402E7DC0BE438462146C84734EA200A5E
:10EEC00028BFBA46DFE540463946C84737EA20053D
:10EED00028BF4546C6E5A7423FF639AB009B63B95C
:10EEE000386822683A602060DDF804E04FF00109DC
:10EEF0007744CEEB0404FFF727BB0098012833D0FA
:10EF0000DDF80490207897F800E009F1FF313A46E7
:10EF100002F8010B234601F00100002903F801EB80
:10EF2000E2DD48B1107893F800C00139002902F8F9
:10EF300001CB03F8010BD7DD93F800B092F800E0A5
:10EF4000944618460CF801BB00F801EB92F80190CA
:10EF500093F801B0023962460346002902F801BB6A
:10EF600003F8019BE8DCBFE739462346DDF80CE0F7
:10EF700053F8042B51F8040B0EF1FF3C41F8042C1C
:10EF80000CF0010243F8040C04310433BCF1000F0F
:10EF9000AADD72B151F8040C53F8042C0CF1FF3CBB
:10EFA00041F8042C43F8040C04310433BCF1000F85
:10EFB0009ADD53F8042C51F8049C084641F8042CBF
:10EFC0001A4643F8049C50F8043B52F8041BACF179
:10EFD000020C40F8041C011D42F8043C131DBCF156
:10EFE000000FE6DC80E700BF830770B5064614D14A
:10EFF0000368A3F1013222EA030010F0803F0CD134
:10F00000331D1A4653F8044BA4F1013525EA0404D4
:10F0100014F0803FF5D0104600E0304603782BB165
:10F02000421C147810460132002CFAD100F080F80E
:10F03000304670BDC9B2F0B400294BD082070FD062
:10F040000278002A71D0914242D0431C05E013F8A7
:10F05000012B002A3BD091423AD09A071846F6D1AC
:10F06000036841EA0127A3F1013222EA030212F008
:10F07000803F47EA07471CD17B40A3F1013222EAD7
:10F08000030313F0803F14D1021D02E014F0803F0F
:10F090000FD1104652F8043BA3F1013687EA03046E
:10F0A00026EA0303A4F1013513F0803F25EA0404A6
:10F0B000ECD00278002A38D0914209D0431C01E0FC
:10F0C000914205D0184613F8012B002AF8D11046BA
:10F0D000F0BC704783070BD00278002AF8D0431C9D
:10F0E00003E0017801330029F2D099071846F8D1DE
:10F0F0000168A1F1013323EA010212F0803F0AD135
:10F10000031D184653F8041BA1F1013424EA01023F
:10F1100012F0803FF5D00378002BD9D0421C117833
:10F12000104601320029FAD1D2E71046D0E700BFDD
:10F1300080EA0102844612F0030F4FD111F0030F51
:10F1400032D14DF8044D11F0040F51F8043B0BD0AF
:10F15000A3F101329A4312F0803F04BF4CF8043B04
:10F1600051F8043B16D100BF51F8044BA3F1013212
:10F170009A4312F0803FA4F101320BD14CF8043BCA
:10F18000A24312F0803F04BF51F8043B4CF8044BFB
:10F19000EAD023460CF8013B13F0FF0F4FEA33236C
:10F1A000F8D15DF8044B704711F0010F06D011F84B
:10F1B000012B0CF8012B002A08BF704711F0020F39
:10F1C000BFD031F8022B12F0FF0F16BF2CF8022B24
:10F1D0008CF8002012F47F4FB3D1704711F8012B47
:10F1E0000CF8012B002AF9D1704700BF20F0030171
:10F1F00010F00300C0F1000051F8043B00F1040CD2
:10F200004FEACC0C6FF000021CBF22FA0CF2134341
:10F210004FF0010C4CEA0C2C4CEA0C4CA3EB0C020A
:10F2200022EA030212EACC1204BF51F8043B043074
:10F23000F4D013F0FF0F1FBF013013F47F4F0130E4
:10F2400013F47F0F18BF0130704700BFF0B4002ADD
:10F2500063D0344B04461B6814F8010B571E1D186D
:10F260006E7807F0010706F00305012D58D011F85C
:10F27000015B5E19767806F00306012E08BF203583
:10F28000401B4BD1002D49D0013A47D02FB314F881
:10F29000010B1D186E7806F00305012D11F8015BB6
:10F2A00008BF20305E19767806F00306012E08BFED
:10F2B0002035401B32D18DB3013A0ED12EE011F82A
:10F2C000012B9E18767806F00306012E08BF203227
:10F2D000801A23D112B36A1E20D014F8010B1D1816
:10F2E0006E7806F00305012D11F8015B08BF203090
:10F2F0005E19767806F00306012E08BF2035401B04
:10F300000CD15DB114F8010B551E1A18567806F091
:10F310000302012AD3D12030D1E71046F0BC704758
:10F320002030A4E7A401002041EA00039B07F0B4C9
:10F3300074D1032A72D90C4654F8045B161FA5F148
:10F34000013727EA050717F0803F0346C6F3800C14
:10F3500031D10346032E324643F8045B2AD9BCF16F
:10F36000000F0AD0214654F8045BA5F1013626EAC5
:10F37000050616F0803F18D01DE0264656F8045BBF
:10F380002146A5F1013727EA050717F0803F12D182
:10F3900043F8045B65683146A5F1013626EA0506A7
:10F3A000043A0C1D16F0803F05D1043A032A43F8B5
:10F3B000045BE2D821467AB30D78013A03F8015B89
:10F3C0009DB112F0010F1C462AD1234622B311F839
:10F3D000015F013A03F8015B3DB111F8015F013AA9
:10F3E00065705C1C2346002DEFD1AAB100219C184A
:10F3F000DA4303F8011BA218A34202F001020BD06A
:10F400001AB103F8011BA34206D01A4602F8011BE9
:10F410005970531CA342F8D1F0BC70470346CAE7A9
:10F4200011F8015F1C4604F8015B013A2346002DE8
:10F43000CBD1DAE72DE9F00701273C4600254FF054
:10F44000FF3663198B4200EB060C0DD21CF804A0AA
:10F4500010F80380D0452ED201241D469F1B63194E
:10F460008B4200EB060CF1D34FF0010A17605446B3
:10F4700000254FF0FF3C6319994200EB0C080ED9B0
:10F4800018F8048010F80390C1451AD901241D46CC
:10F49000CCEB030A6319994200EB0C08F0D80CF18D
:10F4A00001000136B0423CBFBA463046C2F800A067
:10F4B000BDE8F00770470BD001272E463C46ED19FA
:10F4C000BFE709D04FF0010AAC4654465544D2E795
:10F4D000BC4205D00134B4E7544505D00134CAE735
:10F4E00027461D460124ACE7A2461D460124C2E77B
:10F4F0002DE9F04FADF2244D1546064689461046DB
:10F50000194607AA1C46FFF795FF07AB82460DF286
:10F510001C411A1D5C6008338B425460F9D114B34E
:10F5200001232F78611E08A8A34240F8271001EAA2
:10F53000030218D032B16A7802234F1EA34240F86A
:10F54000227010D0B046A4465C1C15F803E0CE1A19
:10F550002A5D02330F1B634540F82E6040F822708D
:10F56000F2D146466446079928466918524600F08B
:10F5700045FC002840F0B6800AF1FF3E05EB0E0C7A
:10F58000CDF808E0CAF1010E834604F1FF38CDF84A
:10F590000CC0CDF814E00746CDF810A04A460095FF
:10F5A000019408E027B1079FBB4201D20199CB1B10
:10F5B0009B4400272246019CB0185C440021A21AFB
:10F5C00000F07CFB002840F08780002C00F0848055
:10F5D000301910F8013C08A951F82330002BE1D173
:10F5E000049B9F4228BF3B46434527D2DDF800904D
:10F5F00006EB0B0119F80350CA5C09EB03009542B6
:10F6000066D1DD43454415F0010F024613D00133A6
:10F61000434513D24078CD5C013285420BD057E090
:10F6200012F8010FCD5C854252D1013312F8010F5F
:10F63000CD5C85424CD101334345F1D3DDF81090C8
:10F64000029B4F4528BF4B4639D2DDF808C0DDF894
:10F65000009006EB0B0519F80C1015F80C00814210
:10F6600040F0C080DDF80CE009EB070ACAEB0E01A0
:10F67000C80772461ED5DDF8089009F1FF31DDF8A4
:10F680000C90685C19F801CC09F1FF32844516D161
:10F690000B460FE012F8019C15F800E04A1EF145F8
:10F6A0000DD10346013815F800C011F8011C614561
:10F6B00005D10346581E524502F1FF31EAD1013708
:10F6C0009F4200F29180079F019ABB44D71B71E7CC
:10F6D000DDF814E0F3446BE7002009B00DF5806D10
:10F6E000BDE8F08FCAEB0400504538BF5046CAF160
:10F6F0000102431C0AF1FF3C05EB0A0704F1FF3B42
:10F70000019200944A460793B1464FF000086446C0
:10F710003E46009909EB020008EB0107BA1A0021E6
:10F7200000F0CCFA0028D7D1002FD5D009EB070084
:10F7300010F8013C08AA52F8230000284AD1DA4503
:10F7400009EB08002AD210F80A303178994218BF24
:10F75000534642D16FEA0A0303EB0B01C907324655
:10F76000534618D50AF101035B4517D2324612F809
:10F77000011F10F803E08E450DD02EE012F8011F96
:10F7800010F803C08C4528D1013312F8011F10F87E
:10F7900003E08E4521D101335B45EFD3621C234644
:10F7A0009BD0295D025D914213D1E10709D5631E0B
:10F7B000E95CC25C914204D00BE0E95CC25C91421E
:10F7C00007D15A1E002B88D0A95C825C023B914273
:10F7D000F3D0079880443A469BE7DDF804C0E04444
:10F7E0009844F8E7049B6AE706EB0B0075E700BF57
:10F7F0002DE9F04F037889B080460D46002B00F0CC
:10F8000065810A789AB184460131012602E011F837
:10F81000012B5AB1934214BF002606F001061CF8D2
:10F82000013F0C46002BF2D1207820B936B140467A
:10F8300009B0BDE8F08F4FF00008F8E708F10100CB
:10F840002978FFF7F7FB641B06460028F3D0012C4C
:10F8500000F0B580A044404594BFC0EB08070127E5
:10F860001F2C06D939462A462346FFF741FE80461B
:10F87000DDE7214607AA2846FFF7DCFD079903903C
:10F8800069182846039A00F0B9FA002840F09980D8
:10F89000DDF80CC0DDF80C900CF1FF3E05EB0E011D
:10F8A000C9F1010C8346CDF808E080460491CDF8FB
:10F8B00014C03A46B146019508EB040609EB020074
:10F8C0000021B21A00F0FAF90028B4D1002EB2D00B
:10F8D000039B9B4528BF5B469C4227D9019D09EBB2
:10F8E000030010F80820E95CE81891425FD1DD437D
:10F8F0002D1915F0010F024609EB080113D0013351
:10F900009C4213D94078CD5C013285420BD04EE049
:10F9100012F8010FCD5C854249D1013312F8010F75
:10F92000CD5C854243D101339C42F1D8DDF80CE037
:10F93000029ADE4540F2CD80019B09EB0805995CF7
:10F94000A85C814240F0C580DDF804A0049BDA4445
:10F95000CAEB0301C8071AD5029FDDF810C0791E53
:10F96000685C1CF8017C0CF1FF33874214D10A4615
:10F970000DE013F801EC2F5C4B1EBE450CD1024686
:10F9800001382F5C11F8011CB94205D10246501E06
:10F99000534503F1FF31ECD10BF1010B934500F21C
:10F9A0009A80079A9044C2EB040B324684E7059D87
:10F9B00005EB080B0BEB03084FF0000BF5E7804657
:10F9C00035E7DDF80CA00399CAEB0403534538BFB3
:10F9D0005346CAF1010B581C06EB0A0205EB0A0854
:10F9E000CDF808B03B4607904FF00009019201F1B5
:10F9F000FF3B37468A4609EB0406F8180021F21A45
:10FA000000F05CF900287FF416AF002E3FF413AF2E
:10FA1000544598BF07EB09002CD9DDF804E098F8AD
:10FA200000001EF8093098424AD16FEA0A02111903
:10FA3000C9074246534607EB090018D50AF10103EE
:10FA40009C4217D9424612F8011F10F803C08C459A
:10FA50000DD036E012F8011F10F803E08E4530D1CA
:10FA6000013312F8011F10F803C08C4529D101336E
:10FA70009C42EFD8BBF1FF3F5B463FF4F8AE15F870
:10FA80000B1010F80B20914216D11BF0010F0AD079
:10FA90000BF1FF33E95CC25C914204D00CE0E95CFD
:10FAA000C25C914208D15A1E002B3FF4E0AEA95C23
:10FAB000825C023B9142F2D00798814433469AE738
:10FAC0005346DDF808E0F1449944F7E70C46012677
:10FAD000AAE6039A60E74E46C844A8E640F2D0532F
:10FAE000C2F200031A6801235C3200F001B800BFC3
:10FAF000F0B4002825D0074638463E780D46013739
:10FB000015F8014B3CB1A642FAD1002BF4D1176095
:10FB100007F8013C11E0C6B13D4600E01BB915F8FD
:10FB2000016B0C46284614F8013B9E42F6D136B1D3
:10FB3000002105F8011C1060781EF0BC70473046AB
:10FB4000F9E710680028D6D1F7E716603046F4E7E9
:10FB50002DE9F00F494C82B0D4F800C001900F4657
:10FB60003C4614F8015B0CEB05004678274606F08E
:10FB70000800C6B2002EF3D12D2D61D02B2D04BF6D
:10FB8000244614F8015BB346002B41D1302D43D0FD
:10FB90000A239A46BBF1000F0CBF6FF000474FF0ED
:10FBA0000047B7FBFAF90AFB197000900020804665
:10FBB0000CE0303DAB421BDD461C05D0C84539D8B2
:10FBC00035D00AFB0858012014F8015B0CEB050640
:10FBD000767806F00407FFB2002FEAD116F003068C
:10FBE00006D0012E14BF57263726AD1BAB42E3DCEF
:10FBF000431C2AD0BBF1000F01D0C8F10008002A35
:10FC000031D0D0B94046116002B0BDE8F00F704766
:10FC1000102BBED1302DBCD12578782D25D0582D74
:10FC200023D043BB4FF0080A30255346B2E7009873
:10FC30008542C6DD4FF0FF30C6E74046611EE2E771
:10FC400014F8015B4FF0010B9EE7BBF1000F019927
:10FC50000CBF6FF000404FF0004022230B60002AE1
:10FC6000D2D0611ECFE74046CEE74FF0100A65784C
:10FC7000534602348EE79A4630258BE7A4010020D4
:10FC800070B440F2D054C2F2000406460D4620681B
:10FC9000134631462A4670BCFFF75ABF024B13B1D8
:10FCA000024800F005B870470000000045E1000878
:10FCB0000146002002460346FEF7C4B98307F0B4AC
:10FCC000C9B200F09680531E002A00F0948002789A
:10FCD0008A420BD0421CD8071AD512F0030F1046E7
:10FCE0001CD01478013B01328C4211D1F0BC70471A
:10FCF000002B7CD01278013B8A42F7D014F0030F1E
:10FD0000204604F1010209D02478013B8C42EDD059
:10FD100012F0030F104602F10104E9D1032B3FD981
:10FD2000046841EA012545EA054585EA0407A7F18B
:10FD3000013222EA07021E1F041D12F0803FC6F3A3
:10FD400080072DD1032E334629D967B12668204676
:10FD500085EA0602A2F1013626EA0202043412F014
:10FD6000803F19D01CE020462468061D85EA040265
:10FD7000A2F1013424EA020212F0803F10D134686B
:10FD8000043B85EA0402A2F1013424EA0202341D94
:10FD900012F0803F304603D1043B032BE3D82046CA
:10FDA0005D1E23B303788B42A0D0431C0022E807DA
:10FDB00014D51C781846012201338C4296D0954206
:10FDC000184603F1010402F102020ED01B788B42A7
:10FDD0008CD020462478431C8C4287D0954218460C
:10FDE00003F1010402F10202F0D100207EE718467F
:10FDF0007CE7134692E7104678E700BF032AF0B489
:10FE000031D941EA00039C072ED106680F68151FFF
:10FE1000031D0C1DBE42C5F3800C24D1032D2A46C0
:10FE20001FD9BCF1000F08D01E682568214618466E
:10FE300004340433AE4211D015E0214618461C6844
:10FE40000B68051D0E1D9C420DD1314628462E68BB
:10FE50000D68043A031D0C1DAE4204D1043A032A76
:10FE6000EBD8214618461AB303780C78A3420AD17E
:10FE7000551E0022EB0714D510F8013F11F8014F71
:10FE80000122A3420DD0181B10E010F8013F11F819
:10FE9000014FA342F7D110F8013F11F8014FA342DF
:10FEA000F1D1AA4202F10202EFD10020F0BC70476A
:10FEB0001046FBE71E1E6464646464640001010371
:10FEC000080409040A040B040C040D0404040504CA
:10FED00006040704FFFF00010103080409040A05E2
:10FEE0000B050C050D050405050506050705FFFFB7
:10FEF00000FF0008BCFE00081EFF0008D6FE000838
:10FF000000020102020203020402050206020702C5
:10FF1000080409040A040B040C040D04FFFF00028A
:10FF2000010202020302040205020602070208049B
:10FF300009040A050B050C050D05FFFFF722000853
:10FF4000AF220008CB2200087124000871220008AB
:10FF50006D220008E128000829270008452700082D
:10FF600023270008A92600081D27000800000040DC
:10FF70000008014001000000001C002800000040B3
:10FF80000008014002000000041C0028000000409E
:10FF90000008014004000000081C00280000004088
:10FFA00000080140080000000C1C0028000400406C
:10FFB0000008014040000000001D0028000400402F
:10FFC0000008014080000000041D002800040040DB
:10FFD000000C014001000000081D00280004004042
:10FFE000000C0140020000000C1D0028002C014004
:10FFF0000008014000010000001B0128002C014006
:020000040801F1
:1000000000080140000800000C1B01280008004007
:10001000000C014040000000001E002800080040C5
:10002000000C014080000000041E00280008004071
:10003000000C014000010000081E002800080040DC
:10004000000C0140000200000C1E0028002C0140A2
:1000500000000040000400400008004000000400D0
:1000600008000C00D00732003200320032003200AB
:1000700032003200C8006400000041455452313261
:100080003334003031323334353637383941424336
:100090004445464748494A4B4C4D4E4F50515253A8
:1000A0005455565758595A00C53F0008214000087A
:1000B000FD3F000839400008614000087140000819
:1000C000D13F000829410008E53F0008F13F000842
:1000D0000000803FF704353FF70435BF0000803F44
:1000E0000000803FF70435BFF70435BF0000803FB4
:1000F0000000803FF70435BFF704353F0000803F24
:100100000000803FF704353FF704353F0000803F93
:100110000000803F00000000000080BF000080BFA2
:100120000000803F000080BF00000000000080BF92
:100130000000803F000000000000803F000080BF02
:100140000000803F0000803F00000000000080BFF2
:100150000000803F000000000000803F000080BFE2
:100160000000803F000080BF000080BF0000000052
:100170000000803F000000000000803F0000803F42
:100180000000803F0000803F000080BF00000000B2
:100190000000803F000000BFD0B35D3F0000803F03
:1001A0000000803F000000BFD0B35DBF0000803F73
:1001B0000000803F0000003FD0B35D3F000080BFE3
:1001C0000000803F0000003FD0B35DBF000080BF53
:1001D0000000803F000080BF00000000000080BFE2
:1001E0000000803F0000803F000000000000803FD2
:1001F0000000803F000000000000803F0000803FC2
:100200000000803F000080BF000080BF00000000B1
:100210000000803F000000000000803F000080BF21
:100220000000803F0000803F000080BF0000008091
:100230000000803F00000000A8AAAA3F00000000C4
:100240000000803F000080BFB0AA2ABF000000006D
:100250000000803F0000803FB0AA2ABF00000000DD
:100260000000803F0000803F000000000000000010
:100270000000803F000080BF000000000000000080
:100280000000803F0000803F000000BF0000803F72
:100290000000803F000000BF000080BF0000803FE2
:1002A0000000803F000080BF0000003F0000803F52
:1002B0000000803F0000003F0000803F0000803FC2
:1002C0000000803F0000003F000080BF000080BFB2
:1002D0000000803F000080BF000000BF000080BF22
:1002E0000000803F000000BF0000803F000080BF92
:1002F0000000803F0000803F0000003F000080BF02
:100300000000803F0000000000000000000080BFEF
:100310000000803F00000000000000000000803F5F
:10032000000000000000000003010000300201088E
:10033000040000005805010804000000B80401088A
:10034000020100006002010800010000000000003E
:10035000060000009805010806000000F8040108E6
:10036000010100000000000004000000500101082D
:100370000600000090010108080000003804010890
:1003800008000000D00001080800000080020108F9
:10039000010100000000000000010000000000005A
:1003A000000100000000000004000000F00101084E
:1003B00006000000D8030108000100000000000052
:1003C000020100000003010801010000000000001C
:1003D00000000000000000000000803F000080BF1F
:1003E0000000803F000080BF0000803F000080BF11
:1003F000000080BF0000803F0000803F0000803F81
:100400000000803F0000803F0000803F0000803FF0
:10041000000080BF000080BF0000803F000000009F
:1004200000000000000000000000803F000000000D
:1004300000000000000000000000803F000080BFBE
:100440000000803F000080BF0000803F000080BFB0
:10045000000080BF0000803F0000803F0000803F20
:100460000000803F0000803F0000803F0000803F90
:10047000000080BF000080BF0000803F000080BF00
:100480000000803F0000803F0000803F000080BFF0
:10049000000080BF000080BF0000803F0000803F60
:1004A0000000803F000080BF0000803F0000803FD0
:1004B000000080BF0000803F0000803F000080BF40
:1004C0000000803F000080BF0000803F000080BF30
:1004D000000080BF0000803F0000803F0000803FA0
:1004E0000000803F0000803F0000803F0000803F10
:1004F000000080BF000080BF0000803FD0B35DBF20
:100500000000003F0000803F0000803FD0B35DBF8F
:10051000000000BF000080BF0000803FD0B35D3FFF
:100520000000003F0000803F0000803FD0B35D3FEF
:10053000000000BF000080BF0000803F00000000FE
:10054000000080BF0000803F0000803F00000000EE
:100550000000803F000080BF0000803F00000000DE
:100560000000803F000080BF0000803F000080BF8F
:10057000000000000000803F0000803F0000803F3E
:10058000000000000000803F0000803F00000000ED
:10059000000080BF000080BF0000803F000000001E
:1005A000A8AAAA3F0000803F0000803F000080BF53
:1005B000B0AA2ABF000080BF0000803F0000803F3B
:1005C000B0AA2ABF000080BF0000803F00000000EA
:1005D000A8AAAA3F000080BF0000803F000080BFA3
:1005E000B0AA2ABF0000803F0000803F0000803F8B
:1005F000B0AA2ABF0000803F24505542582C343105
:100600002C312C303030332C303030312C313135EE
:100610003230302C302A31450D0A0024504D544BD5
:100620003235312C3131353230302A31460D0A0025
:1006300024505542582C34312C312C303030332C4E
:10064000303030312C35373630302C302A32440DB2
:100650000A0024504D544B3235312C35373630306A
:100660002A32430D0A0024505542582C34312C3183
:100670002C303030332C303030312C333834303073
:100680002C302A32360D0A0024504D544B3235316D
:100690002C33383430302A32370D0A00245055427A
:1006A000582C34312C312C303030332C3030303128
:1006B0002C31393230302C302A32330D0A0024509C
:1006C0004D544B3235312C31393230302A32320DE3
:1006D0000A00B56206010300F00500FF19B56206C5
:1006E000010300F00300FD15B56206010300F001EF
:1006F00000FB11B56206010300F00000FA0FB562BD
:1007000006010300F00200FC13B56206010300F0CD
:100710000400FE17B562060103000102010E47B591
:1007200062060103000103010F49B56206010300DF
:10073000010601124FB562060103000112011E6796
:10074000B56206160800030703000000000031E54B
:10075000B56206080600C80001000100DE6A00005C
:100760000000000000C20100F80501081B06010896
:100770000100000000E100003006010852060108F7
:1007800002000000009600006606010888060108C5
:1007900003000000004B00009C060108BE06010893
:1007A00004000000802500005B0F01085B0F0108BA
:1007B00041455254313233340000271008042302DB
:1007C00020010000000000008025000000C20100A0
:1007D00002000000010000008025000000C20100AE
:1007E000030000000200000080250000004B000014
:1007F000050000000300000080250000004B000001
:1008000005000000020000008025000000C2010079
:1008100000000000100000008025000000C2010060
:1008200001000000200000008025000000C201003F
:1008300000000000010000008025000000C201004F
:1008400000000000080000008025000000C2010038
:10085000000300000400000080250000004B0000A1
:1008600000000000061801080D1801081218010800
:10087000231801082D180108381801084318010829
:100880004E18010818170108571801081217010817
:10089000601801086A180108751801087B1801081A
:1008A0007E1801088E180108951801080000000044
:1008B000581701085C17010862170108681701083A
:1008C0006B17010872170108751701087A170108DC
:1008D00086170108891701088F1701089617010864
:1008E000A0170108AA170108B3170108C1170108CA
:1008F000CD170108D4170108DA170108E717010816
:10090000F2170108FF170108000000006215010836
:1009100066150108A19E00088D15010892150108B1
:100920006D990008A6150108AF1501085599000832
:10093000CC150108D1150108059F00080016010813
:100940005B0F01081D990008051601080D16010826
:100950003198000821160108301601081198000886
:100960004A1601085B0F0108619500084F1601083F
:100970005316010869970008A01501086F160108B1
:10098000B99B00088216010888160108F99D000825
:10099000A3160108AB160108AD9D0008BA160108A0
:1009A000BF160108419700083B0C0108CF1601084B
:1009B000599C0008FD160108F11601088D950008E4
:1009C0004F1101085B0F0108559500085B0F0108E6
:1009D000241701082C170108341701083C170108D7
:1009E000431701084E1701085317010800000000C3
:1009F0004166726F333220434C49207665727369C9
:100A00006F6E20322E32204D617920323420323008
:100A10003134202F2030303A30373A3538202D20ED
:100A200028636C65616E666C69676874290041763D
:100A300061696C61626C6520636F6D6D616E64737A
:100A40003A0D0A0025730925730D0A005379737452
:100A5000656D20557074696D653A20256420736555
:100A6000636F6E64732C20566F6C746167653A20F7
:100A70002564202A20302E315620282564532062F8
:100A8000617474657279290D0A00435055202564FC
:100A90004D487A2C206465746563746564207365C1
:100AA0006E736F72733A20002573200041434348F0
:100AB000573A202573002E2563004379636C652027
:100AC00054696D653A2025642C20493243204572D3
:100AD000726F72733A2025642C20636F6E666967AB
:100AE0002073697A653A2025640D0A002025642068
:100AF0002564000D0A5265626F6F74696E672E2E51
:100B00002E00536176696E672E2E2E004D7573741C
:100B100020626520616E79206F72646572206F6655
:100B20002041455452313233340D0A0043757272FC
:100B3000656E742061737369676E6D656E743A20BB
:100B4000004572726F723A20456E61626C65206179
:100B50006E6420706C756720696E20475053206664
:100B6000697273740D0A00456E61626C656420667B
:100B7000656174757265733A2000417661696C61D4
:100B8000626C652066656174757265733A20004910
:100B90006E76616C69642066656174757265206E3D
:100BA000616D652E2E2E0D0A0044697361626C65BD
:100BB000642000456E61626C656420000D0A4C651E
:100BC0006176696E6720434C49206D6F64652E2EF7
:100BD0002E0D0A00526573657474696E6720746F18
:100BE0002064656661756C74732E2E2E004E470965
:100BF000004F4B0900437573746F6D206D69786504
:100C0000723A200D0A4D6F746F720954687209525E
:100C10006F6C6C095069746368095961770D0A003B
:100C20002325643A09002573090053616E697479BC
:100C300020636865636B3A09007265736574006CC4
:100C40006F616400496E76616C6964206D697865D6
:100C50007220747970652E2E2E0D0A004C6F61641F
:100C60006564202573206D69782E2E2E0D0A00579D
:100C7000726F6E67206E756D626572206F6620619F
:100C80007267756D656E74732C206E656564732074
:100C90006964782074687220726F6C6C207069745B
:100CA0006368207961770D0A004D6F746F72206E52
:100CB000756D626572206D75737420626520626562
:100CC000747765656E203120616E642025640D0A9D
:100CD0000043757272656E74206D697865723A2092
:100CE00025730D0A00417661696C61626C65206D47
:100CF00069786572733A20004D6978657220736572
:100D00007420746F2025730D0A0043757272656E2E
:100D1000742073657474696E67733A200D0A002538
:100D2000732073657420746F20004552523A205628
:100D3000616C75652061737369676E6D656E742093
:100D40006F7574206F662072616E67650D0A0045CD
:100D500052523A20556E6B6E6F776E2076617269D3
:100D600061626C65206E616D650D0A00437572727B
:100D7000656E742070726F66696C653A2025640D2B
:100D80000A0055736167653A0D0A6D6F746F7220C2
:100D9000696E646578205B76616C75655D202D20D9
:100DA00073686F77205B6F72207365745D206D6F61
:100DB000746F722076616C75650D0A004E6F20733A
:100DC000756368206D6F746F722C20757365206178
:100DD000206E756D626572205B302C2025645D0D80
:100DE0000A004D6F746F722025642069732073654B
:100DF000742061742025640D0A00496E76616C6967
:100E000064206D6F746F722076616C75652C203173
:100E10003030302E2E323030300D0A00536574746D
:100E2000696E67206D6F746F7220256420746F2067
:100E300025640D0A006175782025752025750D0A39
:100E400000496E76616C69642046656174757265EF
:100E500020696E6465783A206D7573742062652030
:100E60003C2025750D0A0043757272656E7420432F
:100E70006F6E6669673A20436F7079206576657298
:100E8000797468696E672062656C6F772068657237
:100E9000652E2E2E0D0A006D697865722025730D62
:100EA0000A00636D697820256400636D69782025E8
:100EB0006420302030203020300D0A0066656174D7
:100EC000757265202D25730D0A0066656174757253
:100ED000652025730D0A006D61702025730D0A00D1
:100EE000736574202573203D20000D0A456E7465DE
:100EF00072696E6720434C49204D6F64652C2074E5
:100F00007970652027657869742720746F20726571
:100F10007475726E2C206F72202768656C70270DB7
:100F20000A000D0A2320000D1B5B4B001B5B324A9D
:100F30001B5B313B3148004552523A20556E6B6E77
:100F40006F776E20636F6D6D616E642C20747279A3
:100F5000202768656C702700082008006C6F6F7090
:100F600074696D6500656D665F61766F6964616E59
:100F70006365006D69647263006D696E63686563C3
:100F80006B006D6178636865636B00727373695F92
:100F90006368616E6E656C00727373695F70776D04
:100FA0005F70726F7669646572006D696E746872E5
:100FB0006F74746C65006D61787468726F74746CB2
:100FC00065006D696E636F6D6D616E64006465616F
:100FD0006462616E6433645F6C6F77006465616442
:100FE00062616E6433645F68696768006E6575741A
:100FF00072616C3364006465616462616E64336461
:101000005F7468726F74746C65006D6F746F725F7B
:1010100070776D5F7261746500736572766F5F7073
:10102000776D5F7261746500726574617264656486
:101030005F61726D00666C6170735F73706565648B
:1010400000666978656477696E675F616C74686F64
:101050006C645F6469720073657269616C5F706F64
:1010600072745F315F7363656E6172696F0073657F
:101070007269616C5F706F72745F325F7363656E0B
:101080006172696F0073657269616C5F706F727411
:101090005F335F7363656E6172696F007365726958
:1010A000616C5F706F72745F345F7363656E6172E1
:1010B000696F007265626F6F745F6368617261630C
:1010C000746572006D73705F6261756472617465DE
:1010D00000636C695F62617564726174650067705A
:1010E000735F6261756472617465006770735F70CD
:1010F0006173737468726F7567685F62617564723B
:10110000617465006770735F70726F766964657291
:101110000073657269616C72785F70726F76696472
:1011200065720074656C656D657472795F70726F5D
:1011300076696465720074656C656D657472795F5B
:10114000737769746368006672736B795F696E7632
:10115000657273696F6E00766261747363616C654A
:1011600000766261746D617863656C6C766F6C7427
:1011700061676500766261746D696E63656C6C763B
:101180006F6C7461676500706F7765725F6164632F
:101190005F6368616E6E656C00616C69676E5F6746
:1011A00079726F00616C69676E5F61636300616C87
:1011B00069676E5F6D616700616C69676E5F626F22
:1011C0006172645F726F6C6C00616C69676E5F6204
:1011D0006F6172645F706974636800616C69676EE7
:1011E0005F626F6172645F796177006D61785F61E2
:1011F0006E676C655F696E636C696E6174696F6E52
:10120000006779726F5F6C7066006D6F726F6E5FF2
:101210007468726573686F6C64006779726F5F637E
:101220006D70665F666163746F72006779726F5F7D
:10123000636D70666D5F666163746F7200616C747C
:101240005F686F6C645F7468726F74746C655F6EF6
:1012500065757472616C00616C745F686F6C645F5B
:10126000666173745F6368616E6765007468726F4E
:1012700074746C655F636F7272656374696F6E5FBF
:1012800076616C7565007468726F74746C655F6309
:101290006F7272656374696F6E5F616E676C650013
:1012A0007961776465616462616E64007961775F1A
:1012B000636F6E74726F6C5F646972656374696F7B
:1012C0006E007961775F646972656374696F6E003F
:1012D0007472695F756E61726D65645F7365727655
:1012E0006F0072635F726174650072635F6578702E
:1012F0006F007468725F6D6964007468725F65780E
:10130000706F00726F6C6C5F70697463685F72619C
:101310007465007961775F72617465007470615FF4
:1013200072617465007470615F627265616B706F89
:10133000696E74006661696C736166655F64656C93
:101340006179006661696C736166655F6F66665F8F
:1013500064656C6179006661696C736166655F7470
:1013600068726F74746C65006661696C7361666540
:101370005F6D696E5F75736563006661696C73614B
:1013800066655F6D61785F757365630067696D623F
:10139000616C5F666C616773006163635F68617253
:1013A0006477617265006163635F6C70665F66613C
:1013B00063746F720061636378795F64656164620E
:1013C000616E64006163637A5F6465616462616E2B
:1013D00064006163635F756E61726D656463616C07
:1013E000006163635F7472696D5F70697463680044
:1013F0006163635F7472696D5F726F6C6C006261D0
:10140000726F5F7461625F73697A65006261726FA7
:101410005F6E6F6973655F6C7066006261726F5FAB
:1014200063665F76656C006261726F5F63665F61C1
:101430006C74006D61675F6465636C696E6174698B
:101440006F6E006770735F706F735F7000677073AB
:101450005F706F735F69006770735F706F735F6455
:10146000006770735F706F73725F70006770735F97
:10147000706F73725F69006770735F706F73725F14
:1014800064006770735F6E61765F70006770735F92
:101490006E61765F69006770735F6E61765F64008E
:1014A0006770735F77705F726164697573006E61F6
:1014B000765F636F6E74726F6C735F686561646989
:1014C0006E67006E61765F73706565645F6D696EEF
:1014D000006E61765F73706565645F6D6178006E44
:1014E00061765F736C65775F7261746500706964C3
:1014F0005F636F6E74726F6C6C657200705F7069A1
:1015000074636800695F706974636800705F726F0C
:101510006C6C00695F726F6C6C00705F7961770052
:10152000695F79617700705F616C7400695F616CFD
:101530007400645F616C7400705F6C6576656C004C
:10154000695F6C6576656C00645F6C6576656C00E0
:10155000705F76656C00695F76656C00645F7665C8
:101560006C0061757800666561747572655F6E61A7
:101570006D6520617578666C6167206F7220626CA2
:10158000616E6B20666F72206C69737400636D69A5
:10159000780064657369676E20637573746F6D207E
:1015A0006D697865720064656661756C747300724C
:1015B0006573657420746F2064656661756C7473FF
:1015C00020616E64207265626F6F740064756D7067
:1015D000007072696E7420636F6E66696775726100
:1015E000626C652073657474696E677320696E2020
:1015F00061207061737461626C6520666F726D004A
:10160000657869740066656174757265006C6973EC
:1016100074206F72202D76616C206F722076616C61
:1016200000677073706173737468726F75676800B8
:10163000706173737468726F756768206770732068
:10164000746F2073657269616C0068656C70006D01
:101650006170006D617070696E67206F66207263E3
:10166000206368616E6E656C206F72646572006DD8
:1016700069786572206E616D65206F72206C697388
:1016800074006D6F746F72006765742F73657420DA
:101690006D6F746F72206F75747075742076616CE5
:1016A00075650070726F66696C6500696E64657857
:1016B00020283020746F2032290073617665007312
:1016C00061766520616E64207265626F6F74006E72
:1016D000616D653D76616C7565206F7220626C612D
:1016E0006E6B206F72202A20666F72206C69737493
:1016F0000073686F772073797374656D20737461FC
:10170000747573004759524F0041434300424152A0
:101710004F00534F4E415200475053004750532BF8
:101720004D4147004144584C333435004D505536F7
:10173000303530004D4D413834357800424D41321E
:101740003830004C534D333033444C48430046410D
:101750004B45004E6F6E650054524900515541444F
:10176000500051554144580042490047494D4241BB
:101770004C005936004845583600464C59494E47AA
:101780005F57494E47005934004845583658004F76
:1017900043544F5838004F43544F464C4154500027
:1017A0004F43544F464C41545800414952504C41CC
:1017B0004E450048454C495F3132305F4343504D00
:1017C0000048454C495F39305F4445470056544115
:1017D000494C340048455836480050504D5F544FEE
:1017E0005F534552564F004455414C434F5054456A
:1017F000520053494E474C45434F505445520043C5
:101800005553544F4D0052585F50504D0056424171
:101810005400494E464C494748545F4143435F4357
:10182000414C0052585F53455249414C004D4F5472
:101830004F525F53544F5000534552564F5F5449D7
:101840004C5400534F465453455249414C004C456B
:10185000445F52494E47004641494C53414645007A
:1018600054454C454D4554525900504F5745524DE3
:101870004554455200564152494F00334400525896
:101880005F504152414C4C454C5F50574D005258AF
:101890005F4D535000525353495F50574D00000065
:1018A00004170108091701080D170108201701087E
:1018B00012170108181701081C1701080000000082
:1018C0005C0F0108020000006C19002000000000FD
:1018D00028230000650F0108000000006E19002099
:1018E0000000000001000000730F0108020000006A
:1018F000721A0020B0040000A4060000790F01084D
:1019000002000000741A002000000000D007000050
:10191000820F010802000000761A0020000000007B
:10192000D00700008B0F010801000000781A00208A
:101930000000000012000000980F010801000000E4
:10194000791A00200000000001000000AA0F010821
:1019500002000000301A002000000000D007000044
:10196000B60F010802000000321A0020000000003B
:10197000D0070000C20F010802000000341A002046
:1019800000000000D0070000CD0F01080200000099
:10199000361A002000000000D0070000DC0F01080C
:1019A00002000000381A002000000000D0070000EC
:1019B000EC0F0108020000003A1A002000000000AD
:1019C000D0070000F60F0108020000003C1A0020BA
:1019D00000000000D00700000A100108020000000B
:1019E0003E1A002032000000007D0000191001089E
:1019F00002000000401A002032000000F201000046
:101A000028100108000000007A1A002000000000E1
:101A10000100000035100108000000007B1A0020C2
:101A200000000000640000004110010801000000F7
:101A30007C1A0020FFFFFFFF010000005710010883
:101A400000000000801A00200000000008000000D4
:101A50006E10010800000000811A00200000000044
:101A6000080000008510010800000000821A002014
:101A700000000000080000009C10010800000000A9
:101A8000831A00200000000008000000B3100108C5
:101A900000000000941A0020300000007E000000CA
:101AA000C410010804000000841A0020B0040000E3
:101AB00000C20100D110010804000000881A0020B3
:101AC000B004000000C20100DE10010804000000A4
:101AD0008C1A00200000000000C20100EB10010879
:101AE00004000000901A0020B004000000C20100B1
:101AF00004110108000000007E1A00200000000010
:101B0000020000001111010800000000701A0020FE
:101B10000000000003000000231101080000000085
:101B2000981A002000000000010000003611010892
:101B300000000000991A00200000000001000000D1
:101B400047110108000000009A1A00200000000060
:101B5000010000005711010800000000641A002075
:101B60000A000000C8000000611101080000000028
:101B7000651A00200A0000003200000074110108FC
:101B800000000000661A00200A0000003200000079
:101B90008711010800000000671A00200000000003
:101BA000090000009911010800000000421A0020FD
:101BB0000000000008000000A4110108000000005F
:101BC000431A00200000000008000000AE110108C8
:101BD00000000000441A002000000000080000007F
:101BE000B811010803000000461A00204CFFFFFF57
:101BF00068010000C911010803000000481A002014
